:100000000C94C7000C94EF000C94EF000C94EF00DC
:100010000C94EF000C94EF000C94EF000C94EF00A4
:100020000C94EF000C94EF000C94EF000C94EF0094
:100030000C9426050C94EF000C94EF000C94EF0048
:100040000C94EF000C94EF000C94FB040C94EF0064
:100050000C94F60C0C94BE0C0C94EF000C94EF0076
:100060000C94EF000C94EF000C94EF000C94EF0054
:100070000C94EF000C94EF000C94EF000C94EF0044
:100080000C94680C0C94EF000C94EF006E616E0001
:10009000696E660000407A10F35A00A0724E18098B
:1000A0000010A5D4E80000E87648170000E40B54DF
:1000B000020000CA9A3B000000E1F50500008096AE
:1000C0009800000040420F000000A08601000000E0
:1000D000102700000000E80300000000640000009A
:1000E00000000A00000000000100000000002C7663
:1000F000D888DC674F0823DFC1DFAE59E1B1B7967E
:10010000E5E3E453C63AE651997696E8E6C28426DA
:10011000EB898C9B62ED407C6FFCEFBC9C9F40F2B6
:10012000BAA56FA5F490055A2AF75C936B6CF96732
:100130006DC11BFCE0E40D47FEF520E6B500D0EDF7
:10014000902E0300943577050080841E080000205F
:100150004E0A000000C80C333333330F986E1283FD
:100160001141EF8D2114893BE65516CFFEE6DB18D1
:10017000D1844B381BF77C1D901DA4BBE424203296
:1001800084725E228100C9F124ECA1E53D2711248F
:100190001FBECFEFD0E4DEBFCDBF14BE88E10FB6E7
:1001A000F89480936000109260000FBE1AE0A0E007
:1001B000B1E0E6EFF8ED00E00BBF02C007900D9252
:1001C000AC3AB107D9F71FE2ACEABAE001C01D9220
:1001D000A13EB107E1F70E940E040C94F4560C9472
:1001E00000008091951E089580E01B9981E008959C
:1001F00029982B988DE090E00197F1F7299A0895BE
:1002000008950895089581E06FE140E00E9460063E
:1002100008950E940301282F8151823058F0223026
:1002200049F0213039F080E090E02E3129F481E06E
:1002300090E0089581E090E00895CF93DF93EC0182
:100240000E940301863021F0813011F084E407C060
:1002500086E06FE140E00E946006888380E4DF91E1
:10026000CF91089588E06FE140E00E946006089514
:1002700086E06FE140E00E9460068093AD0A109234
:10028000301F08951F93CF93DF93EC0114E269911F
:10029000812F0E94FB051F5F1C32C9F7DF91CF91B0
:1002A0001F9108951F93682F192F80E20E94FB056C
:1002B00081E2612F0E94FB051F9108951F93682F13
:1002C000192F82E20E94FB0583E2612F0E94FB0549
:1002D0001F910895282F8EE268E043E00E944106B6
:1002E00008952B988DE090E00197F1F782E06FE19F
:1002F00040E023E00E94410683E090E00197F1F79F
:1003000008950E94F400882311F080E408950E946B
:1003100071018BE490E00197F1F70E9403018830AE
:1003200011F083E408952B9A80E408951F93162F0B
:10033000663010F082E414C0882329F483E068E07A
:1003400043E021E004C083E068E043E020E00E9455
:10035000410683E067E040E0212F0E94410680E4EF
:100360001F9108950E94F400882379F02B9881EE64
:1003700096E00197F1F781E060E00E9496010E940B
:100380000301883011F083E4089580E408951F93F9
:10039000182F803110F082E40DC00E94F4008823F1
:1003A00011F084E407C085E06FE040E0212F0E9457
:1003B000410680E41F9108951F93182F8B508031C0
:1003C00010F082E421C00E94F400882311F084E43C
:1003D0001BC00E9432018117B1F088E06FE140E05C
:1003E000212F0E9441060E940301863011F08930BE
:1003F00021F48DE291E00197F1F70E94320181171B
:1004000011F083E401C080E41F9108958091AC0A4B
:10041000882329F48CE10E9427068093AC0A8091FE
:10042000AC0A0895FF920F931F93082F0E940301B7
:10043000182F0E940602833021F00E9406028730A6
:10044000B1F4163029F4F02EF69410E000E00CC060
:10045000163169F4F8CF86E060E645E00E94600658
:10046000110F110F182B0F5F0F15A8F303C00E9477
:100470004868182F812F1F910F91FF9008951F93A7
:10048000182F0E940602823031F485E060E847E0D0
:10049000212F0E9441060E940602833031F484E03D
:1004A00060E245E0212F0E9441061F9108950F93BD
:1004B0001F93182F883051F0863041F0893031F089
:1004C000863121F0893111F082E455C00E94F40098
:1004D000882311F084E44FC00E9409018823E1F7CA
:1004E0000E940602823039F40E949009882319F094
:1004F000163109F416E00E940301082F1817D1F1F4
:10050000183019F40E9471012FC0193159F4893043
:10051000E1F082E06FE140E029E00E94410606310F
:1005200081F40CC0163189F4893079F082E06FE1F2
:1005300040E029E00E944106093119F483E090E08F
:1005400002C089E691E00197F1F782E06FE140E0B7
:10055000212F0E944106083019F489E691E002C07B
:1005600083E090E00197F1F70E940301811711F0F9
:1005700083E401C080E41F910F910895FF920F93CF
:100580001F93DF93CF9300D00F92CDB7DEB7F82E35
:100590008B019091321F892F8250823010F484E4B5
:1005A00030C0992389F0CB016F2D40E025E738E278
:1005B0000E941720882341F08AE189831B821A82D6
:1005C000CE0101960E941308F7FE02C082E419C012
:1005D0000E9409018823E1F789E10E9457020E94E5
:1005E00003018931C9F7F8018581968190932F1F06
:1005F00080932E1FF2E0FF0EC8016F2D0E94AE0502
:1006000080E40F900F900F90CF91DF911F910F9189
:10061000FF900895DF93CF9300D000D00F92CDB715
:10062000DEB70E9403018A838A81813151F08A8179
:10063000863039F08A81813021F08A81863109F053
:1006400081C08091321F882331F41D821C821B825D
:100650000E94C00520C0833009F4A6C0813079F41F
:100660000E94C00581E090E09D838C838AE18B83AA
:10067000CE0103960E9413081D821C820CC085E7E0
:1006800098E20E947020882309F48EC08AE18B834F
:100690001D821C8252C09091171E80E02091161E70
:1006A000AC01420F511D9A015093171E4093161E24
:1006B00080911B1E8F3F41F480911C1E8F3F21F4BF
:1006C000842F807F09F070C01B8258E821363507DF
:1006D00021F188E82236380740F448E02330340717
:1006E00081F02050304849F512C08CE82336380795
:1006F00001F148EC23363407D1F023563848E9F4A9
:100700000EC08091211F8823C1F085E115C00E9491
:100710009009882391F084E10FC080E10DC08091A1
:100720001F1E823031F08B3B31F0813031F487E194
:1007300003C088E101C089E18B83CE0103960E944A
:10074000130832C08A81823049F08A81823131F0C7
:100750008A81893119F08A81893031F51092301FF0
:100760001B821D821C8282E060EE45E00E946006D2
:1007700089838981833051F0843018F4823050F4B9
:1007800003C0853039F404C081E103C083E101C0B6
:1007900082E18B838B81882321F0CE0103960E9416
:1007A000130886E10E9457020F900F900F900F9050
:1007B0000F90CF91DF9108950E940602823011F4CC
:1007C00086E108958091AD0A0895FF920F931F93DB
:1007D000F82E0DEF13E0C8010197F1F70E948A058A
:1007E0000E94F80082E06FE140E023E00E944106B1
:1007F000C8010197F1F78EE06CE00E94FB0589E0EB
:100800006FE040E027E00E944106FF2011F00E94C7
:10081000840480E41F910F91FF900895109264006A
:10082000109265000E944A0480E090E00E94CC068D
:100830000E94AC0C0E94A54C0E94051778940E945F
:100840009E0F0E945F08FACF9C01F999FECF32BD3E
:1008500021BDF89A80B508959C01F999FECF1FBA81
:1008600032BD21BD60BD0FB6F894FA9AF99A0FBE59
:10087000089584B1806A84B92F9A249A2C9A80E5CD
:100880008CBD81E08DBD08958EBD0DB407FEFDCFFA
:100890008EB5089508959C01CB01B9012CE234E096
:1008A0000E94B6690895DF93CF930F92CDB7DEB75C
:1008B000FC01362FCA012FB72983F894BF01432FBB
:1008C00050E00E944B0489818FBF0F90CF91DF9140
:1008D000089524E234E00E949A690895DF93CF934B
:1008E0000F92CDB7DEB7FC01362FCA012FB729838F
:1008F000F894BF01432F50E00E94690489818FBFA3
:100900000F90CF91DF910895DF92EF92FF920F93B6
:100910001F93DF93CF9300D0CDB7DEB78091AE0A9F
:10092000882311F011E05CC081E08093AE0AD09082
:100930006600F89461E00E949601E090B100F090AA
:100940008100009180001092B100109281001092FD
:10095000800020E030E063E056E04FEF6093B100AC
:10096000509381001092B200109285001092840082
:1009700046BB47BBB89BFECF809184009091850019
:100980009A838983109281001092B10089819A81A3
:100990008A5F934020F48091660081500AC089816B
:1009A0009A818650944010F411E00CC0809166004A
:1009B0008F5F809366002F5F3F4F83E0283E3807AC
:1009C00069F610E081E060E00E949601E092B100DB
:1009D000F092810000938000112311F4D092660000
:1009E000812F0F900F90CF91DF911F910F91FF906A
:1009F000EF90DF9008951F920F920FB60F920BB6F3
:100A00000F9211242F933F934F935F936F937F9394
:100A10008F939F93AF93BF93EF93FF9385B58D7F94
:100A200085BD0E949909FF91EF91BF91AF919F9170
:100A30008F917F916F915F914F913F912F910F9087
:100A40000BBE0F900FBE0F901F9018951F920F9224
:100A50000FB60F920BB60F9211240F931F932F9383
:100A60003F934F935F936F937F938F939F93AF9336
:100A7000BF93EF93FF938FE00E942706082F182F54
:100A800083FF02C00E940A0314FF02C00E9499095A
:100A900012FF10C02C9880E28EBD0DB407FEFDCF72
:100AA0008EB51EBC0DB407FEFDCF8EB52C9A0E94EC
:100AB00038010AC007FF08C08EE00E942706682F91
:100AC0006F778EE00E94FB05FF91EF91BF91AF9190
:100AD0009F918F917F916F915F914F913F912F9156
:100AE0001F910F910F900BBE0F900FBE0F901F9094
:100AF0001895239A219A0E948705EFE6F0E08081FD
:100B00008062808383E480938100B59A08950E9477
:100B1000390408950E9479050E948705EFE6F0E008
:100B200080818062808383E480938100B59A0895F8
:100B30001F93CF93DF93EC01162F2C9880E60E9431
:100B40004404812F0E94440489910E94440411505E
:100B5000D9F72C9ADF91CF911F910895DF93CF930E
:100B60000F92CDB7DEB72FB72983F8942B9A2B9825
:100B70000E94980589818FBF0F90CF91DF910895D2
:100B8000EF92FF921F93DF93CF930F92CDB7DEB713
:100B90008FB78983F8942C9880E20E94440480E007
:100BA0000E944404182F83508D37A8F41093151E0B
:100BB00086E1E82E8EE1F82E80E00E944404F701E1
:100BC00081937F011150C1F780E00E94440480931B
:100BD000951E2C9A07C02C9A1092151E1092951EE5
:100BE0001092961E89818FBF0F90CF91DF911F9138
:100BF000FF90EF9008950F931F93DF93CF930F9281
:100C0000CDB7DEB7062F182F106C8FB78983F894F5
:100C10002C98812F0E944404802F0E9444042C9A17
:100C200089818FBF1F73123061F4602F6F7166303E
:100C300011F0663121F481E08093ED1C02C0109226
:100C4000ED1C0F90CF91DF911F910F9108951F938D
:100C5000DF93CF930F92CDB7DEB7182F10688FB701
:100C60008983F8942C98812F0E944404812F0E943C
:100C700044042C9A99819FBF0F90CF91DF911F91CF
:100C80000895DF92EF92FF920F931F93D82EF62EC6
:100C9000E42E022F0E9427066F2D6095682310E036
:100CA00002C0000F111FEA94E2F7F0226F298D2D88
:100CB0000E94FB051F910F91FF90EF90DF90089528
:100CC000FF920F931F93062FF42E0E9427060823EE
:100CD00010E002C015950795FA94E2F7802F1F9156
:100CE0000F91FF900895009711F48CEE96E0909389
:100CF0000101809300010895009711F48AE097E0C4
:100D000090930301809302010895FC011182818177
:100D100080830895DC019C919F5F97FF05C090E060
:100D200003C0222319F008952091F41D11968C918F
:100D300011979817B1F38C91FD01E80FF11D6283B3
:100D40009C930895DC0111969C911197FD01E90F88
:100D5000F11D22818C91981711F42FEF06C0892F75
:100D60008F5F87FD80E011968C93822F0895FC01A0
:100D70009081818120E0981321E0822F0895FC0169
:100D80008081282F30E08181281B310937FF02C084
:100D900020583F4F822F08950F931F938C018EEEA2
:100DA0009CE10E94850682E79DE10E94850688E914
:100DB0008093C10086E08093C2001092C5008CE051
:100DC0008093C4001093711D0093701D1F910F91AB
:100DD00008951092C1000895682F8091B00A882369
:100DE000C1F4789482E79DE10E948A068091C10057
:100DF00085FD0FC08091C00085FFFCCF82E79DE19B
:100E00000E94A2068093C6008091C10080628093F8
:100E1000C1000895CF93DF93EC0103C00E94EC065C
:100E2000219688818823D1F7DF91CF910895CF93C0
:100E3000DF93EC0102C00E94EC06FE012196849132
:100E40008823C9F7DF91CF9108958EEE9CE10E942F
:100E5000BF0608958EEE9CE10E94BF06089582E7CA
:100E60009DE10E94BF06089582E79DE10E94A206CF
:100E700008958EEE9CE10E94BF068823D1F38EEE8A
:100E80009CE10E94A2060895DF92EF92FF920F93D9
:100E90001F93CF93DF93EC01D42E00E0E62EFF24C6
:100EA0000894E108F1080E943907182F802F90E07C
:100EB0008E159F0534F01D3021F01A3011F01830D6
:100EC00091F7DD2019F0812F0E94EC061A3029F0ED
:100ED0001D3019F0183089F40AC01882802FDF9174
:100EE000CF911F910F91FF90EF90DF900895002315
:100EF000D1F2015018822197D6CF19930F5FD3CF2B
:100F000090E08091B00A882309F491E09093B00AB0
:100F10000895682F81E08093F41D8EEE9CE10E947D
:100F20008A061092F41D08950E942507882309F46B
:100F300045C00E943907282F809110018533E1F0C8
:100F4000863328F4833341F08433A1F509C0863316
:100F5000C9F0873379F526C0213089F484E30FC0C6
:100F6000822F2B3008F08AE08093040185E3809380
:100F700010011092AF0A14C02093050186E38093FC
:100F800010010EC09091AF0A80910401981750F49F
:100F9000E92FF0E0EC5FFE4F22839F5F9093AF0A52
:100FA00080E0089583E38093100180E0243031F4E1
:100FB00081E0089583E38093100180E00895EF922B
:100FC000FF920F931F93CF93DF93082F162F7A0171
:100FD00081E00E94EC06812F0E94EC06802F0E9487
:100FE000EC0600E0C12FD0E006C0EE0DFF1D8081B1
:100FF0000E94EC060F5FE02FF0E0EC17FD07ACF36A
:1010000084E00E94EC06DF91CF911F910F91FF9039
:10101000EF9008959091F51D8091F61D20E09813B2
:1010200021E0822F08950F931F93482F192F0091CD
:10103000F51DE02FF0E02091F61DCF0101966AE04A
:1010400070E00E94C46B30E082179307B9F0DF01B3
:10105000AA0FBB1FAE0FBF1FA950B24E842F912FF6
:101060009C01F90183E001900D928150E1F7802FFE
:101070008F5F8A3008F080E08093F51D1F910F91FB
:101080000895DF93CF930F92CDB7DEB78091F61D11
:101090008983998189818F5F898389818A3008F06A
:1010A000198289818093F61D23E0929F900111247B
:1010B0002950324EC9010F90CF91DF9108951F93AF
:1010C00011E0A1C00E944108FC018081853109F432
:1010D0004DC0863190F4823109F48BC0833130F4F5
:1010E000803151F1813109F08EC086C0833109F41D
:1010F0007DC0843109F087C012C0883109F449C02D
:10110000893130F4863199F0873109F07CC03AC0DA
:10111000893109F464C08A3109F075C070C08091CA
:10112000211F882309F06FC00E94080A6CC001804B
:10113000F281E02D099567C08091211F882309F471
:1011400062C086E19EE10E945D1920911F1E3091D0
:10115000201E8091261F9091271F2817390719F408
:101160000E949B0D50C00E949C1B4DC08091211F6E
:10117000882309F448C081E090E062EB7EE00E94A1
:101180000D0C41C08091211F8823E9F10E94661C4B
:101190003AC08091171E8C38D9F48091161E833680
:1011A000B9F41093211F8091231E9091241E9093D7
:1011B000291F8093281F8091261E9091271E9093AF
:1011C000271F8093261F0E9452010E943B1B1BC0B9
:1011D0008091211F8823B9F00E94A71D14C080911F
:1011E000211F882381F00E94241D0DC00E941A1720
:1011F0000AC00E941D1707C00E949C1704C081816D
:1012000092810E94531F0E940A08882309F05ACF36
:101210001F91089580932D1F0E94DC0108951F9354
:10122000DF93CF93CDB7DEB728970FB6F894DEBF24
:101230000FBECDBF182F8FEF9FEF9093251F809388
:10124000241F9093271F8093261F1092211F909395
:10125000291F8093281F90932B1F80932A1F109281
:101260002C1F1092301F81E08093311F0E94E503F4
:1012700010932D1F1F3F19F0812F0E94DC0181E088
:101280000E943F0288E00E9457020E94020187E10B
:1012900064E042E021E00E94410686E10E9457029C
:1012A00080E090E068E049E15FE10E946E0480E048
:1012B0000E946A018FEF9FEF0E9452018FEF9FEF14
:1012C0000E945E018CE260EF44E022E00E94410651
:1012D0008091191F898380911A1F8A8380911B1F17
:1012E0008B8380911C1F8C8380911D1F8D83809127
:1012F0001E1F8E8380911F1F8F838091201F8887E0
:10130000CE0101960E9442010E94BA1828960FB69B
:10131000F894DEBF0FBECDBFCF91DF911F9108952E
:101320008091B10A0895809311010895809111016F
:10133000089508958091B10A8823B1F08091E01F4B
:10134000882321F085B58D7F85BD08C08EE00E9481
:101350002706682F6F7E8EE00E94FB058091721F2A
:101360000E94150B1092B10A08951F9310E080910E
:10137000601F8F3FE1F011E080915C1F90915D1F35
:101380009093251F8093241F20915E1F30915F1F33
:101390003093291F2093281F0E945E018091601FB7
:1013A0000E940A098091641F8F5F80932C1F812FF8
:1013B0000E946F141F9108952091951E8091171E11
:1013C000829586958695837080935B1F8091191E08
:1013D00090911A1E90935D1F80935C1F80911B1E3D
:1013E00090911C1E90935F1F80935E1F8091201E22
:1013F0008093641F80912D1F81508093601F1092F5
:10140000611F2093651F0E94DC038093661F08956F
:101410001F939091951E20911D1E30911E1E80914C
:10142000B10A882339F14091621F5091631F3093B4
:10143000631F2093621F8091631F87FF05C0509335
:10144000631F4093621F16C08091651F891780F04B
:10145000891781F49091641F8091201E891740F0B4
:10146000981741F41091661F0E94DC03181710F4BE
:101470000E94DC091F91089583E098E09093991EE3
:101480008093981E8091221F80939A1E8F5F809375
:10149000221F8FEF9FEF90939C1E80939B1E909333
:1014A0009E1E80939D1E87E080939F1E88E068E9C2
:1014B0007EE10E94BE02089590912D1F9F3FA9F4E6
:1014C00081E08093B10A86E1EBE5FFE1DF011D9247
:1014D0008A95E9F79093601F8BE080932D1F809190
:1014E0001101803811F080932D1F40912D1F4B3139
:1014F00048F4242F30E08091110190E001962817E4
:10150000390741F41092B10A8FEF80932D1F0E948A
:10151000B5090895842F0E940A090E943C0A80910F
:101520002D1F8F5F80932D1F84E190E06CE57AE0A2
:101530000E940D0C0895DF93CF930F92CDB7DEB7C5
:101540009C01009711F421E030E08FB78983F89473
:10155000309302202093012089818FBF0F90CF917B
:10156000DF910895DF93CF930F92CDB7DEB78FB79A
:101570008983F8942091FF1F3091002089818FBFCB
:10158000C9010F90CF91DF910895DF93CF930F9210
:10159000CDB7DEB78FB78983F8942091E21F3091E1
:1015A000E31F4091E41F5091E51F89818FBFB9016E
:1015B000CA010F90CF91DF9108950F931F93CF939E
:1015C000DF938C010E94B20AE801C80FD91F012BDA
:1015D00029F00E94B20AC817D907D9F7DF91CF9135
:1015E0001F910F9108959091B20A9F5F09F491E0C5
:1015F000E5E0F0E221E08081891709F420E03596EA
:1016000080E2E936F807B9F7E8EEFFE18081891753
:1016100009F420E0359680E2E130F807B9F722239B
:1016200021F39093B20A892F0895982FE5E0F0E214
:1016300020E030E08081891751F4F901EE0FFF1F9F
:10164000EE0FFF1FE20FF31FED5FFF4D16C02F5F80
:101650003F4F35962431310569F7E8EEFFE120E090
:1016600030E08081891769F4F901EE0FFF1FEE0F5A
:10167000FF1FE20FF31FEA51F04E11821082128217
:1016800008952F5F3F4F35962530310551F7089566
:10169000DF92EF92FF920F931F93DF93CF9300D0CF
:1016A0000F92CDB7DEB78091E21F9091E31FA0911A
:1016B000E41FB091E51F0196A11DB11D8093E21FAB
:1016C0009093E31FA093E41FB093E51F8091120154
:1016D0009091130101979093130180931201892B2C
:1016E00049F003E010E236E1D32E7E010894E11CBC
:1016F000F11C27C088EE93E09093130180931201B0
:1017000006EE1FE126E1D22E7E010894E11CF11CB9
:10171000F80180819181009769F00197918380831E
:10172000892B41F4D982838194819B838A83C70169
:101730000E9413080B5F1F4FFFE10F3F1F0741F788
:10174000D0CFF80180819181009769F00197918352
:101750008083892B41F4D982838194819B838A83FE
:10176000C7010E9413080B5F1F4FF0E207361F07E7
:1017700041F70F900F900F90CF91DF911F910F9134
:10178000FF90EF90DF900895EF92FF920F931F93D9
:10179000DF93CF930F92CDB7DEB7AC01009719F46A
:1017A000FB01099531C0E6EEFFE120E080819181E7
:1017B000892B31F5E22EFF248701000F111F000F46
:1017C000111F0E0D1F1D0A51104EF8015183408349
:1017D000748363830E94F30AF80182838FB789833D
:1017E000F8940E94590C89818FBFF701EE0FFF1FFB
:1017F000EE0FFF1FEE0DFF1DEA51F04E828105C076
:101800002F5F3596253091F680E00F90CF91DF91D4
:101810001F910F91FF90EF9008950F931F93DF9307
:10182000CF930F92CDB7DEB7AC01009719F4FB014F
:10183000099538C08FB78983F894E3E0F0E200E0BF
:1018400080819181892B51F5202F30E0F901EE0F35
:10185000FF1FEE0FFF1FE20FF31FED5FFF4DCA01E9
:101860004115510511F481E090E091838083890155
:10187000000F111F000F111F020F131F0D5F1F4DCF
:10188000F801748363830E94F30AF80182830E9443
:10189000590C89818FBFF801828105C00F5F359691
:1018A000043171F680E00F90CF91DF911F910F917D
:1018B00008958091B30A882351F4109295001092F4
:1018C000940082E08093710081E08093B30A0895D0
:1018D0001F920F920FB60F920BB60F9211242F93F7
:1018E0003F934F935F936F937F938F939F93AF93A8
:1018F000BF93EF93FF938091FF1F9091002001967B
:10190000909300208093FF1F8091E21F9091E31F2E
:10191000A091E41FB091E51F0196A11DB11D809318
:10192000E21F9093E31FA093E41FB093E51F0E9472
:10193000480BFF91EF91BF91AF919F918F917F9154
:101940006F915F914F913F912F910F900BBE0F9030
:101950000FBE0F901F901895E1E9F0E080818A603A
:10196000808388EE93E09093990080939800809113
:101970009400909195000E944D6808951F920F92D7
:101980000FB60F920BB60F9211242F933F934F93E4
:101990005F936F937F938F939F93AF93BF93EF93D7
:1019A000FF9382E79DE10E94B706882339F082E722
:1019B0009DE10E94A2068093C60005C08091C100EF
:1019C0008F7D8093C100FF91EF91BF91AF919F9167
:1019D0008F917F916F915F914F913F912F910F90D8
:1019E0000BBE0F900FBE0F901F9018951F920F9275
:1019F0000FB60F920BB60F9211241F932F933F93A4
:101A00004F935F936F937F938F939F93AF93BF9306
:101A1000EF93FF931091C60081E08093F41D8EEE4A
:101A20009CE1612F0E948A061092F41DE091701DC6
:101A3000F091711D309711F0812F0995FF91EF9171
:101A4000BF91AF919F918F917F916F915F914F91D6
:101A50003F912F911F910F900BBE0F900FBE0F90D3
:101A60001F90189508950895DF93CF93CDB7DEB7F3
:101A700060970FB6F894DEBF0FBECDBF81E698E841
:101A80009A8389838091231F8B838F5F8093231F89
:101A90008091241F9091251F9D838C838091261F08
:101AA0009091271F998788879D878C878091B40A9A
:101AB0009091B50A9B878A878091B60A8E870E948B
:101AC000DC038F870E94F100888B8091281F909102
:101AD000291F9F838E8380E1BE016F5F7F4F0E942D
:101AE000BE0260960FB6F894DEBF0FBECDBFCF9199
:101AF000DF910895282F8091261F9091271F681746
:101B0000790789F08091211F882369F07093B50AC5
:101B10006093B40A2093B60A1092B70A0E94340D5B
:101B200081E08093301F08958091971E68E97EE1DF
:101B30000E94BE0208958091231E90E08F779070DE
:101B40008330910571F18430910534F48130910531
:101B500061F00297D9F51EC08530910581F185307D
:101B6000910534F1069791F503C00E94BD140895C4
:101B70004091241E20911D1E30911E1E8091281F11
:101B80009091291F2817390709F5842F90E00E94AA
:101B9000BB1808958091211E9091221E0E94081664
:101BA00008958091211E9091221E0E94BC170895D5
:101BB0008091241E9091251E0E944D1A08956091D7
:101BC000151E605186E19EE10E940D500895CF924E
:101BD000DF92FF920F931F93CF93DF93EC01162FA9
:101BE0006A01F22E2091261F3091271F821793073A
:101BF00009F47CC08FEFCF3FD80709F477C08091FC
:101C0000211F882309F472C081E698E89093991EF9
:101C10008093981E8091231F80939A1E8F5F8093DC
:101C2000231F8091241F9091251F90939C1E8093C9
:101C30009B1E3093A01E20939F1ED093A21EC09384
:101C4000A11E3093A41E2093A31ECE010E949A1BB6
:101C5000A6E0FA1629F4D0939E1EC0939D1E08C0DC
:101C60008091281F9091291F90939E1E80939D1E06
:101C7000F092A51E90E009C0E92FF0E0E856F14E81
:101C8000D6018D916D0186879F5F9117A8F32091F2
:101C90009D1E30919E1E8091261F9091271F281710
:101CA000390721F12F5F3F4F09F1125F1093971E03
:101CB00081E08093301F2F2D2650002361F02230C9
:101CC00018F087E090E002C080E090E00E94DD0A1A
:101CD0000E94940D0BC0223018F087E090E002C003
:101CE00080E090E064E97DE00E940D0CDF91CF91EF
:101CF0001F910F91FF90DF90CF9008950F93022FC7
:101D000025E00E94E70D0F9108950F93DF93CF9385
:101D100000D0CDB7DEB77A83698362E0AE014F5F52
:101D20005F4F26E000E00E94E70D0F900F90CF91EB
:101D3000DF910F9108950F9321E000E00E94E70DDD
:101D40000F9108950F93AC01DC010D900020E9F78D
:101D5000A81B80E090E06A2F27E000E00E94E70DDA
:101D60000F91089580E090E89093991E8093981EBB
:101D70008091221F80939A1E8F5F8093221F8091F3
:101D8000241F9091251F90939C1E80939B1E8091F1
:101D9000261F9091271F90939E1E80939D1E8FEF6C
:101DA00090E09093A01E80939F1E86E08093A11EDA
:101DB00080912C1F8093A21E8BE068E97EE10E9437
:101DC000BE02089508950895089508950895089508
:101DD000089508950895E0910201F091030184E1CE
:101DE00091E00995E0910201F091030184E491E012
:101DF0000995E0910201F091030184E691E00995D3
:101E000008956F927F928F929F92AF92BF92CF92DE
:101E1000DF92EF92FF920F931F93DF93CF93CDB793
:101E2000DEB7A8970FB6F894DEBF0FBECDBFE09126
:101E30000201F091030187E691E009952EEAE22E76
:101E400027E0F22E9EE0C92E95E0D92E4E0108948F
:101E5000811C911C86E7682E81E0782ED7018C9139
:101E60000E942706182FEDB7FEB738970FB6F894E3
:101E7000FEBF0FBEEDBF3196ADB7BEB712969C92B6
:101E80008E92119773826282D582C4828683178272
:101E90000E94066AEDB7FEB738960FB6F894FEBFFB
:101EA0000FBEEDBFE0910201F0910301C40109955D
:101EB00007E0A12EBB24E0910001F0910101C501D2
:101EC000002E02C0959587950A94E2F780FD02C026
:101ED00080E301C081E30995015068F7E0910201B8
:101EE000F091030184E891E009950894E11CF11C4C
:101EF00080E190E0C80ED91E98EDE91697E0F9064A
:101F000009F0ACCFE0910201F091030184E891E087
:101F10000995A8960FB6F894DEBF0FBECDBFCF913E
:101F2000DF911F910F91FF90EF90DF90CF90BF90C6
:101F3000AF909F908F907F906F9008959F92AF92F7
:101F4000BF92CF92DF92EF92FF920F931F93DF9396
:101F5000CF93CDB7DEB7CC54D0400FB6F894DEBFE8
:101F60000FBECDBF809167208823D1F08091230BD5
:101F70008823C1F48091240B882329F00E94150B3B
:101F80001092240B09C0E0910201F091030187E84F
:101F900091E009951092672081E08093230B02C0A5
:101FA0001092230B0E942507882309F485C4809191
:101FB000301F882309F080C40E943907082F112799
:101FC00007FD10950431110511F41092B80A8091A3
:101FD000B80A882321F11092220B8091220BE82F5E
:101FE000F0E0E654F54F00838F5F8093220B843638
:101FF00058F40E942507882339F00E943907082FDA
:10200000112707FD1095E9CF8091200B9091210BAE
:102010006091220B4AEB5AE00E949B0E4DC48091C6
:10202000B90A87FD50C0992787FD90958F779070EA
:10203000892B09F448C0E0910001F0910101802F43
:1020400009950D30110519F00A30110581F48091C0
:10205000220BE82FF0E0E654F54F10828F5F80935B
:10206000220B8091B90A80688093B90A2CC08091B4
:10207000220B0830110539F4E82FF0E0E654F54F53
:102080001082815006C0E82FF0E0E654F54F00833F
:102090008F5F8093220B8091220B843640F08091D9
:1020A000B90A80688093B90A1092220B05C40E9475
:1020B0002507882309F400C40E943907082F112737
:1020C00007FD1095B8CF8091B90A87FF04C0082F8B
:1020D000112707FD1095E0910201F091030184E8BA
:1020E00091E0099509361105A1F10A361105CCF4E4
:1020F0000235110509F48BC3033511054CF40D3479
:10210000110509F4ACC30035110509F0CBC375C343
:102110000335110509F453C30436110509F0C2C390
:1021200010C00437110581F0053711050CF0BAC352
:102130000037110509F40FC30337110509F0B2C3C5
:1021400025C30E94010FAEC30E94BB190E94B018A4
:10215000A9C32DB73EB72A5030400FB6F8943EBF02
:102160000FBE2DBFEDB7FEB731960AEB1AE0ADB743
:10217000BEB712961C930E93119789E991E0938351
:1021800082838091261F9091271F9583848380915D
:10219000281F9091291F9783868380912A1F9091F1
:1021A0002B1F918780870E94066AEDB7FEB73A968B
:1021B0000FB6F894FEBF0FBEEDBFE0910201F091A3
:1021C0000301C801099500D000D000D0EDB7FEB7DB
:1021D0003196ADB7BEB712961C930E93119785EC4E
:1021E00091E09383828380912D1F848315820E94C6
:1021F000066AEDB7FEB736960FB6F894FEBF0FBE6F
:10220000EDBFE0910201F0910301C8010995E09151
:102210000201F091030181ED91E0099500D000D019
:1022200000D0EDB7FEB7319603E31FE1ADB7BEB7FF
:1022300012961C930E9311978DED91E093838283F8
:102240008091241F9091251F958384830E94066AA4
:10225000EDB7FEB736960FB6F894FEBF0FBEEDBFD2
:10226000E0910201F0910301C8010995E09102019A
:10227000F091030184E891E009950E940301082F81
:1022800010E0E0910201F091030180EE91E00995E8
:102290000115110539F4E0910201F09103018FEE6F
:1022A00091E07AC00130110539F4E0910201F0911A
:1022B000030184EF91E070C00230110539F4E09120
:1022C0000201F09103018CEF91E066C00630110528
:1022D00039F4E0910201F091030184E092E05CC0E6
:1022E0000830110539F4E0910201F09103018AE010
:1022F00092E052C00930110539F4E0910201F091E9
:10230000030182E192E048C00131110539F4E09106
:102310000201F091030189E192E03EC00231110512
:1023200039F4E0910201F091030186E292E034C0B9
:102330000631110539F4E0910201F091030183E3C4
:1023400092E02AC00931110539F4E0910201F091BF
:1023500003018EE392E020C00C31110539F4E091C5
:102360000201F091030189E492E016C00D311105DC
:1023700039F4E0910201F091030185E592E00CC08F
:10238000E0910201F09103010E31110519F486E686
:1023900092E002C089E792E00995E0910201F09194
:1023A000030184E891E009951091191FB0901A1F5C
:1023B000A0901B1F90901C1F60911D1F70911E1FED
:1023C00080911F1F9091201F2DB73EB72C50304099
:1023D0000FB6F8943EBF0FBE2DBFEDB6FEB6089403
:1023E000E11CF11CFAEBCF2EFAE0DF2EADB7BEB741
:1023F0001296DC92CE92119722E832E0F7013383F5
:102400002283212F3B2D4A2D592D00E20E9478670F
:10241000C901BA01D70114962C93149715969C9371
:10242000159716964C93169717967C9317971896B0
:102430001C9318971996BC9219971A96AC921A97F2
:102440001B969C920E94066AEDB7FEB73C960FB6AB
:10245000F894FEBF0FBEEDBFE0910201F0910301C1
:10246000C60109958091211F882319F428E932E0DB
:1024700002C02EE932E08DB79EB708970FB6F894E8
:102480009EBF0FBE8DBFEDB7FEB731960AEB1AE0C7
:10249000ADB7BEB712961C930E93119783EA92E0E4
:1024A000938382833583248380912C1F86831782B4
:1024B0000E94066AEDB7FEB738960FB6F894FEBFD5
:1024C0000FBEEDBFE0910201F0910301C801099533
:1024D00088E00E94120200D000D000D0EDB7FEB715
:1024E0003196ADB7BEB712961C930E9311972DEB94
:1024F00032E033832283848315820E94066AEDB71B
:10250000FEB736960FB6F894FEBF0FBEEDBFE09152
:102510000201F0910301C80109950E94060283306F
:1025200059F0873069F0823021F4E6EEAE2EB12CFE
:102530000AC0A82EBB2407C077EEA72EB12C03C07B
:1025400064EDA62EB12CE0910201F09103018BEC19
:1025500092E009958DE10E9427062DB73EB72850DD
:1025600030400FB6F8943EBF0FBE2DBFEDB7FEB79B
:1025700031960AEB1AE0ADB7BEB712961C930E93D4
:10258000119723ED32E033832283B582A4828683C0
:1025900017820E94066AEDB7FEB738960FB6F89418
:1025A000FEBF0FBEEDBFE0910201F0910301C80133
:1025B000099500D000D000D0EDB7FEB73196ADB789
:1025C000BEB712961C930E93119780EE92E0938300
:1025D00082835DEEE52E52E0F52EF582E4820E94C4
:1025E000066AEDB7FEB736960FB6F894FEBF0FBE7B
:1025F000EDBFE0910201F0910301C801099500D0FF
:1026000000D000D0EDB7FEB73196ADB7BEB7129689
:102610001C930E93119781EF92E09383828388E05D
:1026200090E0958384830E94066AEDB7FEB73696E4
:102630000FB6F894FEBF0FBEEDBFE0910201F0911E
:102640000301C801099500D000D000D0EDB7FEB756
:102650003196ADB7BEB712961C930E93119780E0DA
:1026600093E093838283F582E4820E94066AEDB749
:10267000FEB736960FB6F894FEBF0FBEEDBFE091E1
:102680000201F0910301C801099500D000D000D0EB
:10269000EDB7FEB73196ADB7BEB712961C930E9349
:1026A00011978FE093E09383828380E293E0958398
:1026B00084830E94066AEDB7FEB736960FB6F8948B
:1026C000FEBF0FBEEDBFE0910201F091030183E276
:1026D00093E0099580918E2E8F3F71F08E010F5EF1
:1026E0001F4FC8016EE77EE20E94EF5BE09102019E
:1026F000F0910301C80106C0E0910201F0910301CD
:1027000089E393E00995E0910201F091030187E4E8
:1027100093E0099580918E2E8F3F71F08E010F5EB0
:102720001F4FC80167EF7EE20E94EF5BE09102015C
:10273000F0910301C80106C0E0910201F09103018C
:1027400089E393E00995E0910201F091030184E8A7
:1027500091E00995A7C0E0910201F09103018CE599
:1027600093E009958AEB9AE062E341E00E94440716
:102770008AEB9AE00E945868682F8093200B909310
:10278000210B82E0792F0E947A0D8CC0E09102012A
:10279000F091030180E793E009958AEB9AE062E308
:1027A00041E00E9444078AEB9AE00E9458689093A7
:1027B000210B8093200B81E08093B80A73C041EE17
:1027C000E42E4EE2F42E31EDA32E37E0B32E84E159
:1027D00090E00E94411E82E060E070E00E947A0D6D
:1027E000C7010197F1F710E00E945F081F5F1436E0
:1027F000D9F7C5010197F1F7EACFE0910201F09115
:10280000030187E893E009950E9480074BC0E0919F
:102810000201F091030186EA93E009958AEB9AE0C0
:1028200060E17AE00E94EF5BE0910201F091030128
:102830008AEB9AE00995E0910201F09103018DEB9A
:1028400093E0099502C00E9439070E94250788235A
:10285000D1F71092BA0A1092220B82E521C0E091C2
:102860000201F09103018BED93E00995E0910201E3
:10287000F091030188E29AE00995E0910201F0915C
:1028800003018DEB93E0099502C00E9439070E9475
:1028900025078823D1F71092BA0A1092220B8DE4F3
:1028A0008093B90A8091B90A882331F48AEF90E0C5
:1028B0006BEE7EE00E940D0CC45BDF4F0FB6F89408
:1028C000DEBF0FBECDBFCF91DF911F910F91FF9063
:1028D000EF90DF90CF90BF90AF909F9008950F93AF
:1028E0001F93882399F18AE090E06BE675E10E94DE
:1028F0000D0CE0910201F09103018DEE93E009953A
:1029000000D000D000D0EDB7FEB7319603E31FE151
:10291000ADB7BEB712961C930E93119787E094E063
:10292000938382838091601F848315820E94066A4C
:102930008DB79EB706960FB6F8949EBF0FBE8DBF9B
:10294000E0910201F0910301C8010CC088EE93E010
:1029500068EF76E10E940D0CE0910201F091030115
:102960008AE094E009951F910F9108958AE090E024
:1029700064EE7EE00E940D0C08958091231E81304C
:10298000A1F48AE090E064EE7EE00E940D0CE091FC
:10299000151EE051F0E0EA5EF14E1686E09102016C
:1029A000F091030184E29EE10995089580E090E0B2
:1029B00064E045E154E00E949B0E88EE93E066EDF2
:1029C00074E10E940D0C089589E190E064EE7EE0D0
:1029D0000E940D0C08958FE260E00E94FB0582E0EA
:1029E00060E070E00E947A0D84EF91E06BEE74E19C
:1029F0000E940D0C8093240B0895CF92DF92EF92EA
:102A0000FF920F931F93DF93CF93CDB7DEB7289735
:102A10000FB6F894DEBF0FBECDBF6E010894C11C87
:102A2000D11C80E090E068E0A6010E946E0476016F
:102A300086019E01275F3F4FF80180818F3FA9F4F7
:102A40000F5F1F4F02171307B9F727C088E00E94D6
:102A50001202F70181937F01E017F107B9F780E0D7
:102A600090E068E0A6010E94530480E190E062E0FB
:102A7000A6010E946E04F601808191818F5F9F4FB5
:102A800099F484E190E0F6019183808380E190E005
:102A900062E0A6010E94530407C080E00E94E503A3
:102AA00086E00E945702D2CF28960FB6F894DEBF78
:102AB0000FBECDBFCF91DF911F910F91FF90EF908F
:102AC000DF90CF9008958091321F833019F480E019
:102AD0000E949A090895EF92FF920F931F93E0913D
:102AE0000201F09103018AE194E0099500D000D041
:102AF00000D0EDB7FEB7319603E31FE1ADB7BEB727
:102B000012961C930E9311978DED91E0938382831F
:102B100080915E1F90915F1F958384830E94066A57
:102B20008DB79EB706960FB6F8949EBF0FBE8DBFA9
:102B3000E0910201F0910301C8010995E0910201C1
:102B4000F09103018CE294E0099500D000D000D010
:102B5000EDB7FEB73196ADB7BEB712961C930E9384
:102B60001197A7E0EA2EA4E0FA2EF382E282809188
:102B7000601F848315820E94066A8DB79EB70696F1
:102B80000FB6F8949EBF0FBE8DBFE0910201F09189
:102B90000301C8010995E0910201F091030184E36A
:102BA00094E0099500D000D000D0EDB7FEB7319683
:102BB000ADB7BEB712961C930E931197F382E282C3
:102BC0008091641F848315820E94066A8DB79EB728
:102BD00006960FB6F8949EBF0FBE8DBFE09102011E
:102BE000F0910301C801099580915E1F90915F1FCC
:102BF0006091601F0E94461B1F910F91FF90EF9004
:102C0000089581EC60E040E050E00E94DF07089505
:102C10000F931F93DF93CF9300D0CDB7DEB79A8386
:102C2000898381E090E064EE7EE00E940D0CE091EB
:102C30000201F09103018EE394E0099500D000D0E9
:102C400000D0EDB7FEB7319603E31FE1ADB7BEB7D5
:102C500012961C930E93119787E094E093838283DE
:102C600089819A81958384830E94066A8DB79EB775
:102C700006960FB6F8949EBF0FBE8DBFE09102017D
:102C8000F0910301C801099581EC62E0AE014F5F4C
:102C90005F4F0E94DF0769817A8183E00E947A0D8D
:102CA0000F900F90CF91DF911F910F910895DF93B7
:102CB000CF9300D0CDB7DEB71A82198281E090E0C1
:102CC00064EE7EE00E940D0C81EC62E0AE014F5F8D
:102CD0005F4F0E94DF070F900F90CF91DF91089513
:102CE000EF92FF920F931F93E0910201F091030185
:102CF000882309F06FC088E594E0099500D000D0E2
:102D000000D0EDB7FEB7319603E31FE1ADB7BEB714
:102D100012961C930E931197BDEDEB2EB1E0FB2E96
:102D2000F382E2828091281F9091291F95838483EA
:102D30000E94066A8DB79EB706960FB6F8949EBF9E
:102D40000FBE8DBFE0910201F0910301C80109950A
:102D5000E0910201F091030189E694E0099500D029
:102D600000D000D0EDB7FEB73196ADB7BEB7129622
:102D70001C930E931197F382E2828091261F90910B
:102D8000271F958384830E94066A8DB79EB7069697
:102D90000FB6F8949EBF0FBE8DBFE0910201F09177
:102DA0000301C80109958AE090E064EE7EE00E948C
:102DB0000D0C83EC62E046E25FE10E94DF07609168
:102DC000261F7091271F8091241F9091251F0E941C
:102DD000244C09C08EE694E0099588EE93E068EFF4
:102DE00076E10E940D0C1F910F91FF90EF900895D6
:102DF000E0910201F091030184E894E009958FEFDE
:102E00000E940F090E945C0A08950E94E4140E9427
:102E1000FD14E0910201F091030181E994E009952C
:102E20000E94F816E0910201F09103018DEA94E00E
:102E3000099508950E94731E08950F931F930E9491
:102E4000731E0E949009882309F06EC0E091020170
:102E5000F09103018BEB94E0099500D000D000D0F5
:102E6000EDB7FEB7319603E31FE1ADB7BEB71296DB
:102E70001C930E93119787E094E093838283809153
:102E8000250B90E00196958384830E94066A8DB796
:102E90009EB706960FB6F8949EBF0FBE8DBFE09109
:102EA0000201F0910301C80109958091281F9091BA
:102EB000291F00E020912E1F30912F1F281739075E
:102EC00039F401E0C90160E040E050E00E949B0E4F
:102ED0008091250B8F5F8093250B883028F100238C
:102EE00071F01092211F88E00E9412029AE0899FDF
:102EF000C0011124C29668EF76E10E940D0C80910A
:102F00002E1F90912F1F0E947018882369F08091C6
:102F10002E1F90912F1F0E944D1AE0910201F091F7
:102F2000030183EC94E009951F910F9108950E948D
:102F3000D7620E94C86108950E94701E20912E1FC2
:102F400030912F1F8091281F9091291F2817390732
:102F500011F41092250B0895482FA82FB92FFD01C9
:102F600001900020E9F73197EA1BFB0B82EC6E2FF2
:102F7000592F0E94DF070895EF92FF920F931F933E
:102F8000DF93CF9300D0CDB7DEB79A838983E091EA
:102F90000201F09103018BEE94E0099500D000D07E
:102FA00000D0EDB7FEB7319603E31FE1ADB7BEB772
:102FB00012961C930E9311978DED91E0938382836B
:102FC00089819A81958384830E94066A8DB79EB712
:102FD00006960FB6F8949EBF0FBE8DBFE09102011A
:102FE000F0910301C8010995E0910201F0910301FC
:102FF00081E095E009950E94F10000D000D000D05A
:10300000EDB7FEB73196ADB7BEB712961C930E93CF
:10301000119797E0E92E94E0F92EF382E2828483FF
:1030200015820E94066A8DB79EB706960FB6F89471
:103030009EBF0FBE8DBFE0910201F0910301C80158
:103040000995E0910201F091030187E095E009956F
:103050000E94DC0300D000D000D0EDB7FEB731965F
:10306000ADB7BEB712961C930E931197F382E2820E
:10307000848315820E94066A8DB79EB706960FB6A6
:10308000F8949EBF0FBE8DBFE0910201F091030145
:10309000C8010995E0910201F091030184E891E0F3
:1030A000099581EC62E0AE014F5F5F4F0E94DF0740
:1030B0008AE090E064EE7EE00E940D0C0F900F908D
:1030C000CF91DF911F910F91FF90EF900895089598
:1030D00080E090E0089580E008958FEF9FEF0895DD
:1030E0009C01009771F0E9E2FBE0808191818217F9
:1030F000930711F481E0089533968CE0E535F807E5
:10310000A1F780E00895AC010097E1F0A9E2BBE0EF
:1031100020E030E08D919C9111978417950761F420
:10312000F901EE0FFF1FE20FF31FE55DF44F808101
:1031300081FF02C081E008952F5F3F4F1396243630
:10314000310541F780E0089580E090E0089580E047
:1031500090E0089580E090E0089580E090E0089588
:1031600008950895089580E090E00895089580E01E
:1031700090E008950895AC01E9E2FBE020E030E042
:10318000808191818417950759F4F901EE0FFF1F93
:10319000E20FF31FE55DF44F808181608083089525
:1031A0002F5F3F4F33962436310551F70895CF9363
:1031B000DF93EC010E9470188823D1F0E9E2FBE074
:1031C00020E030E0808191818C179D0759F4F9014E
:1031D000EE0FFF1FE20FF31FE55DF44F80818E7F3E
:1031E000808306C02F5F3F4F33962436310551F759
:1031F000DF91CF9108951092280B1092270BE9E2EE
:10320000FBE020E030E00EC080819181A9014F5F9A
:103210005F4F3396892B29F03093280B2093270B8F
:103220000AC09A012436310578F33093280B209395
:10323000270B20E030E0C90108952091270B309141
:10324000280BF901EE0FFF1FE20FF31FE75DF44FAC
:103250000EC080819181A9014F5F5F4F3396892B0A
:1032600029F03093280B2093270B0AC09A012436AB
:10327000310578F33093280B2093270B20E030E0C2
:10328000C901089521E0880F991FFC0163E0EE0F4A
:10329000FF1F6A95E1F7E81BF90BDF0111968181A9
:1032A000882341F019968D919C911A97009719F0F7
:1032B0002F5FE9CF20E0822F0895CF92DF92EF9227
:1032C000FF920F931F93CF93DF936C01DC011B964A
:1032D000ED90FC901C97C7010E947018882309F498
:1032E00041C009E21BE0C0E0D0E0F801808191819B
:1032F0008E159F0569F5FE01EE0FFF1FEC0FFD1FF8
:10330000E55DF44F90E0D6011D968C9187FD91E02C
:10331000990F80818D7F892B8083FE01EE0FFF1F27
:10332000EC0FFD1FE55DF44F908190FF0EC0D601BC
:103330001D968C91863019F49E7F90830FC0C70133
:1033400060E070E00E94850E09C0C7010E94330D45
:1033500021960D5F1F4FC436D10539F6F6018585DC
:103360008F778587DF91CF911F910F91FF90EF901D
:10337000DF90CF900895BF92CF92DF92EF92FF92AD
:103380000F931F93DF93CF93CDB7DEB7E2970FB6BE
:10339000F894DEBF0FBECDBFE0910201F0910301B2
:1033A00088ED97E0099500D000D000D0EDB7FEB7CA
:1033B00031968E010F5F1F4FADB7BEB712961C93AB
:1033C0000E9311979EEEE92E97E0F92EF382E2829A
:1033D0008091261F9091271F958384830E94066AFF
:1033E000EDB7FEB736960FB6F894FEBF0FBEEDBF31
:1033F000E0910201F0910301C801099589E2C82E0C
:103400008BE0D82EB02E012F1E2DEF2CD6018D91E2
:103410009C91009711F100D000D000D0EDB7FEB71D
:103420003196ADB7BEB71196BC92119712960C9318
:103430001283E382958384830E94066AEDB7FEB708
:1034400036960FB6F894FEBF0FBEEDBFE0910201B5
:10345000F09103018B2D902F099583E090E0C80E29
:10346000D91E95E5C9169CE0D90681F6E0910201C6
:10347000F091030185EF97E00995E2960FB6F89475
:10348000DEBF0FBECDBFCF91DF911F910F91FF9097
:10349000EF90DF90CF90BF9008950F931F93CF933D
:1034A000DF93EC01E0910201F091030188EF97E0D6
:1034B000099500D000D000D0EDB7FEB7319603E3F8
:1034C0001FE1ADB7BEB712961C930E9311978FE014
:1034D00098E093838283D583C4830E94066A8DB764
:1034E0009EB706960FB6F8949EBF0FBE8DBFE091B3
:1034F0000201F0910301C8010995E9E2FBE020E037
:1035000030E0808191818C179D0751F4F901EE0F15
:10351000FF1FE20FF31FE75DF44F1182108206C018
:103520002F5F3F4F33962436310559F7DF91CF9106
:103530001F910F910895EF92FF920F931F93CF93D6
:10354000DF937C01C9E2DBE0FE0120E030E0808116
:1035500091818E159F05B1F5F901EE0FFF1FE20F66
:10356000F31FE55DF44F80818C7F8083E091020141
:10357000F091030182E198E0099500D000D000D0DD
:10358000EDB7FEB7319603E31FE1ADB7BEB71296B4
:103590001C930E9311978FE098E093838283F582BA
:1035A000E4820E94066A8DB79EB706960FB6F8941D
:1035B0009EBF0FBE8DBFE0910201F0910301C801D3
:1035C000099552C02F5F3F4F33962436310509F0DD
:1035D000BECFE0910201F091030185E298E00995E8
:1035E00000D000D000D0EDB7FEB7319603E31FE165
:1035F000ADB7BEB712961C930E9311978FE098E06B
:1036000093838283F582E4820E94066A8DB79EB717
:1036100006960FB6F8949EBF0FBE8DBFE0910201D3
:10362000F0910301C801099520E030E0888199817B
:10363000892BA1F4F901EE0FFF1FE20FF31FDF0149
:10364000A75DB44FED92FC92E55DF44F80818C7FD5
:103650008083822F90E00E94B61406C02F5F3F4FF8
:1036600023962436310511F7DF91CF911F910F91E9
:10367000FF90EF9008958091260B0E94150B80918A
:10368000211F91E089270E94701608950F931F93C0
:103690008C01862F0E940A0983E698EC9093991E6C
:1036A0008093981E8091231F80939A1E8F5F809332
:1036B000231F8091241F9091251F90939C1E80931F
:1036C0009B1E10939E1E00939D1EE9E1FFE18081E9
:1036D00080939F1E81818093A01E82818093A11E72
:1036E00083818093A21E84818093A31E8581809311
:1036F000A41E86818093A51E87818093A61E81E0EB
:103700008093A71E1093A91E0093A81E82E08093A9
:10371000AA1E83E168E97EE10E94BE0288EE93E082
:103720006BE37BE10E940D0C8093260B1F910F91A0
:103730000895089580E008950F931F93A7E9BEE1CF
:10374000E5E1FEE182E801900D928150E1F78AE027
:1037500090E064EE7EE00E940D0C8091A11E90919D
:10376000A21E0E947018882349F18091231F809324
:103770009A1E8F5F8093231F8091A11E9091A21E9D
:1037800090939E1E80939D1E8091261F9091271FCF
:103790009093A01E80939F1EE0910201F09103017F
:1037A00088E398E009958091A11E9091A21E0E9445
:1037B0008318882309F46AC041E069C02091281F5A
:1037C0003091291F80919F1E9091A01EE0910201CF
:1037D000F09103018217930709F042C08091231FE3
:1037E00080939A1E8F5F8093231F80912A1F909150
:1037F0002B1F90939E1E80939D1E8091261F90915B
:10380000271F9093A01E80939F1E8EE498E0099539
:1038100000D000D000D0EDB7FEB7319603E31FE132
:10382000ADB7BEB712961C930E93119782E698E03F
:103830009383828380912A1F90912B1F9583848389
:103840000E94066A8DB79EB706960FB6F8949EBF83
:103850000FBE8DBFE0910201F0910301C80115C0B8
:103860008091231F80939A1E8F5F8093231F309334
:103870009E1E20939D1E8091261F9091271F90933E
:10388000A01E80939F1E85E698E0099540E0209158
:103890009D1E30919E1E8091A11E9091A21E4423D8
:1038A00041F04091971E425068E97EE10E94320D3E
:1038B0000AC02F5F3F4F39F08091971E825068E910
:1038C0007EE10E94BE021F910F910895DF93CF9376
:1038D000CDB7DEB765970FB6F894DEBF0FBECDBF8C
:1038E0008091171E883C09F04DC083E698E89A83C2
:1038F00089838091231F8B838F5F8093231F809107
:10390000241F9091251F9D838C838091281F909167
:10391000291F9F838E838091261F9091271F99874F
:10392000888781E08A878091261E9091271E9C8738
:103930008B8780911D1E8D8780911E1E8E878091A2
:103940001F1E8F878091201E888B8091211E898B5E
:103950008091221E8A8B8091231E8B8B8091241E46
:103960008C8B8091281E8D8B85E1BE016F5F7F4F10
:103970000E94BE02E0910201F091030185E798E008
:10398000099559C083E698E89093981E8093971EF6
:103990008091231F8093991E8F5F8093231F8091B6
:1039A000241F9091251F90939B1E80939A1E8091B7
:1039B000281F9091291F90939D1E80939C1E80919B
:1039C000261F9091271F90939F1E80939E1E81E03B
:1039D0008093A01E8091201E9091211E9093A21E84
:1039E0008093A11E8091221E8093A31E8091231E8E
:1039F0008093A41E8091241E8093A51E8091251E75
:103A00008093A61E8091261E8093A71E8091271E5C
:103A10008093A81E8091281E8093A91E8091291E44
:103A20008093AA1E80912A1E8093AB1E85E167E9D0
:103A30007EE10E94BE0265960FB6F894DEBF0FBE0F
:103A4000CDBFCF91DF9108950F93CF93DF939091E6
:103A5000151EE7E9FEE1A5E1BEE182E80D900192C5
:103A60008150E1F78091211F882309F46CC0092F50
:103A70000C500695E02FF0E0EE0FFF1FE056F14EE0
:103A80008081918190932B1F80932A1FE0910201E6
:103A9000F09103018AE898E0099500D000D000D0A9
:103AA000EDB7FEB73196C3E3DFE1ADB7BEB712960F
:103AB000DC93CE93119782E698E093838283809182
:103AC0002A1F90912B1F958384830E94066A8DB7CD
:103AD0009EB706960FB6F8949EBF0FBE8DBFE091BD
:103AE0000201F0910301CE010995023060F183E6F5
:103AF00098E89093991E8093981E8091231F80933D
:103B00009A1E8F5F8093231F0150802F90E0FC014D
:103B1000EE0FFF1FEE55F14E2081318130939E1E36
:103B200020939D1E2091261F3091271F3093A01EA9
:103B300020939F1E2BEB2093A11E0596880F68E90A
:103B40007EE10E94BE02DF91CF910F9108950F9305
:103B50001F93CF93DF938091211F882309F486C0A0
:103B60002091201E3091211E8091261F9091271FA9
:103B700007E91EE12817390709F049C083E69CE8E8
:103B80009093981E8093971E8091231F8093991E77
:103B90008F5F8093231F8091241F9091251F909306
:103BA0009B1E80939A1E8091221E80939C1E809162
:103BB000231E80939D1E8091241E80939E1E8091C3
:103BC000251E80939F1E8091261E8093A01E8091AB
:103BD000271E8093A11E8091281E8093A21E809193
:103BE000291E8093A31E3093A51E2093A41E82E05D
:103BF0008093A61E80912A1E90912B1E9093A81E42
:103C00008093A71E0E949B1A82E1B8012DC0E80193
:103C10002196D801E5E1FEE182E801900D92815004
:103C2000E1F78091231F8A838F5F8093231F809108
:103C30002A1F90912B1F9E838D838091261F909128
:103C4000271F98878F838091A21E9091A31E0E94A8
:103C50007018882331F08091A21E9091A31E9E833C
:103C60008D8386E168E97EE10E94BE02DF91CF91FB
:103C70001F910F9108950895089580E090E00895B0
:103C800008950895CF93DF93EC0181E08093550C64
:103C9000C436D10510F5CE01880F991FDC01E3E091
:103CA000AA0FBB1FEA95E1F7A80FB91FA759BF4D8F
:103CB000FB0180E101900D928150E1F7FE01EE0FD2
:103CC000FF1FCF0123E0880F991F2A95E1F7E80F26
:103CD000F91FE759FF4D518B408BDF91CF9108952C
:103CE0001092550C08958091550C882331F08091E5
:103CF0002E1F90912F1F0E94BB181092550C0895F3
:103D0000DF93CF9300D0CDB7DEB79A838983482F56
:103D10005A81FA01EE0FFF1FCF0123E0880F991F90
:103D20002A95E1F7E80FF91FE759FF4D20893189FE
:103D30002115310509F46BC01092802810927F285C
:103D400080E68093FC281092FF281092FE2889E0DC
:103D5000809300291092012980E48093032981E156
:103D600080930229CA01880F991FFC01A3E0EE0F7E
:103D7000FF1FAA95E1F7E80FF91FA4E0B9E2E759A0
:103D8000FF4D80E101900D928150E1F7A4E1B9E28D
:103D9000E7EFFEE280E101900D928150E1F78A8128
:103DA0008093222989818093232980EF92EB90933D
:103DB000272980932629309324292093252980E0E0
:103DC00099E0909329298093282987E780932C29CB
:103DD00010922B2910922A290E94492280959095B1
:103DE00090932B2980932A29892B31F48FEF9FEF11
:103DF00090932B2980932A2981E390E09093802847
:103E000080937F2881E08093E02F0E94F5560F90E9
:103E10000F90CF91DF9108950F931F93182F092FC3
:103E2000E82FF92FEE0FFF1FCF01A3E0880F991F96
:103E3000AA95E1F7E80FF91FE759FF4D208931896D
:103E40002115310569F19091262980912729821742
:103E5000930731F5612F702F660F771FCB01E3E0D9
:103E6000880F991FEA95E1F7680F791F67597F4D11
:103E700084E199E240E150E00E945969009781F4A1
:103E8000E12FF02FEE0FFF1FCF0143E0880F991FA6
:103E90004A95E1F7E80FF91FE759FF4D118A108A9B
:103EA0001F910F910895DF93CF930F92CDB7DEB797
:103EB0009C018091321F823069F4232B59F486E1F2
:103EC0009EE1BE016F5F7F4F45E758E20E94AC1F45
:103ED0008093151E0F90CF91DF9108951F93182F97
:103EE0008093321F85E797E260E071E045E758E292
:103EF0000E948A1F812F8250823010F486E001C018
:103F000086E10E945702133019F480E00E949A095A
:103F10001F910895FA019183808375836483978349
:103F200086839187808761507040860F971F9383A7
:103F300082830895FC0140855185868197814817C9
:103F4000590728F0481B590B2481358101C09C0179
:103F5000241B350BC9010895CF93DF93EC01DA01DF
:103F60001696ED91FC911797508157FD02C0452F91
:103F700023C08D919C91119717969C938E931697C1
:103F800019969C938E93189780E04EC001961796D1
:103F90009C938E9316972817390738F48D919C912E
:103FA000119717969C938E9316971696ED91FC9108
:103FB000179780818993415016968D919C91179700
:103FC00012962D913C911397442301F70196179671
:103FD0009C938E9316972817390738F48D919C91EE
:103FE000119717969C938E9316971696ED91FC91C8
:103FF00017978081FB01808316968D919C9117976E
:10400000019617969C938E93169712962D913C913C
:1040100013972817390738F48D919C9111971796AB
:104020009C938E931697852FDF91CF910895EF92F1
:10403000FF920F931F93CF93DF938C01F62EE42E04
:10404000E901C9010E949A1F2F2D30E02E5F3F4FDA
:104050008217930710F460E03BC0E885F985F08291
:10406000888599850196998788872A813B812817B9
:10407000390720F488819981998788874F2D14C04A
:10408000D8018C9180838885998501969987888746
:104090002A813B812817390720F4888199819987E3
:1040A00088870F5F1F4F4150E885F985442341F70A
:1040B000E082888599850196998788872A813B8146
:1040C0002817390720F488819981998788876F2D6F
:1040D000862FDF91CF911F910F91FF90EF90089560
:1040E000FF920F931F93CF93DF93EC012C9880E204
:1040F0000E94440480E00E944404F82E83508D37CF
:1041000008F04BC0CE010E949A1F2F2D30E02E5F89
:104110003F4F8217930708F440C0E885F985F08285
:10412000888599850196998788872A813B812817F8
:10413000390720F488819981998788870F2D80E03D
:104140000E944404E885F9858083888599850196D5
:10415000998788872A813B812817390720F488812D
:10416000998199878887015051F70885198580E0E2
:104170000E944404F8018083888599850196998777
:1041800088872A813B812817390720F48881998103
:10419000998788872C9A8F2D02C02C9A80E0DF9116
:1041A000CF911F910F91FF900895FC015381560FFD
:1041B00050938628272F33274281420F409385282A
:1041C000A181A0938428E081E0938328842F90E04C
:1041D0008217930748F48A2F8F5F8093842888235F
:1041E00019F4EF5FE0938328852F90E070708617B5
:1041F000970790F4842F8F5F80938528882361F43C
:10420000809184288F5F80938428882329F480916B
:1042100083288F5F8093832808959C0141505040EC
:10422000460F571FFB010EC0708160E08181DB01EA
:10423000A80FB11D2A0F3B1F2A173B0710F42F5F51
:104240003F4F3296E417F50778F3E417F50749F482
:10425000908180E0280F391F2817390710F42F5F4D
:104260003F4FC9010895AC011092590C20E013C0D2
:10427000E22FF0E0322F3F5FEE0FFF1FE850F74DC7
:10428000808191818417950729F42093590C11821C
:1042900010820895232F223058F32093590C08954B
:1042A000AC011092590C20E012C0E22FF0E0322F46
:1042B0003F5FEE0FFF1FE850F74D80819181892B02
:1042C00029F42093590C518340830895232F2230E1
:1042D00060F32093590C0895BC0180919E28909121
:1042E0009F2844960E94D520E0919E28F0919F2817
:1042F00080918328848B80918428858B8091852868
:10430000868B80918628878B0895282F892F922F5E
:104310000895AF92BF92CF92DF92EF92FF920F93E8
:104320001F93CF93DF93B82EA92E6B0100915A0CE7
:1043300010915B0C7CE2E72E0F5F1F4F8DE7003082
:10434000180710F000E010E1FF2411C0FE9CE0010E
:104350001124C056D74D8DA1882341F0C8010E9479
:104360008521288939892817390731F3F39482E0A8
:10437000F81661F700935A0C10935B0C1092590CCD
:10438000C0E0D0E020E03CE216C0239FF001112401
:10439000E056F74D85A1882321F42093590CEF01B5
:1043A0000EC0873039F4209721F096A18EA189178D
:1043B00008F4EF012F5F223040F32093590C20972F
:1043C00089F182E08DA380915C0C888F80915D0CD7
:1043D000898F80915E0C8A8F80915F0C8B8F84EC2B
:1043E00094E09F8F8E8F99A388A381E090E09D8FAA
:1043F0008C8F1FA281E08EA383E08CA31AA280E1A0
:104400008BA3C8010E948521998B888BDB8ACA8A7D
:10441000DE012B2D3A2DC901FC0180E101900D92A6
:104420008150E1F7CE01DF91CF911F910F91FF9065
:10443000EF90DF90CF90BF90AF9008950F931F93B0
:104440001091002900E09091570C091B11099091DF
:104450000129090F111D9801280F311DC90164E0C0
:1044600079E240E250E00E940D216091570C70E02B
:104470006C5D764DA8010E940D21009719F42FEF75
:104480003FEF03C00E9485219C01C9011F910F913C
:10449000089581E10E941E22089586E00E941E2256
:1044A00008958AE30E941E22089580E090E06CEF58
:1044B00078E248E250E00E940D21009719F42FEFB6
:1044C0003FEF03C00E9485219C01C90108959C0112
:1044D000AB0180E090E0B9010E940D210E9485218E
:1044E0000895EF92FF920F931F939C014427552745
:1044F000F22EE32E00E010E0362F272F40E050E0B0
:10450000A90133272227E22AF32A042B152BB7010E
:10451000C8011F910F91FF90EF900895FC01409109
:104520008128509182282CEF3DE2241B350B621725
:1045300073070CF49B011216130664F42093FE2DEE
:104540003093FF2DE417F50729F0CA01BF01A90137
:104550000E946669089582E08093580CA091570CE0
:104560002A2F30E0F901EC5DF64D8181682F70E073
:10457000B3E0660F771FBA95E1F7695F7F4F42E0BE
:10458000285D3F4F3CC0F901E80FF91FE450F74D9B
:104590008081882319F0813019F42EC04F5F2FC01D
:1045A00090E0807C90708038910549F0803C9105C6
:1045B00049F08034910501F54093580C09C04093AF
:1045C000580C08C04093580C809114298F3F11F467
:1045D00081E00895242F30E040E050E02A0F311DA3
:1045E000411D511D285D3F4F4F4F5F4F84E062E0FA
:1045F0000E94192D82E0089581818E5F480F842FDB
:1046000090E0681779070CF0BECF4093580C80E01B
:1046100008950F931F93CF93DF93C0919E28D0915D
:104620009F28843009F4F5C208E319E210939D280D
:1046300000939C281093822800938128833069F48A
:104640008DA18F70833011F00C94DE2B8C8D9D8D9D
:10465000892B11F00C94DE2B94C0823009F095C0A8
:104660001092802810927F281092FF2D1092FE2D1C
:1046700080915F0C8F5F80935F0C882399F4809109
:104680005E0C8F5F80935E0C882361F480915D0CDB
:104690008F5F80935D0C882329F480915C0C8F5F81
:1046A00080935C0C2DA1273011F0253051F48EA1A0
:1046B0008F5F8EA3883711F00C94DE2B1DA20C9413
:1046C000DE2B222311F40C94DE2B8C8D9D8D892BF7
:1046D00009F452C08EA181508EA38F5F11F00C940B
:1046E000DE2B3FA1383029F02150223048F43530FC
:1046F00039F41DA280E8809397280E94315D00C79D
:10470000353010F080E307C083E090E002C0880FEE
:10471000991F3A95E2F78EA38FA18F5F8FA38DA18A
:1047200090E08F7090708330910501F18430910595
:104730004CF48130910509F491C4029711F00C9466
:10474000DE2B0DC08630910509F4EEC68830910548
:1047500009F4EAC6049711F00C94DE2BE5C6E0914B
:10476000570CF0E0EC5DF64D15867FC484E0809335
:1047700097280E94315D06C72F70233011F00C94EA
:10478000DE2B88E080939728AFC6853021F5E09135
:104790009A28F0919B2880899189892B11F40C9497
:1047A000DE2B10929F2810929E28C8010C979093A0
:1047B0009D2880939C289093822880938128109232
:1047C000FF2D1092FE2D1092802810927F2888E0F5
:1047D000809397281CC28091FC28807F803609F046
:1047E000EDC79091002980E020910129AC01420F92
:1047F000511D9A0180917F289091802884179507F8
:1048000008F4DCC7285D3F4F3093802820937F2831
:10481000809104298F3F09F4D1C7C801849760E8CB
:1048200040E00E94C943892B09F067C0C801849702
:104830000E942E44882309F060C0809114298F3F84
:1048400009F058C080911529823009F053C0809139
:10485000162990911729892B09F04CC080911829AD
:1048600090911929892B01F580911A2990911B2982
:10487000892BD1F480911C2990911D29892BA1F4B9
:1048800080911E2990911F29892B71F480912029F4
:1048900090912129892B41F480912229882321F4A8
:1048A00080912329813049F180911829909119290B
:1048B000892B01F580911A2990911B29892BD1F41C
:1048C00080911C2990911D29892BA1F480911E298A
:1048D00090911F29892B71F4809120299091212991
:1048E000892B41F480912229882321F48091232966
:1048F000823019F00E94ED2B69C782E099E2909313
:104900009928809398281092570C1092560CE09199
:104910009828F091992880818B3209F44BC08C3211
:1049200048F4863009F4E0C1813109F4B1C088232C
:1049300089F06BC08A3309F474C08B3320F48C3255
:1049400009F063C03BC78B3309F438C78C3309F0D7
:104950005CC006C08091560C80FD57C0816009C0C4
:104960008091560C81FF04C086FD4FC0806401C059
:1049700082608093560C0E94AB22813009F41EC7DE
:10498000813018F0823019F621C72091570CE22FA0
:10499000F0E0CF018C5D964D9093992880939828F4
:1049A000285FFC018181880F880F880F280F2093D2
:1049B000570CADCF8091560C82FD27C08460809348
:1049C000560C9091570CE92FF0E0DF01AC5DB64D2D
:1049D00013968C911397882349F0BA969F01442728
:1049E00037FD4095542F84E060E018C0B0939928BB
:1049F000A0939828985FEC5DF64D8181880F880F11
:104A0000880F980F9093570C82CFEC5FF8429F016C
:104A1000442737FD4095542F84E061E00E94192D12
:104A2000D5C60E9451228F5F9F4F09F0C7C6E09103
:104A3000570CF0E0EC5DF64DE081E538A9F0E63882
:104A400018F4E038C9F413C0E73829F0E73848F023
:104A5000E83891F403C00E942F3C12C00E94CB3A68
:104A60000FC00E9424350CC00E94884009C00E94DB
:104A700057160E94F82D04C01092802810927F28AB
:104A800080917F2890918028892B09F497C69EC633
:104A900080917F2890918028C09790938028809360
:104AA0007F288CE299E290939D2880939C28E09146
:104AB000570CF0E0EC5DF64D86819781892B31F043
:104AC0000E9449228F5F9F4F09F078C680E09EE2E6
:104AD00090939B2880939A284BC028893989211567
:104AE000310509F440C08091570CE82FF0E0EC5DEF
:104AF000F64D8281938182179307A9F52A893B8914
:104B00002115310529F0808191818217930759F58C
:104B100088819981892BE9F48A819B81892BC9F449
:104B20008C819D81892BA9F48E819F81892B89F4A9
:104B300088859985892B69F48A859B85892B49F419
:104B40008C859D85892B29F48E859F85892B09F479
:104B500049C084E099E2BE0140E150E00E945969F9
:104B6000009709F43FC06996D0939B28C0939A2878
:104B7000C0919A28D0919B28BEE2C233DB0708F48B
:104B8000ACCFE091570CF0E0EC5DF64D8281938163
:104B9000998B888B808191819B8B8A8B20919A281D
:104BA00030919B28C901DC01E4E0F9E280E1019049
:104BB0000D928150E1F782E0809397288CE299E290
:104BC00090939D2880939C2890938228809381289D
:104BD00080917F2890918028C0979093FF2D80939B
:104BE000FE2D15C010929F2810929E2882E080937F
:104BF00097288CE299E290939D2880939C2890932B
:104C00008228809381281092FF2D1092FE2D0E9401
:104C10002E5A2091FE2D3091FF2D2115310509F4DA
:104C2000CDC5C901C0969093802880937F28285FC6
:104C30003F4F30930029885280930129A0919A28F0
:104C4000B0919B2854968C9154978093032981E1CD
:104C500080930229E091570CF0E0EC5DF64D34832F
:104C600025831782168250968D919C91519791833E
:104C7000808352968D919C91539793838283A4E174
:104C8000B9E220919A2830919B28C901FC0180E16A
:104C900001900D928150E1F784E099E264E179E2BC
:104CA0000E94AA4188E399E290939D2880939C28D2
:104CB0008091570CC82FD0E0CC5DD64D0E94492280
:104CC000809590959F838E838091570CE82FF0E01C
:104CD000EC5DF64D86819781892B09F065C58FEFD4
:104CE0009FEF9783868360C50E944D228F5F9F4F01
:104CF00009F064C58091570C082F10E00C5D164D2B
:104D0000C0EAD8E28DA18823D9F0D80112962D915E
:104D10003C911397888999892817390789F42D912F
:104D20003C918A899B892817390751F484E099E2DC
:104D3000BE0140E150E00E945969009709F4B2C1F8
:104D4000AC96B8E2CC3CDB07E9F2E0F2F8018585ED
:104D50008F73823001F5828193819093620C8093EE
:104D6000610C1092590C13C0E42FF0E0EE0FFF1FFE
:104D7000E850F74D2091610C3091620C8081918157
:104D80002817390709F489C04F5F4093590C4091A7
:104D9000590C423048F38091570CE82FF0E0DF01C6
:104DA000AC5DB64D1D968C911D9782FD07C584E1C3
:104DB0001D968C931D978CE390E0909380288093B0
:104DC0007F28FD0180E5848797811B968C911B9736
:104DD00017968C931797938796811A968C911A97AA
:104DE00016968C9316979287958119968C911997A0
:104DF00015968C931597918794819093590C1896DA
:104E00008C91189714968C93149790871B968C917D
:104E10001B978F5F1B968C931B978823C1F41A9660
:104E20008C911A978F5F1A968C931A97882379F42E
:104E300019968C9119978F5F19968C9319978823DF
:104E400031F418968C9118978F5F18968C93E09197
:104E5000570CF0E0DF01AC5DB64D2D913C91119700
:104E60003093620C2093610CFD01828193819183C8
:104E7000808313963C932E931297E4E1F9E2DF01CD
:104E8000509780E10D9001928150E1F784E099E222
:104E900064E179E20E94AA4154C41092590CC0E026
:104EA000D0E04CE250E03CE225C0822F90E0849FAD
:104EB000F001859FF00D949FF00D1124E056F74D01
:104EC00085A1882339F48CE2289FE0011124C05683
:104ED000D74D14C0873059F4209721F096A18EA1A8
:104EE000891728F4239FE0011124C056D74D2F5F66
:104EF0002093590C2091590C2230B8F2209709F4D4
:104F00005DC4D0939F28C0939E2883E08EA38CA37A
:104F10001AA284E08BA31FA2E091570CF0E0EC5D95
:104F2000F64D82819381998B888B808191819B8BB7
:104F30008A8BDE01E4E0F9E280E101900D9281507C
:104F4000E1F781E08DA380915C0C888F80915D0CEE
:104F5000898F80915E0C8A8F80915F0C8B8F81E0AE
:104F600090E09D8F8C8FE091570CF0E0EC5DF64D5A
:104F700087818F8BE091570CF0E0EC5DF64D8681D8
:104F80008E8BE091570CF0E0EC5DF64D85818D8BBA
:104F9000E091570CF0E0EC5DF64D84818C8B81E064
:104FA00090E00E946C21E091570CF0E0EC5DF64D32
:104FB000848590E0807F9070813591050CF44EC01F
:104FC0001092590C35C0F901E450F74D84AD80932F
:104FD000600C882309F442C0813021F44F5F409374
:104FE000590C26C08230C1F485AD8430A9F436ADA9
:104FF00020E087AD90E0822B932B9093620C8093FE
:10500000610CF4E0853C9F0710F084EC94E09F8FE6
:105010008E8F99A388A322C08091590CE82FF0E0CD
:10502000E75CF64DE081EE23C9F0E80FE093590C00
:105030004091590C242F30E0E091570CF0E0EC5DEA
:10504000F64D848582958F7090E00597880F991FA3
:10505000880F991F281739070CF4B5CFE091570C2A
:10506000F0E0EC5DF64D80E18587E091570CF0E0D3
:10507000DF01AC5DB64D1D968C911D9782601D962B
:105080008C931D97FD0182E0848B84E0858B868B59
:1050900084EC878B80E490E09093802880937F2835
:1050A00080E60EC3D0939F28C0939E281092972825
:1050B0008091570CA82FB0E0FD01EC5DF64D858581
:1050C00082FF03C01DA280E293C2848582958F7007
:1050D000880F880F8093590C20917F283091802869
:1050E00028523040281B31093093802820937F2894
:1050F0008DA18F70823039F4AC5DB64D1D968C91C8
:105100008F73823139F1232B59F4E091570CF0E081
:10511000EC5DF64D858590E083709070892BD1F021
:105120008091570CE82FF0E0EC5DF64D94818C896E
:10513000981709F0B2C295818D89981709F0ADC210
:1051400096818E89981709F0A8C297818F89981740
:1051500009F0A3C2E091570CF0E0EC5DF64D8585B7
:1051600084FF52C06C8D7D8D6115710509F44CC0B2
:10517000CE0148960E94D5208091570CE82FF0E090
:10518000EC5DF64D2085809183282817E9F59185FF
:10519000809184289817C1F5928580918528981769
:1051A00099F5938580918628981771F5288F8091BD
:1051B0008428898F809185288A8F809186288B8F7B
:1051C0008FA18823D1F42AA19CA18EA1981B822FA4
:1051D000869586958695981B392F320F3AA38BA119
:1051E000282F26952695821B97FD9195890F8BA3D5
:1051F000369536953695830F8CA381E0809397285A
:105200008CA18EA31D8E1C8E8DA1282F30E0C9018C
:105210008F7090708430910509F4EFC1853091054D
:105220005CF48230910591F1833091050CF0CAC095
:10523000019709F0C3C210C08630910509F425C258
:10524000863091050CF4FDC18730910509F425C223
:10525000089709F0B3C2C6C18091972880FFAEC2FB
:1052600083E08DA380E4809397281D8E1C8E20916F
:105270007F28309180282115310509F431C182E45D
:1052800080939728C9010E946C212AC18091972898
:1052900080FF8DC08091570CE82FF0E0EC5DF64D5B
:1052A00085858F73823109F082C0848590E0807F8C
:1052B0009070813591050CF44EC01092590C35C098
:1052C000F901E450F74D84AD8093600C882309F414
:1052D00042C0813021F44F5F4093590C26C0823088
:1052E000C1F485AD8430A9F436AD20E087AD90E0FF
:1052F000822B932B9093620C8093610C24E0853C6D
:10530000920710F084EC94E09F8F8E8F99A388A36E
:1053100022C08091590CE82FF0E0E75CF64DE08167
:10532000EE23C9F0E80FE093590C4091590C242F5B
:1053300030E0E091570CF0E0EC5DF64D848582950D
:105340008F7090E00597880F991F880F991F281775
:1053500039070CF4B5CF83E08DA3E091570CF0E052
:10536000EC5DF64D84818C8BE091570CF0E0EC5DA8
:10537000F64D85818D8BE091570CF0E0EC5DF64D9C
:1053800086818E8BE091570CF0E0EC5DF64D8781C5
:105390008F8B81E090E00E946C2182E480939728BB
:1053A0001D8E1C8E1092802810927F2899C080E25A
:1053B000809397280E94315DE0919E28F0919F286C
:1053C00015A2E9CC8091570CE82FF0E0EC5DF64D8A
:1053D000858580FF25C024FD23C08C8D9D8D892B64
:1053E00009F0ECC180917F289091802801960E945D
:1053F0006C2120919728822F80618093972880913B
:105400007F2890918028892B19F02261209397287A
:105410000E94315D81E090E09D8F8C8F88E082C09A
:1054200085FF25C0328920E0838990E0282B392B25
:1054300080919C2890919D28820F931F90939D2886
:1054400080939C28E091570CF0E0EC5DF64D32899A
:1054500020E0838990E0282B392B80917F28909140
:105460008028821B930B9093802880937F28209123
:105470007F28309180282115310559F08DA184FDB8
:1054800008C080919728826080939728C9010E9464
:105490006C21E091570CF0E0EC5DF64D968580E0D4
:1054A0002785820F911D9093620C8093610C28A137
:1054B00039A12817390710F0892B21F43093620C99
:1054C0002093610C8091610C9091620C9F8F8E8F64
:1054D0008091972890E083709070892B09F46EC1B9
:1054E0001092FF2D1092FE2D0E94315D8091972821
:1054F000282F85FF0CC01092FF2D1092FE2D1DA2AB
:10550000E091570CF0E0EC5DF64D84E1CCC084FFF7
:1055100012C01092FF2D1092FE2D81E090E09D8F21
:105520008C8F84E08DA31FA2E091570CF0E0EC5D1E
:10553000F64D81E1B8C08091FE2D9091FF2D892B11
:1055400001F120FF02C01D8E1C8E8C8D9D8D009759
:10555000A1F42E8D3F8D8091FE2D9091FF2D281767
:10556000390720F43093FF2D2093FE2D8091FE2DDE
:105570009091FF2D9D8F8C8F04C09093FF2D809371
:10558000FE2D1FA2809181289091822890939D28C2
:1055900080939C288091FE2D9091FF2D892B81F086
:1055A0008C8D9D8D009761F0CC9690938028809390
:1055B0007F28E091570CF0E0EC5DF64D88E110C0DB
:1055C0008091972881FFFAC08CE390E09093802827
:1055D00080937F28E091570CF0E0EC5DF64D80E180
:1055E000858768C08091972880FFE8C01DA280E170
:1055F000809397280E94315DE1C080917F2890912F
:105600008028009711F00E946C21E091570CF0E087
:10561000EC5DF64D85859091972880FF0BC090FF3B
:1056200006C087E08DA31EA21D8E1C8E1DC086E0C5
:105630008DA31AC090FF22C085E08DA31D8E1C8E05
:10564000BDC080917F2890918028009711F00E9422
:105650006C21E091570CF0E0EC5DF64D858580FF04
:105660000DC087E08DA31EA281E090E00E946C2116
:1056700080E1809397280E94315D0FC080917F2840
:1056800090918028892B49F499C08091972880FFB8
:1056900095C087E08DA31EA291C0E091570CF0E069
:1056A000EC5DF64D80E185878CE390E09093802857
:1056B00080937F28E091570CF0E0EC5DF64D80E59B
:1056C0008487E091570CF0E0EC5DF64D8C89808783
:1056D0008D8981878E8982878F898387888D84834E
:1056E000898D85838A8D86838B8D878386E08093E1
:1056F000022988899989918380838A899B899383E8
:105700008283A4E1B9E2FE0180E101900D92815013
:10571000E1F784E099E264E179E20E94AA418DA177
:10572000E091570C84FF06C0F0E0EC5DF64D178663
:10573000168607C0F0E0EC5DF64D84E0868784ECC9
:1057400087878091E02F90E029E730E0829FF00189
:10575000839FF00D929FF00D1124E55BF14D848144
:105760008093032980917F28909180288897909337
:10577000002980917F28885280930129E091570C5D
:10578000F0E08F010C5D164DD80153961C92539793
:1057900052961C92F801118A108A0E944D2280951F
:1057A0009095F801918B808B80E68093FC28109275
:1057B000FD281092FF281092FE2808C01092802821
:1057C00010927F281092570C1092560C1092972826
:1057D000DF91CF911F910F9108951F931091E02FAA
:1057E000212F30E089E790E0289FF001299FF00DFC
:1057F000389FF00D1124E55BF14D8389882399F1E1
:10580000809114298E3F29F480911529803819F44C
:105810002AC08F3F41F11092E02F0BC084E199E242
:105820000E94AD328823C1F48091E02F8F5F809376
:10583000E02F8091E02F823088F327C00E94E42E71
:10584000892B51F48091E02F8F5F8093E02F80911E
:10585000E02F823098F31CC08091032981508093FF
:105860000329882329F41092802810927F2816C0DB
:105870008CEF98E2489660E840E00E94C943892B8B
:1058800069F081E00E94092309C01092E02FDFCF68
:105890001092802810927F281093E02F1F91089576
:1058A000EF92FF920F931F93CF93DF938C017B01B5
:1058B000C0915A0CD0915B0C21968DE7C030D8076F
:1058C00010F0C0E0D0E1CE010E9485219C018091C2
:1058D000102E9091112E8217930771F38091292E2B
:1058E00090912A2E8217930739F3C0935A0CD093C4
:1058F0005B0C1092590C20E049E150E01CC0322FA3
:105900003F5F822F90E0849FF001859FF00D949F70
:10591000F00D1124E050F24D80899189892B51F4CA
:105920002093590C89E1289FD0011124A050B24D39
:1059300049F434C0232F223010F32093590CA0E0F7
:10594000B0E02CC05096DC9350975196CC93519771
:105950005396FC92EE9252970115110531F480E1B5
:10596000ED0119928A95E9F707C0ED01F80180E190
:10597000019009928150E1F78091E02F90E029E7B2
:1059800030E0829FF001839FF00D929FF00D112473
:10599000E55BF14D848154968C935497CD01DF9152
:1059A000CF911F910F91FF90EF9008950F930E9458
:1059B000A5470E94863480E009C0E82FF0E0EE0F92
:1059C000FF1FE850F74D118210828F5F8230A8F3DD
:1059D00020E04CE250E00DC0822F90E0849FF00167
:1059E000859FF00D949FF00D1124E056F74D15A200
:1059F0002F5F223088F380E094E090935B0C8093DB
:105A00005A0C20E049E150E00EC0822F90E0849FC4
:105A1000F001859FF00D949FF00D1124E050F24DA0
:105A2000118A108A2F5F223080F32093590C0F9136
:105A30000895CF92DF92EF92FF920F931F93CF932F
:105A4000DF93D82EC62E79018A011092570CA3E657
:105A5000BCE0E4E1F9E280E101900D928150E1F7D0
:105A600080917F2890918028C09690938028809381
:105A70007F288150954030F080E095E09093802819
:105A800080937F286CEF78E240917F2850918028A6
:105A900040535040CB01C0960E946F6980E68093CE
:105AA000FC281092FD281092FF281092FE288AE30D
:105AB000809302298091E02F90E029E730E0829FD7
:105AC000F001839FF00D929FF00D1124E55BF14DE5
:105AD0008481809303298091042990910529892B41
:105AE00051F58091062990910729892B21F5809104
:105AF000082990910929892BF1F480910A29909124
:105B00000B29892BC1F480910C2990910D29892BA7
:105B100091F480910E2990910F29892B61F4809145
:105B2000102990911129892B31F48091122990919B
:105B30001329892BD1F0E4E1F9E2DF01509780E1EC
:105B40000D9001928150E1F78091630C8F3F91F4A9
:105B500084E0D81651F422E0C21639F484E099E2C8
:105B600063E67CE00E94AA410EC010928028109249
:105B70007F2835C0A4E0B9E2E3E6FCE080E10190D3
:105B80000D928150E1F7E091570CCE2FD0E0FE014D
:105B9000EC5DF64DD082C182C801B7010E9471222E
:105BA000C85DD64D688379838A839B8380917F28E3
:105BB00090918028889790930029889688528093A6
:105BC00001298091570CC82FD0E0CC5DD64D1B82A7
:105BD0001A820E945122809590959B838A83DF913F
:105BE000CF911F910F91FF90EF90DF90CF9008958C
:105BF0004CEF58E28091E02F90E029E730E0829F5F
:105C0000F001839FF00D929FF00D1124E55BF14DA3
:105C1000848180930329809114298F3F81F4DA01D4
:105C20005896FA01389680E101900D928150E1F783
:105C300084E099E264E179E20E94AA411BC0A3E6F4
:105C4000BCE0FA01389680E101900D928150E1F7B5
:105C5000E4E0F9E2DF01509680E10D90019281507D
:105C6000E1F7A4E1B9E2E3E6FCE080E101900D9206
:105C70008150E1F76091570C662301F18AE380932C
:105C8000022970E040917F2850918028461B570BD5
:105C90005093802840937F284852504050930029C9
:105CA000485D5F4F842F885280930129685D764D4F
:105CB0004C52504088E299E20E946F691092570C52
:105CC00081E8809324291092252910922729109287
:105CD00026290E94512280959095909327298093A0
:105CE000262908952091E02F30E040E0ABE0B0E0BD
:105CF00086E190E0289FB001299F700D389F700DBC
:105D000011240FC0842F90E08A9FF0018B9FF00D2B
:105D10009A9FF00D1124E60FF71FE558F24F1286F7
:105D20004F5F423078F340932F0E0895CF93DF9367
:105D3000DC011092350E1092340E10922F0E5091FD
:105D4000E02F252F30E040E0CBE0D0E086E190E08E
:105D5000289FB001299F700D389F700D112429C014
:105D6000842F90E08C9FF0018D9FF00D9C9FF00D93
:105D70001124E60FF71FE558F24F82858823C1F002
:105D8000808191818A179B0799F440932F0E8BE0B5
:105D9000489FC001112426E1529F90011124820FD7
:105DA000931F8558924F9093350E8093340E05C003
:105DB0004F5F4230A8F240932F0E8091340E9091A5
:105DC000350EDF91CF9108950F931F93CF93DF93FB
:105DD0001092350E1092340E10922F0E9091E02FEB
:105DE000292F30E086E1989FD001112440E050E057
:105DF00060E00BE010E086E190E0289FE001299F41
:105E0000D00D389FD00D11242BE035C0862F90E0A7
:105E1000809FF001819FF00D909FF00D1124EC0FF9
:105E2000FD1FE558F24F8285882321F10190F08112
:105E3000E02D3097F9F0818D882311F0853059F4E9
:105E400041155105B9F4629FA00111244A0F5B1F4F
:105E50004558524F0FC060932F0E8BE0689FC001D2
:105E600011248A0F9B1F8558924F9093350E809373
:105E7000340E09C06F5F623048F25093350E409384
:105E8000340E60932F0E8091340E9091350EDF9179
:105E9000CF911F910F910895FC0112860190F0811E
:105EA000E02D818D853009F413A60895FC0181A1B0
:105EB0008D7F81A308952091E02F84E4289F900195
:105EC00011242955324FC90108956F927F928F9204
:105ED0009F92AF92BF92CF92DF92EF92FF920F9379
:105EE0001F93CF93DF931092350E1092340E909142
:105EF000E02F292F30E086E1989FE001112440E057
:105F000050E060E00BE010E086E190E0289FD001D7
:105F1000299FB00D389FB00D11242BE018C0862F9B
:105F200090E0809FF001819FF00D909FF00D112473
:105F3000EA0FFB1FE558F24F8285813039F4629FEA
:105F4000A00111244C0F5D1F4558524F6F5F623006
:105F500030F35093350E4093340E1092330E10925E
:105F6000320E10922F0E8CE2A82EB12C04E8C02E17
:105F7000D12C1CE2712EB4E86B2EA2E08A2EF9E738
:105F8000EF2EF12CE4E09E2EBEC05091E02F252F85
:105F900030E0842F90E08A9DF0018B9DF00D9A9D5A
:105FA000F00D11242C9DC0012D9D900D3C9D900D58
:105FB0001124E80FF91FED58F34F83A5813009F044
:105FC0009DC0479DE0011124569DC0011124C80FBA
:105FD000D91FCD58D34FD093330EC093320E898D35
:105FE0008130E9F0813030F0833039F1843009F0CC
:105FF00085C035C08AA5833010F013A67FC0CE01BE
:1060000082960E943F49892B09F478C04091320E54
:106010005091330E80E090E060E070E03EC0CE0131
:106020004A960E943F49892B09F468C0E091320EDC
:10603000F091330E818E12A661C0CE014A960E9465
:106040003F49892B09F45AC0E091320EF091330E8A
:10605000918E12A680E090E0BF01AF011EC08AA51C
:10606000833070F01AA6CE010E94962E9093350EC2
:106070008093340E009711F00E944C2F1BA63EC057
:10608000CE0182960E943F49892BC1F14091320E88
:106090005091330E80E090E0BA010E94C239009125
:1060A000320E1091330E8091E02F90E08E9DF00122
:1060B0008F9DF00D9E9DF00D1124E55BF14D6585E2
:1060C00076858785908928EE33E040E050E00E9495
:1060D000D76BCA01B90128EE33E040E050E00E94DE
:1060E000A56BAB01BC01C80182960E945949E091A1
:1060F000320EF091330E82A58F5F82A780912F0E12
:106100008F5F80932F0E40912F0E433008F43DCFC8
:106110001092310E1092300E81E080932F0EC4E465
:10612000D0E002E214E440C05091E02F252F30E08F
:10613000842F90E0FC0175E0EE0FFF1F7A95E1F7E8
:10614000880F991FE80FF91F2C9FC0012D9F900DFC
:106150003C9F900D1124E80FF91FE853F24F808106
:1061600081FF1DC0409FF0011124519FC0011124E7
:10617000E80FF91FE955F24FF093310EE093300E1E
:1061800081A180FD0CC0CF0141960E943F49892B1F
:1061900031F08091300E9091310E0E94562F8091F7
:1061A0002F0E8F5F80932F0E40912F0E423008F4F8
:1061B000BBCFDF91CF911F910F91FF90EF90DF90B8
:1061C000CF90BF90AF909F908F907F906F900895E9
:1061D000AF92BF92CF92DF92EF92FF920F931F93F5
:1061E000CF93DF93182FB92EA62E69017A01109252
:1061F000310E1092300E81E080932F0E8091E02FAF
:1062000090E041E024E430E0829FB001839F700D74
:10621000929F700D112419C0242F2F5F842F90E0BE
:10622000FC0155E0EE0FFF1F5A95E1F7880F991F0B
:10623000E80FF91FE60FF71FE853F24F808181FD49
:1062400003C040932F0E0CC0422F423028F34093DE
:106250002F0E423029F40E94486881E080932F0E6F
:1062600090912F0E82E2989FF00111248091E02FEF
:1062700024E4829FC0011124E80FF91FE955F24F71
:10628000F093310EE093300EEF01212F3B2DC90129
:10629000DC0180E10D9009928150E1F7A08AC114E0
:1062A000D104E104F10469F0CF014196B701A601E0
:1062B0000E945949E091300EF091310E81A18E7FFC
:1062C00002C081A1816081A32091E02F30E0609124
:1062D0002F0E862F90E0FC01B5E0EE0FFF1FBA9560
:1062E000E1F7880F991FE80FF91F84E490E0289FD9
:1062F000A001299F500D389F500D1124E40FF51F68
:10630000E853F24F80818260808300FF13C0862FA4
:1063100090E0FC0175E0EE0FFF1F7A95E1F7880F22
:10632000991FE80FF91FE40FF51FE853F24F808122
:10633000846012C0862F90E0FC0135E0EE0FFF1F55
:106340003A95E1F7880F991FE80FF91FE40FF51F41
:10635000E853F24F80818B7F80838091300E909143
:10636000310EDF91CF911F910F91FF90EF90DF9051
:10637000CF90BF90AF900895EF92FF920F931F932D
:10638000CF93DF93EC017A018B011092350E1092BE
:10639000340E10922F0E2091E02F30E040E0ABE061
:1063A000B0E086E190E0289FB001299F700D389FF2
:1063B000700D112416C0242F2F5F842F90E08A9F28
:1063C000F0018B9FF00D9A9FF00D1124E60FF71F3F
:1063D000E558F24F8285882319F440932F0E0FC0A1
:1063E000422F423040F340932F0E423041F40E943E
:1063F000486862E070E00E94C46B80932F0EE091C9
:106400002F0E8BE0E89FF00111248091E02F26E110
:10641000829FC0011124E80FF91FE558F24FF09355
:10642000350EE093340EC193D193CF01B801A7018B
:106430000E94594920912F0E30E04091E02F50E00A
:106440008BE090E0289FF001299FF00D389FF00D20
:10645000112486E190E09C01429FC001439F900D72
:10646000529F900D1124E80FF91FE558F24F81E07B
:1064700082878091340E9091350EDF91CF911F91DC
:106480000F91FF90EF900895EF92FF920F931F935B
:10649000CF93DF937C011092310E1092300E109248
:1064A0002F0E0091E02F202F30E084E490E0289F11
:1064B000E001299FD00D389FD00D11243EC0812FBF
:1064C00090E0FC01B5E0EE0FFF1FBA95E1F7880FF1
:1064D000991FE80FF91FEC0FFD1FE853F24F808161
:1064E00081FF28C0212F30E0C90175E0880F991F76
:1064F0007A95E1F7220F331F820F931F8C0F9D1F98
:106500008955924FB70140E150E00E9459690097C8
:1065100089F482E2189FC001112424E4029F9001B3
:106520001124820F931F8955924F9093310E8093BF
:10653000300E08C01F5F10932F0E10912F0E1230D7
:1065400008F4BDCF8091300E9091310EDF91CF9144
:106550001F910F91FF90EF900895EF92FF921F937C
:10656000CF93DF937C0110922F0E8091E02F90E06B
:1065700024E430E0829FE001839FD00D929FD00DF4
:10658000112442C0812F90E0FC01B5E0EE0FFF1F07
:10659000BA95E1F7880F991FE80FF91FEC0FFD1F5F
:1065A000E853F24F808181FF2CC0212F30E0C901D8
:1065B00075E0880F991F7A95E1F7220F331F820F3C
:1065C000931F8C0F9D1F212F30E0F90155E0EE0F36
:1065D000FF1F5A95E1F7220F331FE20FF31FEC0F55
:1065E000FD1FE955F24F40894695469546958955D8
:1065F000924FB70150E00E945969009711F481E071
:1066000009C01F5F10932F0E10912F0E123008F447
:10661000B9CF80E0DF91CF911F91FF90EF90089567
:10662000AF92BF92CF92DF92EF92FF920F931F93A0
:10663000CF93DF936C011092330E1092320E1092B2
:106640002F0E0091E02F202F30E01CE2A12EB12C64
:1066500084E890E0289F7001299FF00C389FF00C8F
:106660001124E901C952D64F2FC0812F90E08A9D95
:1066700090018B9D300D9A9D300D11242E0D3F1DE4
:10668000F901ED58F34F83A58823D9F04881C9015A
:106690008D57934FB60150E00E945969009789F4D5
:1066A0008CE2189FC001112424E8029F900111245C
:1066B000820F931F8D58934F9093330E8093320E19
:1066C00007C01F5F10932F0E10912F0E133068F22A
:1066D0008091320E9091330EDF91CF911F910F91E7
:1066E000FF90EF90DF90CF90BF90AF900895CF9242
:1066F000DF92EF92FF920F931F93CF93DF937C0172
:106700001092330E1092320E10922F0E0091E02F45
:10671000202F30E08CE2C82ED12C84E890E0289F16
:10672000E001299FD00D389FD00D11242CC0812F5E
:1067300090E08C9DF0018D9DF00D9C9DF00D11243D
:10674000EC0FFD1FED58F34F83A58823C9F0CF014F
:10675000B70140E150E00E945969009789F48CE24A
:10676000189FC001112424E8029F90011124820F78
:10677000931F8D58934F9093330E8093320E07C022
:106780001F5F10932F0E10912F0E133080F2809107
:10679000320E9091330EDF91CF911F910F91FF90A8
:1067A000EF90DF90CF900895EF92FF920F931F9399
:1067B000CF93DF93182F092FEB01F42EE22E1092C6
:1067C000330E1092320E10922F0E2091E02F30E0F7
:1067D00040E0ACE2B0E084E890E0289FB001299F5F
:1067E000700D389F700D112416C0242F2F5F842F39
:1067F00090E08A9FF0018B9FF00D9A9FF00D11247D
:10680000E60FF71FED58F34F83A5882319F4409343
:106810002F0E0FC0422F433040F340932F0E4330D2
:1068200041F40E94486863E070E00E94C46B80936A
:106830002F0E4091E02F90912F0E8CE2989FB00187
:10684000112484E8489FC0011124680F791F6D58F6
:10685000734F7093330E6093320EDB01212F302F74
:10686000C901FC0180E101900D928150E1F7E42F14
:10687000F0E02097B9F010922F0EE952F64F4081C8
:1068800090E00BC0E92FF0E0DB01AE0FBF1FEC0F73
:10689000FD1F808150968C939F5F941798F390937F
:1068A0002F0E0CC0E952F64F40819B01205F3F4FF5
:1068B000C90160E070E050E00E948169E091320E11
:1068C000F091330EF08EE18ECF014A9640E050E019
:1068D00060E070E00E9459498091320E9091330E31
:1068E000829640E050E060E070E00E945949E091FB
:1068F000320EF091330E12A681E083A7CF01DF9113
:10690000CF911F910F91FF90EF9008953091E02F5C
:10691000432F50E020E0ACE2B0E084E890E0489FF4
:10692000B001499F700D589F700D11240FC0822F28
:1069300090E08A9FF0018B9FF00D9A9FF00D11243B
:10694000E60FF71FED58F34F13A62F5F233078F3B0
:1069500020E0ABE0B0E086E190E0489FB001499FC5
:10696000700D589F700D11240FC0822F90E08A9FE8
:10697000F0018B9FF00D9A9FF00D1124E60FF71F89
:10698000E558F24F12862F5F223078F320E084E43E
:1069900090E0489FB001499F700D589F700D1124E1
:1069A00014C0822F90E0FC01B5E0EE0FFF1FBA95F6
:1069B000E1F7880F991FE80FF91FE60FF71FE8535B
:1069C000F24F80818D7F80832F5F223050F32093A0
:1069D0002F0E89E790E0489FF001499FF00D589FE6
:1069E000F00D1124E55BF14D8589882361F184E484
:1069F00090E0489FD001499FB00D589FB00D1124E1
:106A0000FD01E955F24F8EEF90E891838083138268
:106A100012821582148217821682118610861386BE
:106A20001286158614861786168680E4808BA853F6
:106A3000B24F8C9183608C93832F44E650E060E0EA
:106A400070E00E94F24A0895AF92BF92CF92DF9217
:106A5000EF92FF920F931F93CF93DF9380910329BF
:106A60008F3F09F07AC3809104298E3F09F075C3E6
:106A700080910529803809F070C38091570CA82FA8
:106A8000B0E0FD01EC5DF64D8181882309F065C31E
:106A9000A85DB64D4C91442379F08091E02F90E0B1
:106AA00029E730E0829FF001839FF00D929FF00D67
:106AB0001124E55BF14D4483E091570CF0E0E85D73
:106AC000F64D2481358146815781211531054105D7
:106AD000510509F448C08091E02F90E0C9E7D0E06B
:106AE0008C9FF0018D9FF00D9C9FF00D1124E55BB4
:106AF000F14DE580F68007811085CA01B9010E9439
:106B00007122E616F7060807190769F10091E02FD0
:106B100010E0E091570CF0E0E85DF64D648175817E
:106B2000868197810E9471220C9FF0010D9FF00DCC
:106B30001C9FF00D1124E55BF14D658376838783FF
:106B400090870091E02F10E00E9454420C9FF001CA
:106B50000D9FF00D1C9FF00D1124E55BF14D618739
:106B6000728783879487E091570CF0E0E85DF64DDB
:106B70006085718582859385611571058105910513
:106B8000A1F00091E02F10E00E94712229E730E08F
:106B9000029FF001039FF00D129FF00D1124E55BA1
:106BA000F14D658776878787908B1092380E10920B
:106BB000370E10923A0E1092390E40E009C0E42FC1
:106BC000F0E0EE0FFF1FE55CF14F118210824F5F86
:106BD0004230A8F34093470E8CE08093360E6091CC
:106BE0007F287091802839C0F901E450F74D8181E8
:106BF000882309F4B0C28081833071F0853039F088
:106C00008130D9F4F093380EE093370E16C0F0932C
:106C10003A0EE093390E11C080913B0E90913C0EDC
:106C2000892B19F4E0E040E0A9C280913D0E9091DB
:106C30003E0E892B09F4A0C242E08091360EE0910D
:106C4000570CF0E0E450F74DE80FF11D95A5990FB2
:106C5000990F990F980F9093360E9091570C809141
:106C6000360E282F30E0290F311D245D3F4F2617A7
:106C7000370708F4B9CF4093470EE091390EF091F1
:106C80003A0E3097C1F00091E02F10E064817581D9
:106C9000868197810E94712229E730E0029FF001EE
:106CA000039FF00D129FF00D1124E55BF14D608301
:106CB0007183828393831092470E7FC164817581B3
:106CC000868197810E9471227B018C01E091470EA1
:106CD000F0E0EE0FFF1FE55CF14F0190F081E02D39
:106CE00060857185828593850E947122E616F7067C
:106CF0000807190708F45CC1E091470EF0E0EE0FB9
:106D0000FF1FE55CF14F0190F081E02D80898E3FFF
:106D100021F48189803809F44BC1838187FF7CC0CD
:106D2000CF0140960E944432EC019093420E809332
:106D3000410EE091470E0097C1F5F0E0EE0FFF1F06
:106D4000E55CF14F0190F081E02D648175818681D1
:106D50009781611571058105910509F45DC0EF0109
:106D600060966F3F2FEF72072FEF82072FEF92078A
:106D700071F012810E94712228EE33E040E050E071
:106D80000E94A56B9B01AC01CE01612F06C0CE0114
:106D9000628120E030E040E050E000E00E94E83016
:106DA0009093420E8093410E37C0F0E0EE0FFF1F2C
:106DB000E55CF14F0190F081E02D64817581868161
:106DC0009781611571058105910549F06F3F2FEF9E
:106DD00072072FEF82072FEF920749F404C0CE010C
:106DE0000E94562F19C089A1816089A315C00E94F5
:106DF000712228EE33E040E050E00E94A56BAB0129
:106E0000BC01CE0141960E945949E091410EF0919A
:106E1000420E81A18E7F81A3E091470EF0E0EE0F3C
:106E2000FF1FE55CF14F0190F081E02D838186FF2B
:106E3000BFC084819581A681B7810097A105B10566
:106E400009F4B6C0CF014096628141E00E94C94377
:106E5000DC019093460E8093450EE091470E00971B
:106E600009F479C0F0E0EE0FFF1FE55CF14F0190EF
:106E7000F081E02D64817581868197816F3F2FEFCE
:106E800072072FEF82072FEF920709F460C00E946C
:106E9000712261527C418040904040F5E091470E64
:106EA000F0E0EE0FFF1FE55CF14F0190F081E02D67
:106EB00064817581868197810E9471227B018C019A
:106EC0008091450E9091460E41960E9429495B01A2
:106ED0006C01C801B70128EE33E040E050E00E94A9
:106EE000A56BA616B706C806D90600F50091450E93
:106EF0001091460E0F5E1F4FE091470EF0E0EE0F2F
:106F0000FF1FE55CF14F0190F081E02D64817581F8
:106F1000868197810E94712228EE33E040E050E0A4
:106F20000E94A56BAB01BC01C80109C08091450E50
:106F30009091460E419640E05DED6DE670E00E9456
:106F40005949E091450EF091460E118E31C081E015
:106F500059968C932DC0F0E0EE0FFF1FE55CF14FCA
:106F60000190F081E02D6481758186819781EF0128
:106F700060966F3F2FEF72072FEF82072FEF920778
:106F800071F012810E94712228EE33E040E050E05F
:106F90000E94A56B9B01AC01CE01612F06C0CE0102
:106FA000628120E030E040E050E001E00E949B453B
:106FB0008091470E8F5F8093470EE091470EE2303D
:106FC00058F4F0E0EE0FFF1FE55CF14F0190F08107
:106FD000E02D309709F072CE84E099E20E94773379
:106FE000FC019093400E80933F0E6091370E70919C
:106FF000380E6115710509F43FC0009769F46E5FA2
:107000007F4F84E099E241E022E00E94D4339093E4
:10701000400E80933F0E30C0818D882311F482E0B2
:10702000818FC091370ED091380E229600913F0E7D
:107030001091400E005F1F4FE091E02FF0E0E95209
:10704000F64FE080CE01B8014E2D50E00E94596904
:10705000009761F0C801BE014E2D50E00E946669A4
:10706000E0913F0EF091400E82E0818FE0913F0E63
:10707000F091400E81E0808FE091570CF0E0E85DE8
:10708000F64D82819381E0913F0EF091400E892B65
:1070900009F451C0309769F484E099E260E070E04F
:1070A00041E025E00E94D4339093400E80933F0E40
:1070B00002C081E0808F80913F0E9091400E0E942F
:1070C000962E8C019093440E8093430EE091570CC2
:1070D0000097D1F400913F0E1091400EF0E0E85D72
:1070E000F64D828193810E94852128EE33E0829FB4
:1070F000A001839F500D929F500D112460E070E01D
:10710000C8010E94BC3124C0F0E0E85DF64D8281E8
:1071100093810E94852128EE33E0829FA001839F06
:10712000500D929F500D112460E070E0C80102964E
:107130000E9459490DC0309759F0CF010E94962EF8
:107140009093440E8093430E009711F00E944C2FB1
:107150000E94EB5902C04093470E10928028109273
:107160007F28DF91CF911F910F91FF90EF90DF90DB
:10717000CF90BF90AF900895E1E041E0F0E0EE0FD6
:10718000FF1FE55CF14F2450374D3183208355CDEF
:10719000EF92FF920F931F93DF93CF9300D0CDB761
:1071A000DEB7E091E02FF0E0E952F64F2081822F28
:1071B00090E00296022F0E5F87709070081B892B5B
:1071C00009F0085F8CEF98E220E62093FC281092EB
:1071D000FD281092FF281092FE282AE3209302290E
:1071E0002FEF20930329FC0178962FEF32E03093A4
:1071F0001529209314291382128215821482178272
:10720000168211861086138612861586148620E053
:1072100032E0378726870896BF010E94AA41209155
:10722000570CA22FB0E0FD01EC5DF64D85E88083A0
:107230001182FD01E85DF64D1082118212821382E7
:10724000109200298091042990910529892B99F5A4
:107250008091062990910729892B69F58091082949
:1072600090910929892B39F580910A2990910B2950
:10727000892B09F580910C2990910D29892BD9F43E
:1072800080910E2990910F29892BA9F480911029C2
:1072900090911129892B79F48091122990911329C9
:1072A000892B49F488E080930129D096B0938028F7
:1072B000A0937F284EC0E02EFF24822F90E0C0963E
:1072C0008E0D9F1D9093802880937F28085F0093E8
:1072D00001290850A45DB64DB093380EA093370E27
:1072E00081E08C9306950695069511960C9311975F
:1072F0002091E02F129630E0F901E952F64F4081DB
:1073000053E0220F331F5A95E1F72957374DCD012E
:10731000B90150E00E946669E091E02FF0E0E95287
:10732000F64F808190E09701281B390B22503040A6
:107330003A8329832091370E3091380E2E5F3F4FCC
:10734000280F391FC90160E070E049815A810E940D
:1073500081698091570C082F10E00C5D164DF801E3
:10736000138212820E94512280959095F801938396
:1073700082830F900F90CF91DF911F910F91FF901B
:10738000EF900895FF920F931F93CF93DF938C019B
:10739000EA01E091E02FF0E0E952F64F2081822FE0
:1073A00090E00296E2E0FE2EF20E87709070F81ADE
:1073B000892B11F088E0F80E1092570C80E680932C
:1073C000FC281092FD281092FF281092FE288AE3D4
:1073D000809302299FEF90930329E4E1F9E261157C
:1073E0007105B9F49093142982E08183138212828B
:1073F000158214821782168211861086128681E009
:10740000838794878D8585878E859F8597878687D7
:1074100007C0DF01FB0180E101900D928150E1F78F
:1074200087E8809324291092252910922829109208
:10743000292910922A2910922B29ACE2B9E2FE01E7
:1074400080E101900D928150E1F710920029CE0168
:1074500060E840E00E94C943892B09F05FC0011534
:10746000110549F0A4E0B9E2F80180E101900D9224
:107470008150E1F706C084E099E264E179E20E947C
:10748000AA4188E1F80EF092012988EEF80E0F2D3E
:1074900010E0005C1F4F1093802800937F28005459
:1074A0001040E091570CF0E0E45CF64DF093380E9C
:1074B000E093370E81E08083F694F694F694F1829F
:1074C0002091E02F329630E0D901A952B64F4C916D
:1074D00063E0220F331F6A95E1F72957374DCF013B
:1074E000B90150E00E946669E091E02FF0E0E952B6
:1074F000F64F808190E0081B190B0250104020913C
:10750000370E3091380E2E5F3F4F280F391FC901BB
:1075100060E070E0A8010E94816929C010920529ED
:107520001092042910920729109206291092092915
:107530001092082910920B2910920A2910920D29F5
:1075400010920C2910920F2910920E2910921129D5
:1075500010921029109213291092122988E1809319
:10756000012980E490E09093802880937F28809187
:10757000570CC82FD0E0CC5DD64D1B821A820E94DA
:107580005122809590959B838A83DF91CF911F91A3
:107590000F91FF900895CF92DF92EF92FF920F9399
:1075A0001F93CF93DF939091570CE92FF0E0DF0109
:1075B000A85DB64DEC90809103298F3F09F042C140
:1075C000EC5DF64D8181882309F03CC114968C91C5
:1075D00014978F3F09F436C110E4C12ECE20E6FE89
:1075E00005C0809114298F3F09F42CC184E1809358
:1075F000360E1092380E1092370EC0917F28D0911F
:10760000802840E050E064E1292F30E0245D3F4FC6
:107610000FC0FC01E450F74D9181992309F40CC18E
:107620008081823009F4AF01990F990F990F690F8A
:10763000C901860F911D8C179D0758F35093380E82
:107640004093370E6093360ECD01049660E840E01B
:107650000E94C943FC019093460E8093450E00970B
:1076600061F08089882309F0EDC08091570C90E08B
:10767000845D964D0E944044E5C08091570C90E097
:10768000845D964D0E947733EC019093400E809379
:107690003F0E009709F4D6C00091370E1091380EB6
:1076A0000115110511F4FF240FC0BC01605F7F4F6D
:1076B000E091E02FF0E0E952F64F4081C8010296D8
:1076C00050E00E945969F82EF0E8DF2EDE20898D07
:1076D000882309F041C00115110509F4B3C0BE01AA
:1076E000605F7F4FE091E02FF0E0E952F64F40817C
:1076F00098012E5F3F4FCB01B90150E00E946669AF
:10770000C0913F0ED091400ECC2019F181E0898FBD
:107710008091E02F90E029E730E0829FF001839F85
:10772000F00D929FF00D1124E55BF14D618572859E
:107730008385948528EE33E040E050E00E94A56BFD
:107740000E94D76BCE014A96BA01A9010E945949FD
:107750006DC082E0898F6AC0E5FC08C0FF2031F06F
:10776000813009F06FC082E0898F6CC0011511056E
:1077700089F0BE01605F7F4FE091E02FF0E0E952B9
:10778000F64F408198012E5F3F4FCB01B90150E089
:107790000E946669CC2041F100913F0E1091400E8D
:1077A00081E0F801818F8091E02F90E029E730E0BF
:1077B000829FF001839FF00D929FF00D1124E55BF5
:1077C000F14D618572858385948528EE33E040E034
:1077D00050E00E94A56B0E94D76BC8014A96BA017F
:1077E000A9010E9459490EC08091370E9091380E20
:1077F000892B41F0FF2031F0E0913F0EF091400ED7
:1078000082E0818FE0913F0EF091400E808D8823C1
:1078100069F0DD2059F4CF010E94962E9093440E1A
:107820008093430E009711F00E944C2FE0913F0E81
:10783000F091400ED08E06C05093380E4093370E14
:107840006093360E1092802810927F28DF91CF919E
:107850001F910F91FF90EF90DF90CF900895DF92EE
:10786000EF92FF920F931F93CF93DF9380910329A1
:107870008F3F09F02DC28091570C482F50E0FA013C
:10788000E85DF64D84818F3F09F422C2FA01EC5D78
:10789000F64D8181882309F01BC21092380E109298
:1078A000370E84E18093360EC0917F28D0918028D6
:1078B00020E030E064E1FA01BC9611C0DC01A45084
:1078C000B74D11969C911197992309F4FBC18C91A6
:1078D000813009F49D01990F990F990F690FCF011C
:1078E000860F911D8C179D0748F32093370E309318
:1078F000380E6093360E232B09F46FC08091042953
:1079000090910529892B59F5809106299091072995
:10791000892B29F58091082990910929892BF9F45F
:1079200080910A2990910B29892BC9F480910C2907
:1079300090910D29892B99F480910E2990910F290E
:10794000892B69F48091102990911129892B39F4A0
:107950008091122990911329892B09F4B9C184E0EF
:1079600099E20E9477338C019093400E80933F0EF2
:107970006091370E7091380E009749F46E5F7F4F1B
:1079800084E099E240E022E00E94D43326C092E0F5
:10799000E92EF12CE60EF71EE8016096E091E02F4B
:1079A000F0E0E952F64FD080C701BE014D2D50E006
:1079B0000E945969009759F0CE01B7014D2D50E052
:1079C0000E946669E0913F0EF091400E04C0F801FC
:1079D000818D882311F482E0818F8091570C90E093
:1079E000845D964D60E840E00E94C9439093460E46
:1079F0008093450E892B09F46BC1809104299091E5
:107A00000529892B09F073C08091062990910729D7
:107A1000892B09F06CC08091082990910929892B44
:107A200009F065C080910A2990910B29892B09F0F2
:107A30005EC080910C2990910D29892B09F057C0C7
:107A400080910E2990910F29892B09F050C08091C7
:107A5000102990911129892B09F049C08091122990
:107A600090911329892B09F042C084E199E20E9488
:107A70002E44882309F42CC1E091450EF091460E66
:107A80008089882361F18FEF92E09093152980938C
:107A90001429109217291092162910921929109260
:107AA000182910921B2910921A2910921D29109240
:107AB0001C2910921F2910921E2910922129109220
:107AC000202980E091E0909323298093222984E06B
:107AD00099E264E179E20E94AA4130E253C08091C8
:107AE000570C90E0845D964D0E944044F1C084E0C4
:107AF00099E260E840E00E94C943892B09F0E8C0A0
:107B000084E199E20E942E448823B9F0E4E1F9E28D
:107B1000DF01509780E10D9001928150E1F7809153
:107B2000570CE82FF0E0A4E0B9E2E45DF64D80E107
:107B300001900D928150E1F724C084E199E260E860
:107B400040E00E94C9432091450E3091460E28170F
:107B5000390709F0BDC0E4E1F9E2DF01509780E1A7
:107B60000D9001928150E1F78091570CE82FF0E0E1
:107B7000A4E0B9E2E45DF64D80E101900D92815000
:107B8000E1F730E61092570C8091E02FA82FB0E07B
:107B900089E790E0A89FF001A99FF00DB89FF00D34
:107BA0001124E55BF14D838981113068A952B64FEC
:107BB0002C91822F90E00296422F4E5F877090703A
:107BC000481B892B09F0485F80E68093FC281092BF
:107BD000FD281092FF281092FE2810920029485E7E
:107BE0004093012948518AE3809302298FEF8093C3
:107BF000032988E880932429109225293093282985
:107C0000ACE2B9E22091450E3091460EC901FC016B
:107C100080E101900D928150E1F7042F10E0005CAB
:107C20001F4F1093802800937F2800541040E0914C
:107C3000570CF0E0E45CF64DF093380EE093370E0D
:107C400082E0808346954695469541832091E02FBA
:107C5000329630E0D901A952B64F4C9183E0220F01
:107C6000331F8A95E1F72957374DCF01B90150E00D
:107C70000E946669E091E02FF0E0E952F64F8081C2
:107C800090E0081B190B025010402091370E3091E4
:107C9000380E2E5F3F4F280F391FC90160E070E09A
:107CA000A8010E9481698091570CC82FD0E0CC5D5B
:107CB000D64D1B821A820E945122809590959B83FB
:107CC0008A830AC03093380E2093370E6093360EA5
:107CD0001092802810927F28DF91CF911F910F91F1
:107CE000FF90EF90DF9008956F927F928F929F9216
:107CF000AF92BF92CF92DF92EF92FF920F931F93BA
:107D0000DF93CF9300D0CDB7DEB7AC01E091E02F89
:107D1000F0E0E952F64F2081822F90E0029612E0C7
:107D2000D12ED20E87709070D81A892B11F088E06E
:107D3000D80E6115710529F58FEF92E09093152902
:107D4000809314291092172910921629109219293C
:107D50001092182910921B2910921A2910921D298D
:107D600010921C2910921F2910921E29109221296D
:107D70001092202980E091E090932329809322297A
:107D800008C0A4E1B9E2FB0180E101900D928150AD
:107D9000E1F74115510549F0A4E0B9E2FA0180E1AB
:107DA00001900D928150E1F706C084E099E264E110
:107DB00079E20E94AA411092570C80E68093FC2839
:107DC0001092FD281092FF281092FE288AE38093DB
:107DD00002298FEF8093032986E880932429ECEF12
:107DE000F8E211A68091E02F90E009E710E0809F73
:107DF000F001819FF00D909FF00D1124E55BF14D96
:107E0000848180932829818992890E948521909379
:107E10002B2980932A298091570CE82EFF24A8E271
:107E2000B9E2EA0EFB1E8091E02F90E0809FF00106
:107E3000819FF00D909FF00D1124E55BF14D658160
:107E40007681878190850E947122F7016483758312
:107E5000868397838091570CE82EFF2488E299E26D
:107E6000E80EF91E8091E02F90E0809FF001819F45
:107E7000F00D909FF00D1124E55BF14D6585768541
:107E8000878590890E947122D70118966D937D9302
:107E90008D939C931B970D2D10E0085C1F4F109342
:107EA000802800937F2808531040E091570CF0E0A1
:107EB000EC5CF64DF093380EE093370E81E0808352
:107EC0008D2D86958695869581832091E02F32961B
:107ED00030E0D901A952B64F4C91B3E0220F331FC5
:107EE000BA95E1F72957374DCF01B90150E00E940B
:107EF0006669E091E02FF0E0E952F64F808190E072
:107F0000081B190B025010402091370E3091380E8B
:107F10002E5F3F4F280F391FC90160E070E0A801B4
:107F20000E948169BCE0DB0ED092360E0E945B2F6E
:107F30007C011092470EA2E26A2EF3E07F2EE0EC65
:107F40008E2E74E0972EAA24AA94BA2C6501ABC099
:107F5000869DF0011124EE0DFF1D81A181FF9EC0C1
:107F600082FF9CC080818E3F21F48181803809F49A
:107F700095C09091570C8091360E082F10E0090F94
:107F8000111D085D164DD8017C9213968C921397A3
:107F900011969C921197808912968C93129781A1C9
:107FA00080FF0CC0F801A482B582C682D7821896E1
:107FB000AD92BD92CD92DC921B9741C065897689C6
:107FC0008789908D28EE33E040E050E00E94D76B27
:107FD000CA01B9010E947122F80164837583868306
:107FE00097838091570C9091360E092F10E0080F5F
:107FF000111D085D164D8091470E90E0FC0165E073
:10800000EE0FFF1F6A95E1F7880F991FE80FF91F20
:10801000EE0DFF1D658D768D878D90A128EE33E0E6
:1080200040E050E00E94D76BCA01B9010E94712262
:10803000D80118966D937D938D939C931B972091F7
:10804000360E8091570CE22FF0E0E80FF11DE85D4D
:10805000F64D14861586168617868091470E90E099
:10806000DC0145E0AA0FBB1F4A95E1F7880F991F75
:10807000A80FB91F7096AE0DBF1D80E10D90019243
:108080008150E1F7205E2093360E80917F289091F9
:10809000802880969093802880937F288091470E37
:1080A0008F5F8093470E8091470E823008F450CF47
:1080B00080917F289091802888979A8389838A81EC
:1080C000809300298981809301298091570C082F82
:1080D00010E00C5D164DF801138212820E945122AD
:1080E00080959095D80113969C938E9312970F903C
:1080F0000F90CF91DF911F910F91FF90EF90DF9044
:10810000CF90BF90AF909F908F907F906F90089589
:10811000BF92CF92DF92EF92FF920F931F93DF9364
:10812000CF93CDB7DEB760970FB6F894DEBF0FBE22
:10813000CDBF8091E02F90E029E730E0829FF001F1
:10814000839FF00D929FF00D1124E55BF14D838923
:10815000882309F4CCC0809103298F3F09F0C7C060
:108160008091570C682F70E0FB01EC5DF64D81812A
:10817000882309F0BCC01092380E1092370E84E0AC
:108180008093360E00917F281091802820E030E007
:1081900044E0FB01BC9611C0DC01A450B74D119620
:1081A0009C911197992309F49CC08C91813009F41A
:1081B0009D01990F990F990F490FCF01840F911DC0
:1081C0008017910748F32093370E3093380E409371
:1081D000360E232B09F470C0809104299091052953
:1081E000892B59F58091062990910729892B29F52A
:1081F0008091082990910929892BF9F480910A2905
:1082000090910B29892BC9F480910C2990910D290B
:10821000892B99F480910E2990910F29892B69F46B
:108220008091102990911129892B39F4809112297C
:1082300090911329892B09F45AC084E099E20E9495
:1082400077337C019093400E80933F0E6091370E00
:108250007091380E009749F46E5F7F4F84E099E289
:1082600040E022E00E94D43327C002E0C02ED12C8F
:10827000C60ED71E8C01005F1F4FE091E02FF0E08B
:10828000E952F64FB080C601B8014B2D50E00E9474
:108290005969009759F0C801B6014B2D50E00E9472
:1082A0006669E0913F0EF091400E04C0F701818DA8
:1082B000882311F482E0818F1092802810927F2809
:1082C000DE011196E4E0F9E280E101900D92815027
:1082D000E1F780E090E0BE016F5F7F4F0E94C142F6
:1082E0000AC03093380E2093370E4093360E10920A
:1082F000802810927F2860960FB6F894DEBF0FBEDC
:10830000CDBFCF91DF911F910F91FF90EF90DF9044
:10831000CF90BF90089540E020E030E0FC01E20FF4
:10832000F31F5081FB01E20FF31FE0815E1731F470
:10833000485F2F5F3F4F403889F70AC0E527842FF9
:10834000885FE7FD05C04F5F481711F0EE0FF9CFCA
:10835000842F08959F92AF92BF92CF92DF92EF92B7
:10836000FF920F931F93CF93DF93E82E992EEB018B
:1083700088818E3F21F48981803819F437C08F3F7E
:10838000A9F1FF2400E011E09BE1A92EB12C89E7BF
:10839000C82ED12C26C08091E02F90E0212F30E014
:1083A0002A9DB0012B9D700D3A9D700D11249C01EA
:1083B0002C9DC0012D9D900D3C9D900D1124680FAA
:1083C000791FFB01E55BF14D80A5813049F46D59C2
:1083D000714DCE010E948B418F1510F0F82E012FA8
:1083E0001F5F1330C0F21093520E01C000E0402F07
:1083F00050E02091E02F30E08BE190E0489FF001C9
:10840000499FF00D589FF00D112489E790E0AC01D1
:10841000249FC001259F900D349F900D1124E80FDB
:10842000F91F2E2D392DC901DC01ED59F14D80E1E7
:1084300001900D928150E1F7DF91CF911F910F9143
:10844000FF90EF90DF90CF90BF90AF909F900895F6
:10845000E091E02FF0E0DF01AD5AB14F1C92EE0F3A
:10846000FF1FDF01A75AB14F6D917C91EB5AF14F7D
:10847000808191810E94743E08950E944868AA27D5
:1084800097FDA095BA2FBC01CD0120E532E246E070
:1084900050E00E94D76B9B01AC0120593A4F4C4FE2
:1084A0005F4FB901CA0108954F925F926F927F9218
:1084B0008F929F92BF92CF92DF92EF92FF920F9393
:1084C0001F938091E02F90E04BE4C42E4EE2D42E17
:1084D00039E7432E512C849DF001859DF00D949D2C
:1084E000F00D1124EC0DFD1D65817681878190854D
:1084F0000E94B46A20E030E040E05FE30E941A6B23
:108500000E94886A3B014C010E944868B82E0E9474
:108510004868FB2CEE24E80EF91E00E010E0809184
:10852000E02F90E09C01249DC001259D900D349D7D
:10853000900D1124C80ED91EF601658176818781C0
:1085400090850E94B46A0E94886A9B01AC01C801B0
:10855000B7010E94D76B9B01AC01260D371D481D4A
:10856000591DB901CA011F910F91FF90EF90DF9043
:10857000CF90BF909F908F907F906F905F904F9023
:1085800008951F93CF93DF939C011091E02FA12FAB
:10859000B0E0FD01ED5AF14F8081882309F04AC017
:1085A0002115310591F0CDE5DEE0F90180E1019082
:1085B00009928150E1F7FD01EE0FFF1FEB5AF14FD9
:1085C0008DE59EE09183808307C0FD01EE0FFF1FC4
:1085D000EB5AF14F118210826115710591F0CDE6D1
:1085E000DEE0FB0180E1019009928150E1F7FD019D
:1085F000EE0FFF1FE75AF14F8DE69EE091838083D7
:1086000007C0FD01EE0FFF1FE75AF14F11821082E4
:10861000AD5AB14F81E08C930E94486864EF71E0DD
:108620000E94C46BAC01662757FD6095762F812FA1
:108630000E949C49DF91CF911F910895EF92FF9284
:108640000F931F930E943D427B018C01E091E02F2C
:10865000F0E0E05BF14F8081833078F481E8E81648
:108660008EE3F80680E0080780E0180730F020E885
:10867000E22E2EE3F22E012D112D80E090E060E03D
:1086800070E00E94743E8091E02FE82FF0E0E05B04
:10869000F14F90819F5F9083B801A7010E94DF494D
:1086A0001F910F91FF90EF9008958091E02FA82FD8
:1086B000B0E089E790E0A89FF001A99FF00DB89F76
:1086C000F00D1124E55BF14D84898823E1F0A05B76
:1086D000B14F8C918823B9F40E943D42AC01CB018B
:1086E000DA01AC01BD0141388EE3580780E068072C
:1086F00080E0780720F040E85EE360E070E0809181
:10870000E02F0E94DF4908951F931091E02FE12F81
:10871000F0E0E25BF14F8081882371F40E944868A9
:1087200060ED77E00E94C46BAC01662757FD609551
:10873000762F812F0E942B4A1F9108950E94E42ECC
:10874000892BD1F4E091E02FF0E0E25BF14F8081E2
:10875000843090F40E94C8388091E02FE82FF0E038
:10876000E25BF14F90819F5F908348E853E160E0C6
:1087700070E00E942B4A08958091E02F0E94794971
:10878000E091E02FF0E0E25BF14F10820E945D5932
:108790000895BF92CF92DF92EF92FF920F931F93B3
:1087A000CF93DF937C01062FB42E1092520E2091AE
:1087B000E02F30E00695069506954BE1C42ED12CAE
:1087C00089E790E0289FE001299FD00D389FD00DC8
:1087D000112433C0212F30E02C9DF0012D9DF00D90
:1087E0003C9DF00D1124EC0FFD1FE55BF14D80A5C4
:1087F0008F3F01F182A98B1511F0BB20D9F42C9D7C
:10880000C0012D9D900D3C9D900D11248C0F9D1F3E
:108810008D59914DB701402F50E00E945969009742
:1088200049F48BE1189F900111242C0F3D1F2D5905
:10883000314D09C01F5F1093520E1091520E13302C
:1088400048F220E030E0C901DF91CF911F910F91F4
:10885000FF90EF90DF90CF90BF9008956091E02F50
:1088600029E7629FB00111246C54714D40E150E042
:108870000E9459699C0180E0232B09F481E008954E
:108880001F93CF93DF93BC011091E02FE12FF0E015
:10889000EE0FFF1FE85BF14F8081918140E150E0D6
:1088A0000E9459690097A9F4812F0E948349A091E1
:1088B000E02FB0E0FD01EE0FFF1FE85BF14F80817C
:1088C00091812FEFEC01288B11821082A45BB14FB4
:1088D0001C928FEF9FEF0E94F4561F93DC0150967D
:1088E0008C9150978823E1F41091E02FE12FF0E074
:1088F000EE0FFF1FE85BF14F80819181892B81F49E
:10890000B183A0830E94486860ED77E00E94C46B49
:10891000AC01662757FD6095762F812F0E94B74ADC
:108920001F9108951F93CF93DF932091E02FA22FE3
:10893000B0E0FD01EE0FFF1FE85BF14F4081518178
:108940004115510509F489C0C9E7D0E0AC9FF00199
:10895000AD9FF00DBC9FF00D1124E55BF14DA45BC4
:10896000B14F9C918789981788F580E090E060E08E
:1089700070E00E94C2391091E02F212F30E0F90100
:10898000E45BF14F80818F5F80832C9FF0012D9FEE
:10899000F00D3C9FF00D1124E55BF14D658576856A
:1089A0008785908928EE33E040E050E00E94D76B45
:1089B000CA01B90128EE33E040E050E00E94A56B07
:1089C000AB01BC01812F0E94B74A47C0822F0E9491
:1089D00083492091E02F30E0F901EE0FFF1FE85BA3
:1089E000F14FA081B18181E050968C931182108269
:1089F000F901E45BF14F10821092520E40E0ABE1BE
:108A0000B0E02C9FB0012D9F700D3C9F700D112484
:108A100020C0242F2F5F842F90E08A9FF0018B9F2E
:108A2000F00D9A9FF00D1124E60FF71FE55BF14D55
:108A300080A5882369F44093520E8BE1489FC001C2
:108A40001124860F971F8D59914D0E946D4405C0CA
:108A5000422F4330F0F24093520EDF91CF911F919D
:108A60000895CF93DF93DC01EB01E091E02FF0E07C
:108A7000E952F64FE081E83061F49C01285F3F4FF6
:108A8000FB0188E00190E90109929E018150D1F734
:108A900023C0E63039F59C01285F3F4FAB0183E0EE
:108AA000FA010190AF01F90101929F018150C1F7D4
:108AB0008FEF1B968C931B978EEF1C968C931C97B5
:108AC0009D01235F3F4FFE01339683E00190E90152
:108AD00009929E018150D1F718968C91189792E0D7
:108AE000892720C0E23019F589811F968C931F9742
:108AF00088811E968C931E971D961C921D978EEF53
:108B00001C968C931C978FEF1B968C931B971A9631
:108B10001C921A978091BE2F19968C931997809169
:108B2000BD2F8D7F18968C93DF91CF9108958FEF95
:108B30009FEF0E94F4569F92AF92BF92CF92DF9226
:108B4000EF92FF920F931F93CF93DF93A82E992E4E
:108B500069017A01B02E21E0021719F4603409F09E
:108B6000BDC01092520E5091E02FC52FD0E040E0D2
:108B70000BE110E089E790E0C89FD001C99FB00DDC
:108B8000D89FB00D1124A5C0642F70E0942F9F5F73
:108B9000609F9001619F300D709F300D11242A0F4E
:108BA0003B1FF901E55BF14D80A58F3F09F090C0B7
:108BB0004093520EF901ED59F14D8A2D992D9C01EA
:108BC000D90180E10D9001928150E1F731E0B316B7
:108BD00019F58BE190E09C01629FC001639F900DAD
:108BE000729F900D112429E730E0B901C69F9001D2
:108BF000C79F300DD69F300D1124820F931F652F14
:108C000070E043E0660F771F4A95E1F76957774DAB
:108C10008D59914D0E9431458091E02F90E0209137
:108C2000520E30E00BE110E0209FA001219F500D7B
:108C3000309F500D1124C9E7D0E09C012C9FC0014A
:108C40002D9F900D3C9F900D1124480F591FFA0144
:108C5000E55BF14D10A6B2AAC114D104E104F10400
:108C600011F1CA018C58914DB701A6010E945949D2
:108C70002091520E30E08091E02F90E0209FF00193
:108C8000219FF00D309FF00D1124BC016C9FC0019D
:108C90006D9F900D7C9F900D1124E80FF91FE55BEF
:108CA000F14D11AA02C081E081AB8091520E2BE1FF
:108CB000829FC00111242091E02F49E7249F900159
:108CC0001124820F931F8D59914D0E946D4406C04F
:108CD000492F433008F458CF4093520EDF91CF9183
:108CE0001F910F91FF90EF90DF90CF90BF90AF90CA
:108CF0009F900895FF920F931F93CF93DF9381E08E
:108D00008093520E0BE110E0C9E7D0E0FF24FA9403
:108D100044C08091E02F90E030E0209FA001219F8F
:108D2000500D309F500D11249C012C9FC0012D9F90
:108D3000900D3C9F900D1124480F591FFA01E55BDF
:108D4000F14D80A58F3F21F181A9813009F1CA0140
:108D50008C58914D0E943F49892BD1F02091520EA1
:108D600030E08091E02F90E0209FF001219FF00DF6
:108D7000309FF00D11249C012C9FC0012D9F900D60
:108D80003C9F900D1124E80FF91FE55BF14DF0A613
:108D90008091520E8F5F8093520E2091520E23309D
:108DA00008F4B7CFDF91CF911F910F91FF900895F5
:108DB0008F929F92AF92BF92CF92DF92EF92FF92EB
:108DC0000F931F93DF93CF93CDB7DEB7E2970FB624
:108DD000F894DEBF0FBECDBF1092520EFBE1CF2E36
:108DE000D12CE9E7EE2EF12C8E010F5F1F4F77EBB0
:108DF000A72E78E0B72E6BE1862E59E7952E8DC011
:108E000030E08091E02F90E02C9DF0012D9DF00D41
:108E10003C9DF00D11249C012E9DC0012F9D900DB5
:108E20003E9D900D1124E80FF91FE55BF14D80A5E3
:108E30008F3F09F46DC0E0910201F09103018BE9CD
:108E400098E009952091520E30E08DB79EB70897B3
:108E50000FB6F8949EBF0FBE8DBFADB7BEB71196CB
:108E6000EDB7FEB7128301831396BC92AE921297B0
:108E700015963C932E9314978091E02F90E02C9DB3
:108E8000F0012D9DF00D3C9DF00D11249C012E9DB7
:108E9000C0012F9D900D3E9D900D1124E80FF91FEC
:108EA000E55BF14D80A5992787FD909517969C93DA
:108EB0008E9316970E94066A8DB79EB708960FB6D6
:108EC000F8949EBF0FBE8DBFE0910201F0910301A7
:108ED000C80109956091520E689DB00111248091DE
:108EE000E02F899DC0011124680F791F6D59714DC4
:108EF000C8010E94EF5BE0910201F0910301C801FB
:108F00000995E0910201F091030187EC98E0099541
:108F10008091520E8F5F8093520E2091520E23301B
:108F200008F46ECFE2960FB6F894DEBF0FBECDBF49
:108F3000CF91DF911F910F91FF90EF90DF90CF9035
:108F4000BF90AF909F908F9008957F928F929F9245
:108F5000AF92BF92CF92DF92EF92FF920F931F9347
:108F60004B015C01142F722E8091E02F90E029E7D5
:108F7000C22ED12C8C9D70018D9DF00C9C9DF00C0F
:108F800011242BE43EE2E20EF31E80E095E0A0E027
:108F9000B0E0F70180839183A283B38380E484836C
:108FA00080E395E7A0E0B0E085839683A783B08750
:108FB0000E945442F7016187728783879487F090FB
:108FC000E02F6F2D70E06C9D90016D9D300D7C9DAC
:108FD000300D1124F901E55BF14D88EE93E0A0E03E
:108FE000B0E085879687A787B08B81E0878B928AD0
:108FF000818A138A148B758A068B40E0ABE1B0E05E
:109000005FEF0FC0842F90E08A9FF0018B9FF00DDF
:109010009A9FF00D1124E20FF31FE55BF14D50A76D
:109020004F5F433078F34093520E09E710E0609FA2
:109030009001619F300D709F300D1124D901A55B07
:10904000B14DA759BF4F9FEF9D9382E08D931D9225
:109050001D921D921D921D921D921D921D921D9298
:10906000EE24E394ED929D93FB01E952F64F80814B
:10907000FB0193E0EE0FFF1F9A95E1F7E957F74DDB
:10908000E80FF11D339781918D9381918D938081AC
:109090008C93A857B040772009F45AC08EEF90E81F
:1090A00059969C938E9358975B961C921E925A9752
:1090B0005D961C921E925C975F961C921E925E9724
:1090C00091961C921E92909793961C921E92929744
:1090D00095961C921E92949797961C921E92969724
:1090E0006F2D70E0A3E0660F771FAA95E1F769572F
:1090F000774DC9018D59914D0E9431458091E02FE6
:1091000090E09C01209FC001219F900D309F900D09
:109110001124FC01E55BF14D10A623E022ABE1AA8E
:109120008D59914D0E946D440E9484438114910495
:10913000A104B10469F08091E02F90E0809FF001DC
:10914000819FF00D909FF00D1124E55BF14DE38AB6
:109150008091E02F48EE53E060E070E00E94664AA4
:109160001F910F91FF90EF90DF90CF90BF90AF9045
:109170009F908F907F900895FFCF08950895DF937B
:10918000CF93CDB7DEB728970FB6F894DEBF0FBEEA
:10919000CDBFDC018091E02F882309F046C01097F5
:1091A00089F483E389838A83809120298B8380914A
:1091B00021298C83809122298D83809123298E837C
:1091C000DE011196E0917F28F0918028E550F74D5F
:1091D00003C080818687319788E2EB3FF807C9F7A3
:1091E0008C91818311968C911197828312968C9128
:1091F0001297838313968C911397848314968C9182
:109200001497858315968C918683A7E8B8E23796E4
:109210008D91819388E2AD38B807D1F786E88093C5
:1092200008298DED8093092905C0813039F4CD01DD
:109230000E949D551092802810927F2880E090E037
:1092400028960FB6F894DEBF0FBECDBFCF91DF9149
:109250000895EF92FF920F931F93FC01E080F1803D
:10926000028113810E94C50AE61AF70A080B190B3E
:10927000B701C8011F910F91FF90EF900895EF92F1
:10928000FF920F931F93FC01E080F1800281138114
:109290000E94C50A20E030E0E616F7060807190725
:1092A00010F421E030E0C9011F910F91FF90EF9081
:1092B0000895CF92DF92EF92FF920F931F936C016C
:1092C0007A018B01FC0144835583668377830E9476
:1092D000C50A6E0D7F1D801F911FF601608371838B
:1092E000828393831F910F91FF90EF90DF90CF9037
:1092F0000895E82FF0E0E754F04D8081882311F0C5
:109300000E94150B0895E82FF0E0E954F04D80819C
:10931000882311F00E94150B0895CF93DF93C9EABB
:10932000DFE288810E94150B19928FE2C53BD807B6
:10933000C1F7DF91CF910895CF92DF92EF92FF9224
:109340000F931F93C82ECB01BA0128EE33E040E003
:1093500050E00E94D76BC901DA017C018D0181E0E8
:10936000E81680E0F80681E0080780E0180728F09A
:10937000E12CF12C81E0082F112D81E0C81621F499
:10938000C7016BE97BE403C0C70164E97BE40E9489
:10939000C40BD82E882339F4E114F104010511051A
:1093A00011F00E94BC48EC2DF0E0E755F04DD2865C
:1093B0001F910F91FF90EF90DF90CF900895CF9283
:1093C000DF92EF92FF920F931F93C82E7A018B01C9
:1093D000413080E0580781E0680780E0780768F452
:1093E00081E0C81621F4CA016AEA7BE403C0CA011D
:1093F00063EA7BE40E940D0C18C0CB01BA0128EE91
:1094000033E040E050E00E94D76BC901DA017C01F3
:109410008D0181E0C81621F4C7016AEA7BE403C02C
:10942000C70163EA7BE40E94C40BD82E882339F479
:10943000E114F1040105110511F00E94BC48EC2D66
:10944000F0E0E755F04DD0861F910F91FF90EF901F
:10945000DF90CF900895CF92DF92EF92FF920F931B
:109460001F93C82ECA01DB017C018D0181E0E81643
:1094700080E0F80681E0080780E0180728F0E12C7A
:10948000F12C91E0092F112D81E0C81621F4C701BC
:1094900069EB7BE403C0C70162EB7BE40E940D0C27
:1094A000D82E882339F4E114F1040105110511F0D7
:1094B0000E94BC48EC2DF0E0E754F04DD0821F91A3
:1094C0000F91FF90EF90DF90CF900895CF92DF92B1
:1094D000EF92FF920F931F93C82E7A018B014130B8
:1094E00080E0580781E0680780E0780788F441153C
:1094F00051056105710589F4EC2DF0E0EE0FFF1FB9
:10950000E358F14F808191817C0100E010E00DC0B3
:10951000E12CF12C31E0032F112DEC2DF0E0EE0FBA
:10952000FF1FE358F14FF182E08281E0C81621F479
:10953000C7016FEC7BE403C0C70161EC7BE40E94D0
:109540000D0CD82E882339F4E114F104010511051E
:1095500011F00E94BC48EC2DF0E0E755F04DD682AA
:109560001F910F91FF90EF90DF90CF900895CF92D1
:10957000DF92EF92FF920F931F93C82ECA01DB0177
:109580007C018D0181E0E81680E0F80681E00807A3
:1095900080E0180728F0E12CF12C51E0052F112D67
:1095A00081E0C81621F4C70164EE7BE403C0C70163
:1095B0006DED7BE40E940D0CD82E882339F4E11464
:1095C000F1040105110511F00E94BC48EC2DF0E0FA
:1095D000E954F04DD0821F910F91FF90EF90DF90F2
:1095E000CF900895CF92DF92EF92FF920F931F9347
:1095F000C82E7A018B01413080E0580781E068076E
:1096000080E0780788F4411551056105710589F4FA
:10961000EC2DF0E0EE0FFF1FEF57F14F80819181AD
:109620007C0100E010E00DC0E12CF12C71E0072F6F
:10963000112DEC2DF0E0EE0FFF1FEF57F14FF182EF
:10964000E08281E0C81621F4C7016AEF7BE403C021
:10965000C7016CEE7BE40E940D0CD82E882339F4F0
:10966000E114F1040105110511F00E94BC48EC2D34
:10967000F0E0E755F04DD2821F910F91FF90EF90EF
:10968000DF90CF900895CF92DF92EF92FF920F93E9
:109690001F93C82E7A018B01413080E0580781E08A
:1096A000680780E0780788F4411551056105710568
:1096B00089F4EC2DF0E0EE0FFF1FEB57F14F8081A6
:1096C00091817C0100E010E00DC0E12CF12C11E053
:1096D000012F112DEC2DF0E0EE0FFF1FEB57F14F96
:1096E000F182E08281E0C81621F4C70166E17CE4E2
:1096F00003C0C70168E07CE40E940D0CD82E8823CB
:1097000039F4E114F1040105110511F00E94BC487F
:10971000EC2DF0E0E755F04DD0821F910F91FF90B6
:10972000EF90DF90CF9008951092E02F0E94284292
:109730000E94F556089581E08093E02F0E94284210
:109740000E94F55608951092E02F0E941E430E9439
:10975000F556089581E08093E02F0E941E430E94F9
:10976000F55608951092E02F0E949E430E94F556F0
:10977000089581E08093E02F0E949E430E94F55659
:1097800008951092E02F80E040E050E060E070E04B
:109790000E94664A0E947A460E94F556089581E02A
:1097A0008093E02F40E050E060E070E00E94664A65
:1097B0000E947A460E94F55608951092E02F0E946A
:1097C00092440E94F556089581E08093E02F0E9414
:1097D00092440E94F55608951092E02F80E040E0F8
:1097E00050E060E070E00E94F24A0E94652F0E9403
:1097F000F556089581E08093E02F40E050E060E06E
:1098000070E00E94F24A0E94652F0E94F55608956A
:109810001092E02F80E040E050E060E070E00E94B5
:10982000434B0E940F5A0E94F556089581E08093A1
:10983000E02F40E050E060E070E00E94434B0E9467
:109840000F5A0E94F55608950F93DF93CF9300D0DF
:1098500000D0CDB7DEB79A8389837C836B8381E0A8
:109860008093E02F8C8180938F288B818093902828
:109870008A818093BD2F89818093BE2F60E070E044
:1098800080E090E040E021E000E00E94D62C81E002
:1098900044EF51E060E070E00E94434B0F900F9066
:1098A0000F900F90CF91DF910F9108950F93DF9359
:1098B000CF93CDB7DEB760970FB6F894DEBF0FBE7B
:1098C000CDBFAC011092E02F009779F020E030E09E
:1098D000F901E957F74DDA01A20FB31F8C9180838C
:1098E0002F5F3F4F2630310599F7FE01319680E119
:1098F000DF011D928A95E9F780E2898381E08A83FE
:1099000084E08B8380E78C8381EF8D838CE38E836F
:10991000CF010E94D45668E077E080E090E041E01B
:1099200021E000E00E94D62C80E044EF51E060E0AE
:1099300070E00E94434B60960FB6F894DEBF0FBEF6
:10994000CDBFCF91DF910F91089589E89EE090936C
:10995000422F8093412F0E948D490E941E4D0895F1
:10996000382F1092351420E02CC0822F90E0FC019B
:1099700073E0EE0FFF1F7A95E1F7880F991FE80F4C
:10998000F91FE35EFB4E80818130D1F4822F90E09D
:10999000FC0153E0EE0FFF1F5A95E1F7880F991F66
:1099A000E80FF91FE35EFB4E8181831749F4209392
:1099B00035148AE0289F90011124235E3B4E07C096
:1099C0002F5F223090F22093351420E030E0C9015F
:1099D0000895AC0181E08093351421E02AC0322F34
:1099E0003F5F822F90E0FC01B3E0EE0FFF1FBA95BE
:1099F000E1F7880F991FE80FF91FE35EFB4E8081A6
:109A00008823B1F481E0809327142093281490E0F8
:109A10000AC0E92FF0E0DA01AE0FBF1F8C91E35EC0
:109A2000FB4E84879F5F9830A0F390933514089580
:109A3000232F2230A0F220933514089581E08093E3
:109A40001D1410921E148EEF80931F1480E88093D3
:109A5000201421E010C0822F90E0FC0143E0EE0FC3
:109A6000FF1F4A95E1F7880F991FE80FF91FE35E82
:109A7000FB4E10822F5F223070F32093351408952F
:109A8000EF92FF920F931F93CF93DF937C01E091AE
:109A9000080FF091090F80910A0F90E00396DF0103
:109AA000A80FB91F0397B0933414A0933314E80F91
:109AB000F91F818186FD29C087FD12C0FD018191BA
:109AC0009191A191B19180930D0F90930E0FA0935E
:109AD0000F0FB093100FF0933414E093331431C090
:109AE00080E680930D0F8C918F7080930E0F1196EE
:109AF0008D919C9112979093100F80930F0F139656
:109B0000B0933414A09333141CC087FD11C08C9102
:109B100082958F70806680930D0FFD0181918295F3
:109B2000807F80930E0FF0933414E093331405C0BC
:109B300080E680930D0F10920E0F1092100F10926E
:109B40000F0F80910A0FC091080FD091090FC80F15
:109B5000D11D898185FD0BC0E0913314F09134143F
:109B600081918093130FF0933414E093331489811F
:109B700090E0887190708830910561F0893091058E
:109B80001CF4892B79F019C08031910529F0489790
:109B9000A1F406C081E001C080E48093140F0DC0E1
:109BA0008FEFFBCFE0913314F091341481918093C7
:109BB000140FF0933414E09333148A8190E080738F
:109BC000907054E0959587955A95E1F70E94B04CB6
:109BD000AC0190933214809331148A81282F30E0A5
:109BE000207C30702034310509F46FC021343105F8
:109BF00024F4232B09F489C09EC020383105C1F01C
:109C0000203C310509F097C04115510509F428C1E0
:109C1000A5E1BFE0FA01329688E001900D928150F3
:109C2000E1F785E19FE06DE37FE20E94314583C06B
:109C3000A0913314B09134148C9187FD23C0411549
:109C4000510509F40DC1A5E1BFE0FA01329688E0A3
:109C500001900D928150E1F786E0EDE1FFE0DF0138
:109C60001D928A95E9F7E0913314F09134148191B3
:109C700091919093240F8093230FF0933414E093E9
:109C8000331459C080FDE2C011968C911197815018
:109C9000823008F0DBC08FEF8093150F8C91869592
:109CA0008F708093160F8DE0E7E1FFE0EF011992CE
:109CB0008A95E9F711968C9111978093240F12964B
:109CC000B0933414A093331436C04115510509F4F0
:109CD000C7C0A5E1BFE0FA01329688E001900D927D
:109CE0008150E1F7ADE1BFE08091331490913414DD
:109CF0009C01F90188E001900D928150E1F780917B
:109D0000331490913414089612C0A5E1BFE08091FD
:109D10003314909134149C01F90180E101900D926B
:109D20008150E1F7809133149091341440969093D0
:109D300034148093331480910A0F0091080F10910E
:109D4000090F080F111DF801828183700E94B04C29
:109D5000AC019093321480933114D80112968C91F7
:109D6000282F30E02C7030702430310509F475C094
:109D70002530310524F4232B09F495C0AAC02830DE
:109D80003105C1F02C30310509F0A3C04115510552
:109D900009F466C0A5E2BFE0FA01329688E00190BE
:109DA0000D928150E1F785E29FE06FE37FE20E9430
:109DB00031458FC0A0913314B09134148C9187FD3C
:109DC00023C04115510509F44BC0A5E2BFE0FA01DB
:109DD000329688E001900D928150E1F786E0EDE245
:109DE000FFE0EF0119928A95E9F7E0913314F091C1
:109DF0003414819191919093340F8093330FF093A9
:109E00003414E093331465C080FD20C011968C910A
:109E1000119781508230D0F48FEF8093250F8C9171
:109E200086958F708093260F8DE0E7E2FFE0EF01CB
:109E300019928A95E9F711968C9111978093340FB6
:109E40001296B0933414A093331443C0E0910201EE
:109E5000F09103018FE099E0A9C04115510539F453
:109E6000E0910201F09103018AED98E09FC0A5E224
:109E7000BFE0FA01329688E001900D928150E1F73F
:109E8000ADE2BFE080913314909134149C01F9014C
:109E900088E001900D928150E1F780913314909108
:109EA0003414089612C0A5E2BFE08091331490915B
:109EB00034149C01F90180E101900D928150E1F789
:109EC000809133149091341440969093341480937D
:109ED000331480910C0F885D80930C0F80910A0FD2
:109EE000E091080FF091090FE80FF11D818185FFC6
:109EF0005FC0A0913314B09134148C918C7F883F53
:109F000009F056C081E18093130F8C91883F29F1AD
:109F10008B3F09F045C0EDE0FFE0B89611968C91BB
:109F2000119782958F7090E080559F409093350FE8
:109F3000818311968C91119790E08F70907080556D
:109F40009F409283838312968D919C911397909357
:109F50003C0F80933B0F149619C011968D919C91E4
:109F600012979093360F8093350F13968D919C9195
:109F700014979093380F8093370F15968D919C917D
:109F8000169790933C0F80933B0F1796B093341421
:109F9000A093331480910C0F885F80930C0F08C03E
:109FA000E0910201F091030183E599E009952EC04B
:109FB000209133148091080F281B20930A0FE1147D
:109FC000F10451F41092110F80910C0F885290916E
:109FD000432F890F821B0CC0E8EDFFEFEE0EFF1E32
:109FE000F092110F88E290E0E80EF91E8E2D885253
:109FF0008093120F8091130F813141F48091110FE2
:10A000009091120F90933A0F8093390FDF91CF9177
:10A010001F910F91FF90EF900895DF92EF92FF92C2
:10A020000F931F93DF93CF93CDB7DEB764970FB62F
:10A03000F894DEBF0FBECDBF8C01462F81E0809328
:10A04000E02F10920C0F10920A0F8091412F9091E7
:10A05000422F8093080F9093090F6093432F109223
:10A06000442F9801225F3F4FB90150E00E9466697A
:10A07000D8011B968D919C911C979A838983FE0130
:10A080003196818180933D2F898180933E2F19964F
:10A090008D919C911A979A838983818180933F2F18
:10A0A00089818093402F85E194E10E943F49892B6B
:10A0B00041F010920E1410920D1410921014109280
:10A0C0000F14E091080FF091090F808191810E9497
:10A0D00085218070987F892F9927803C910549F0D0
:10A0E000803E910521F1EE24FF24DD2400E010E004
:10A0F0003BC0E091080FF091090F808191810E948F
:10A100008521EFEFEE2EE7E0FE2EE822F922E09126
:10A11000080FF091090F828193810E9485218C01A3
:10A1200080910A0F8C5F80930A0FDD241DC0E0919F
:10A13000080FF091090FD480828193810E948521BC
:10A140008C01E091080FF091090F808191810E94AC
:10A1500085217FEFE72E77E0F72EE822F922809124
:10A160000A0F8B5F80930A0F80910F149091101447
:10A17000892B19F1E114F10409F4E9C080910D145F
:10A1800090910E14E816F90609F0E1C080911314BD
:10A19000909114148017910709F0D9C09091BB2FAA
:10A1A00080913D2F981709F0D2C09091BC2F8091DB
:10A1B0003E2F981709F0CBC01BC0E114F104C1F089
:10A1C000F0920E14E0920D141093141400931314D3
:10A1D00085E194E144EF51E060E070E00E9459496C
:10A1E00080913D2F8093BB2F80913E2F8093BC2F79
:10A1F00080910A0F853049F12091080F3091090FA5
:10A20000F901E80FF11DE081E33021F0E13409F0BC
:10A210009EC004C0C7010E94404D17C08F5F80934D
:10A220000A0FADE0BFE0F901E80FF11D88E20190EF
:10A230000D928150E1F780910A0F885D80930A0F9B
:10A2400080910C0F885D80930C0F90910A0F4091C4
:10A25000432F491B40930B0F2D2D30E063E0220F5D
:10A26000331F6A95E1F780910C0F280F311D235F92
:10A27000304FE091080FF091090FE90FF11DC9016E
:10A28000BF0150E00E946669EF28C9F080910F1469
:10A2900090911014892B31F480910C0F80930F143E
:10A2A0001092101420910B0F80910F1490911014A4
:10A2B000820F911D9093101480930F140BC0209166
:10A2C0000C0F80910B0F90E0820F911D90930E1454
:10A2D00080930D1420910F14309110142115310525
:10A2E00039F080910D1490910E142817390779F5E3
:10A2F0000CEF18E22DE03FE040910D1450910E1448
:10A30000C801B9010E94666960910D1470910E1424
:10A3100010920E1410920D141092101410920F142B
:10A320001092802810927F281B8290913D2F80915F
:10A330003E2F8C839D831C861E861D86C801AE0120
:10A340004D5F5F4F9E01245F3F4F0E94D35C649638
:10A350000FB6F894DEBF0FBECDBFCF91DF911F9136
:10A360000F91FF90EF90DF9008951F93CF93DF93AD
:10A37000EC011092351430C0812F90E0FC0133E0E5
:10A38000EE0FFF1F3A95E1F7880F991FE80FF91FAD
:10A39000E35EFB4E80818130E1F4212F30E0C90182
:10A3A000B3E0880F991FBA95E1F7220F331F820F90
:10A3B000931F815E9B4EBE0148E050E00E945969A8
:10A3C000009739F48AE0189F90011124235E3B4ED8
:10A3D00009C01F5F1093351410913514123060F2CC
:10A3E00020E030E0C901DF91CF911F9108950F93D4
:10A3F0001F93182F092FE091080FF091090F339642
:10A40000F0933414E0933314339780910A0FE80FDC
:10A41000F11D1282118280910A0FE091080FF091D4
:10A42000090FE80FF11D83E080838091FD28282F1C
:10A4300030E0C9018F709070892B09F03FC0809186
:10A44000FE289091FF28892BC9F580910A0FE09191
:10A45000080FF091090FE80FF11D8181806481835D
:10A460008091FC28282F30E0C9018F709070892BD3
:10A4700081F48091FD28807F61F480910A0FE09142
:10A48000080FF091090FE80FF11D81818068818329
:10A490005FC0E0913314F091341464E0220F331F55
:10A4A0006A95E1F78091FD2882958F70822B8083D9
:10A4B0008091331490913414019646C08091FC2809
:10A4C00090E08F709070892B51F5822F807F39F545
:10A4D00080910A0FE091080FF091090FE80FF11D2C
:10A4E000818180688183E0913314F09134149091DC
:10A4F000FD289F708091FC28807F982B9083E091AD
:10A500003314F09134148091FE289091FF289283A7
:10A5100081838091331490913414039615C0E09197
:10A520003314F09134148091FC289091FD28A0916F
:10A53000FE28B091FF2880839183A283B38380910A
:10A5400033149091341404969093341480933314FC
:10A5500080910229813161F480910A0FE091080F06
:10A56000F091090FE80FF11D8181806281830EC097
:10A57000E0913314F09134148083809133149091DE
:10A5800034140196909334148093331480910329EA
:10A59000803479F08F3FC9F0813011F580910A0F36
:10A5A000E091080FF091090FE80FF11D818188609B
:10A5B0000AC080910A0FE091080FF091090FE80F8F
:10A5C000F11D81818061818319C080910A0FE09122
:10A5D000080FF091090FE80FF11D81818861F3CF19
:10A5E000E0913314F091341480838091331490916E
:10A5F00034140196909334148093331484E099E2D8
:10A600000E94B551DC01909332148093311400976D
:10A6100009F49FC080910A0FE091080FF091090F93
:10A62000E80FF11D11968C918295807F9281892B84
:10A63000828320910C2930E08091BD2F90E08D7FA6
:10A6400028173907B9F590910D298091BE2F9817D9
:10A6500089F580910E29882369F580910F298F3F14
:10A6600049F5809110298E3F29F580911129882381
:10A6700009F58091E02FE82FF0E053E0EE0FFF1F87
:10A680005A95E1F7E957F74D909112298081981773
:10A6900089F4909113298181981761F480910A0FB0
:10A6A000E091080FF091090FE80FF11D8281806C95
:10A6B000828365C080910C2990910D29892B59F5D1
:10A6C00080910E2990910F29892B29F580911029CD
:10A6D00090911129892BF9F48091122987FD1BC0D3
:10A6E00080910A0FE091080FF091090FE80FF11D1A
:10A6F000828180688283E0913314F09134148091D8
:10A700001229909113299183808380913314909121
:10A710003414029630C080910A0FE091080FF09136
:10A72000090FE80FF11D8281806482832091331428
:10A7300030913414C901DC01ECE0F9E288E00190C9
:10A740000D928150E1F78091331490913414089662
:10A7500012C080913314909134149C01D901E4E02B
:10A76000F9E280E101900D928150E1F7809133147C
:10A7700090913414409690933414809333148091C4
:10A7800014298F3F09F065C08091162990911729EF
:10A79000892B09F050C08091182990911929892B93
:10A7A00009F049C080911A2990911B29892B09F041
:10A7B00042C080911C2990911D29892BE1F580913F
:10A7C0001E2990911F29892BB1F580912029909104
:10A7D0002129892B81F580912229882361F5809197
:10A7E00023298150823038F580910A0FE091080FBB
:10A7F000F091090FE80FF11D828188608283E0915A
:10A800003314F091341480EA8083E0913314F09192
:10A8100034148091152990E08F709070880F991FE3
:10A820002081282B2083E0913314F09134148091FF
:10A83000232981838AC080913314909134149C0120
:10A84000D901E4E1F9E280E101900D928150E1F754
:10A85000ADC084E199E20E94B551DC0190933214BD
:10A8600080933114009709F494C080910A0FE0910D
:10A87000080FF091090FE80FF11D828111969C914C
:10A88000892B828320911C2930E08091BD2F90E09C
:10A890008D7F2817390771F590911D298091BE2F62
:10A8A000981741F580911E29882321F580911F2951
:10A8B0008F3F01F5809120298E3FE1F4809121297D
:10A8C0008823C1F4E12FF02F9091222980819817DD
:10A8D00089F4909123298181981761F480910A0F5E
:10A8E000E091080FF091090FE80FF11D82818C6053
:10A8F000828365C080911C2990911D29892B59F56F
:10A9000080911E2990911F29892B29F5809120295A
:10A9100090912129892BF9F48091222987FD1BC070
:10A9200080910A0FE091080FF091090FE80FF11DD7
:10A93000828188608283E0913314F0913414809195
:10A9400022299091232991838083809133149091BF
:10A950003414029630C080910A0FE091080FF091F4
:10A96000090FE80FF11D82818460828320913314E6
:10A9700030913414C901DC01ECE1F9E288E0019086
:10A980000D928150E1F78091331490913414089620
:10A9900012C080913314909134149C01D901E4E1E8
:10A9A000F9E280E101900D928150E1F7809133143A
:10A9B000909134144096909334148093331488E229
:10A9C00080930C0F80910229813109F064C090912D
:10A9D000242980912529805B904F0F9770F59091E5
:10A9E00026298091272920EF803B920730F18F5B49
:10A9F000904F18F5E0913314F09134148BEF80836D
:10AA0000E0913314F091341490912729905B809158
:10AA100025298295807F980F9183E0913314F091DE
:10AA2000341480912A2990912B29938382838091D9
:10AA3000331490913414049625C0E0913314F091AE
:10AA4000341488EF8083E0913314F09134148091B2
:10AA5000242990912529A0912629B0912729818325
:10AA60009283A383B483E0913314F09134148091E2
:10AA70002A2990912B299683858380913314909174
:10AA800034140796909334148093331480910C0FF0
:10AA9000885F80930C0F809133149091080F891B6D
:10AAA00080930A0F1F910F9108950F931F93CF93D7
:10AAB000DF93EC018B010E94B551892B31F1288580
:10AAC00030E08091BD2F90E08D7F28173907E9F4A1
:10AAD00099858091BE2F9817C1F48A858823A9F49F
:10AAE0008B858F3F91F48C858E3F79F48D858823FB
:10AAF00061F49E85F8018081981739F420E09F85E4
:10AB00008181981719F421E001C020E0822FDF91A4
:10AB1000CF911F910F910895FC014091412F5091C9
:10AB2000422F818190816091432F21E00E947E0E0F
:10AB30001092442F1092432F08950F931F93DF9389
:10AB4000CF9300D0CDB7DEB7FC0110920C0F10925E
:10AB50000A0F1092442F1092432F8091412F909111
:10AB6000422F9093090F8093080F309709F5809139
:10AB700002298A33D1F48091570C282F30E0F90153
:10AB8000EC5DF64D8081873881F4F901E85DF64D82
:10AB90008289898383898A83A4E1B9E2349680E13A
:10ABA00001900D928150E1F707C019821A8204C00A
:10ABB0008081898381818A838E010F5F1F4FC80145
:10ABC0000E94F75180910C0F482F50E0E0917F28B0
:10ABD000F0918028E41BF50BA0910A0F2A2F30E09A
:10ABE0008FE690E0821B930B6091080F7091090F24
:10ABF0008E179F0708F0B4C0CB0104964A2F50E08F
:10AC00000E946F69E091080FF091090F80917F28F1
:10AC100090918028906C9083818390911114809101
:10AC200012148283938380910A0F8C5F80930A0FA2
:10AC30004FE6481B487F40930B0FE80FF11D209112
:10AC40000C0F30E02450374DCF01B90150E00E9485
:10AC5000666920910A0F80910B0F90E0820F911D81
:10AC60009093442F8093432FC8010E948C552091CC
:10AC70000C0F80910B0F90E0820F911D9093101498
:10AC800080930F1485E080930A0FE091080FF091F4
:10AC9000090F80917F2890918028906E9083818306
:10ACA00088E680930B0F42C0A091080FB091090F66
:10ACB000CF0173E0969587957A95E1F714968C937A
:10ACC00014979A012E1B3F0B80910B0F90E02817D1
:10ACD000390720F4842F8E1B80930B0F80910A0F6D
:10ACE0009D01280F311D40910B0FE450F74DC90114
:10ACF000BF0150E00E94666920910A0F80910B0FFE
:10AD000090E0820F911D9093442F8093432FC801B0
:10AD10000E948C5520910B0F80910F14909110146C
:10AD2000820F911D9093101480930F14E0910F14D3
:10AD3000F091101440917F2850918028E417F50776
:10AD400008F4B2CF8091111490911214019690934F
:10AD50001214809311141092101410920F141CC02E
:10AD6000260F371F4450574DC901BA01AF010E9449
:10AD7000666920910A0F80917F2890918028820F28
:10AD8000911D20910C0F821B91099093442F809369
:10AD9000432FC8010E948C5581E00F900F90CF91F6
:10ADA000DF911F910F910895CF93DF932091E02FB2
:10ADB000E22FF0E0DF0124E0AA0FBB1F2A95E1F7A4
:10ADC000A054B04DEC0180E109900D928150E1F763
:10ADD00084E0EE0FFF1F8A95E1F7E054F04D8FEF0E
:10ADE0008787DF91CF910895FFCF0F931F93DF9354
:10ADF000CF93CDB7DEB728970FB6F894DEBF0FBE5E
:10AE0000CDBF80917F2890918028009709F41CC1C4
:10AE10008150954008F009C180911429909115291D
:10AE2000892B59F58091162990911729892B29F59D
:10AE30008091182990911929892BF9F480911A2968
:10AE400090911B29892BC9F480911C2990911D296F
:10AE5000892B99F480911E2990911F29892B69F4DF
:10AE60008091202990912129892B39F480912229E0
:10AE700090912329892B09F4D8C0809114298F3F00
:10AE800009F4D8C084E199E20E94AD32882341F0F0
:10AE900084E199E20E9477338C01E0E0F0E008C0A1
:10AEA0000E94E42EFC01009709F4BFC000811181CB
:10AEB0008091E02F813071F5EF2B01F520911C2955
:10AEC00030E08091BD2F90E08D7F28173907B1F4D5
:10AED00090911D298091BE2F981781F480911E2991
:10AEE000882361F480911F298F3F41F480912029AC
:10AEF0008E3F21F480912129882319F019821A822A
:10AF000006C0809122298983809123298A83CE01DA
:10AF1000019689C00115110531F0F801818D853048
:10AF200009F049C00AC084E199E260E070E040E0C5
:10AF300020E00E94D4338C0102C0F801118E84E01D
:10AF400099E260E840E00E94C943892B19F084E04F
:10AF500099E202C080E090E060E070E0A8010E9409
:10AF6000C2398091E02F90E029E730E0829FF00124
:10AF7000839FF00D929FF00D1124E55BF14D6585E7
:10AF800076858785908928EE33E040E050E00E9486
:10AF9000D76BCA01B90128EE33E040E050E00E94CF
:10AFA000A56BAB01BC01C80182960E94594981E0A2
:10AFB000F80182A73FC0882309F446C0823059F4C3
:10AFC00083E0F801818FC8014A9648E853E160E0C8
:10AFD00070E00E9459498091E02F90E029E730E02D
:10AFE000829FF001839FF00D929FF00D1124E55B8D
:10AFF000F14D658576858785908928EE33E040E0C0
:10B0000050E00E94D76BCA01B90128EE33E040E05E
:10B0100050E00E94A56BAB01BC01C80182960E9462
:10B020005949C80140960E94BF481092802810924A
:10B030007F280AC080E090E00E94BF4810928028DC
:10B0400010927F281092570C28960FB6F894DEBF06
:10B050000FBECDBFCF91DF911F910F9108950F9338
:10B060001F93DF93CF93CDB7DEB760970FB6F894F9
:10B07000DEBF0FBECDBF8C016436710520F0FC0130
:10B08000108280E032C0FB01EB5BF04D80818823B1
:10B0900019F4F801108229C04091072FDE011196A2
:10B0A00020E030E0413019F4EBE1F0E002C0E0E0F4
:10B0B000F0E0C901880F991FE80FF91FE452F14D24
:10B0C000808191818D939D932F5F3F4F2730310574
:10B0D00049F7CB010E948521988B8F87C801BE015B
:10B0E0006F5F7F4F0E94EF5B81E060960FB6F89430
:10B0F000DEBF0FBECDBFCF91DF911F910F9108959D
:10B10000CF92DF92EF92FF920F931F93DF93CF9333
:10B1100000D0CDB7DEB71092E02F04E119E28FEF37
:10B1200092E0909315298093142910921729109278
:10B130001629109219291092182910921B29109281
:10B140001A2910921D2910921C2910921F29109261
:10B150001E29109221291092202980E092E09093DC
:10B1600023298093222978EEE72E7FEFF72EE00E39
:10B17000F11E89E0D70197968C93C8014097B801DA
:10B180000E94AA411092570C80E68093FC28F70198
:10B1900011821382128281E186832FEF278360E17F
:10B1A000C62ED12CC00ED11E82E099E0D601139696
:10B1B0009C938E931297909325298093242980E065
:10B1C00094E315969C938E93149717961C921E9257
:10B1D0001697085E1F4F82E080932C2981E0F801CA
:10B1E000818313821282278B158A148A168A809192
:10B1F000E02F90E029E730E0829FA001839F500D6F
:10B20000929F500D1124FA01E55BF14D82A988232C
:10B21000B1F0D701D496FA01ED59F14D80E10190DA
:10B220000D928150E1F781E08093E02F0E945B2F27
:10B230001092E02FFC01B29681A181FD05C0109211
:10B24000802810927F282EC024E439E2AF0180E1EB
:10B25000DA010D90AD01D9010D929D018150C1F728
:10B260008089F80182A711A610A681E083A78CE54A
:10B2700090E09093802880937F2884E390E09A83E5
:10B2800089838A81D70114968C93149789811596A6
:10B290008C930E94492280959095F601978386832E
:10B2A0000E94F5560F900F90CF91DF911F910F9153
:10B2B000FF90EF90DF90CF9008950F93CF93DF939F
:10B2C0000E94E42E892BB9F58091E02FE82FF0E061
:10B2D000A4E0EE0FFF1FAA95E1F7E054F04D87853B
:10B2E0008823D9F01786CF0160E420E030E040E009
:10B2F00050E001E00E94E8308091E02F90E0E4E02F
:10B30000880F991FEA95E1F78054904D60E420E0A2
:10B3100030E040E050E00E949B458091E02F882380
:10B3200011F40E94BE488091E02F813021F487EF14
:10B330009EE20E94E94C8091E02F90E0C9E7D0E0C6
:10B340008C9FF0018D9FF00D9C9FF00D1124E55B0B
:10B35000F14D83898823A1F00E94E42E892B71F09E
:10B360008091E02F90E08C9FF0018D9FF00D9C9FCD
:10B37000F00D1124E55BF14D128A118A0E945543AC
:10B38000E0910201F091030182E999E00995809131
:10B39000E02F882339F4E0910201F09103018EE956
:10B3A00099E00BC0E0910201F0910301813019F4A2
:10B3B00087EA99E002C08FEA99E00995E0910201DD
:10B3C000F091030185EB99E009950E94D846DF9141
:10B3D000CF910F9108958091E02F813059F48091A1
:10B3E000072F8F3FD9F087EF9EE20E94E94C0E9421
:10B3F000971708958091D72E882381F48091072F85
:10B400008F3F61F480918E2E8F3F41F08091602EAE
:10B41000882321F08EE79EE20E94E94C08958091F6
:10B42000C528882359F080EA98E290939F2880935A
:10B430009E2882E00E9409230E94F5568091F128FF
:10B44000882359F08CEC98E290939F2880939E2853
:10B4500082E00E9409230E94F55608958091972862
:10B460008830E9F4E0913614F09137143097F9F010
:10B4700028E334E18091812890918228B901AF01BD
:10B480000E94666980913614909137149093FF2D35
:10B490008093FE2D10923714109236140895823046
:10B4A00031F41092FF2D1092FE2D1092A9140895E0
:10B4B000FF920F931F93DF93CF93CDB7DEB76997BA
:10B4C0000FB6F894DEBF0FBECDBFF82E092FE62FC2
:10B4D0006237D0F51091072F1130B1F580913614F5
:10B4E00090913714892B81F58091A914882361F5F7
:10B4F000609336141092371428E334E1C901BA017D
:10B500004E2F50E00E9466691093E02F80EF93EB7E
:10B510009A8B898B9C8B8B8B80E48D8BDE011196B3
:10B52000E7EFFEE280E101900D928150E1F70F8795
:10B53000F88ACE01019690939B2880939A2885E003
:10B540000E9409230E94F55669960FB6F894DEBF53
:10B550000FBECDBFCF91DF911F910F91FF90089546
:10B56000FC0120E090818181808391832E5F32965F
:10B570002031C1F70895992787FD90950E94586C56
:10B580008833A1F1893384F4843341F185333CF469
:10B59000823301F1833304F58133D1F417C086334C
:10B5A00009F187330CF51CC0833641F184363CF435
:10B5B000813601F1823604F5893351F419C085369C
:10B5C00009F18536ECF0863619F41EC081E0089545
:10B5D00080E0089582E0089583E0089584E008956E
:10B5E00085E0089586E0089587E0089588E008954D
:10B5F00089E008958AE008958BE008958CE008952D
:10B600008DE008958EE008958FE00895EF92FF9207
:10B610001F93CF93DF937C01EC0110E001C01F5F0B
:10B620008881992787FD90950E94446C892B19F495
:10B63000C0E0D0E022C02196143089F7F9CFF7019D
:10B6400080810E94BB5A90E0143029F4982F8827FB
:10B650009295907F0CC0133019F4982F882707C05B
:10B66000123029F424E0880F991F2A95E1F7C80FBA
:10B67000D91F11500894E11CF11C112301F7CE01D0
:10B68000DF91CF911F91FF90EF9008955F926F929D
:10B690007F928F929F92AF92BF92CF92DF92EF9262
:10B6A000FF920F931F93DF93CF9300D000D00F92A0
:10B6B000CDB7DEB74C016B018C019C01FF24A8E0E3
:10B6C000EA2EF8E05F2E5E010894A11CB11CE5E0B3
:10B6D0006E2E712C6C0E7D1E02C00F5F1F4FF80185
:10B6E00040814A3311F04423C1F7C801821B930BF8
:10B6F000059714F080E05EC0F80182918F010F5F22
:10B700001F4F8A3319F0D501F9012FC0442319F0D6
:10B71000F40190E00EC0EF2DF0E0EE0FFF1FEC0DF6
:10B72000FD1D11821082F39440C08A3309F49F5F9B
:10B73000319680818823C9F7252D291B9F2D822FC3
:10B740000AC0E92FF0E0EE0FFF1FEC0DFD1D118286
:10B75000108281509F5F8823A1F7E21AF20E0F5FDB
:10B760001F4F98011FC08D9331969E2F921B808191
:10B770008A3319F0A615B705B1F7F501E90FF11DE8
:10B780001082C5010E94065BEF2DF0E0EE0FFF1F57
:10B79000EC0DFD1D9183808398012F5F3F4FF39443
:10B7A000EA948901EE2009F09ACF80E0F8E0FF16D4
:10B7B00009F481E00F900F900F900F900F90CF91B0
:10B7C000DF911F910F91FF90EF90DF90CF90BF908E
:10B7D000AF909F908F907F906F905F900895AF9201
:10B7E000BF92CF92DF92EF92FF920F931F93CF936E
:10B7F000DF938C01EB016115710509F46BC0EE2438
:10B80000FF243DECC32E39E0D32E20E3A22E9AE391
:10B81000B92E88819981009779F5EE2069F540E08D
:10B820006F2D70E001C04F5F242F30E0F901EE0F63
:10B83000FF1FEC0FFD1F80819181892B29F4260FBA
:10B84000371F283031057CF3413039F4D801AD92EF
:10B850008D01F394229640E030C08F2D90E0840F4C
:10B86000911D089709F44150842F90E0880F991F8B
:10B87000C80FD91FF40E21C00E94852100D000D02E
:10B8800000D0EDB7FEB73196ADB7BEB712961C9398
:10B890000E931197D382C282958384830E94066A95
:10B8A000080F191F2296F3944E2DEDB7FEB736966A
:10B8B0000FB6F894FEBF0FBEEDBFF8E0FF1641F0E3
:10B8C000D801BD928D01B7E0BF1510F0E42EA1CFD5
:10B8D000F8011082DF91CF911F910F91FF90EF90AF
:10B8E000DF90CF90BF90AF900895AF92BF92CF926C
:10B8F000DF92EF92FF920F931F93DF93CF9300D0CD
:10B9000000D000D0CDB7DEB77C01E0910201F0910C
:10B91000030180ED99E0099500E010E06E010894C4
:10B92000C11CD11C42EDA42E49E0B42E00D000D0A1
:10B9300000D0ADB7BEB71196EDB7FEB7D282C182C7
:10B940001396BC92AE921297F701E00FF11F80811F
:10B9500014968C93149715961C920E94066A8DB7C4
:10B960009EB706960FB6F8949EBF0FBE8DBFE091AE
:10B970000201F0910301C60109950F5F1F4F0031CD
:10B980001105A1F626960FB6F894DEBF0FBECDBF07
:10B99000CF91DF911F910F91FF90EF90DF90CF90AB
:10B9A000BF90AF90089541E00E94025D0895CF934B
:10B9B000DF93EC018881833319F48981833389F023
:10B9C00020E030E0FE01E20FF31FD901A957B74D87
:10B9D00090818C91981799F42F5F3F4F2630310555
:10B9E00089F78C859D8586589D4D49F41092E02FEE
:10B9F0006E507040CE010E9640E00E94025DDF91D5
:10BA0000CF9108951F93CF93DF939C01EB01142FE7
:10BA100080917F2890918028892B19F02FEF3FEF9C
:10BA200013C08CEF98E2B901AE010E946F691093C8
:10BA3000E02FD0938028C0937F2881E00E940923C3
:10BA40000E94F55620E030E0C901DF91CF911F91AF
:10BA50000895FC0171A760A70895FC01768B658BA2
:10BA60000895A0919E28B0919F28109719F0FD018C
:10BA7000B89605C0E0919A28F0919B287596809120
:10BA8000972886FF22C050962D913C915197809126
:10BA9000AC149091AD148217930731F48091AE14D9
:10BAA0009091AF14009769F48091B0149091B11403
:10BAB0008217930751F48091B2149091B3140097B8
:10BAC00021F091838083138212822081318121159C
:10BAD000310521F082819381F9010995089500973C
:10BAE00049F090939F2880939E2883E00E94092329
:10BAF0000E94F5560895009749F090939B288093F3
:10BB00009A2885E00E9409230E94F5560895CF9354
:10BB1000DF93EC018091AE149091AF148C179D07C8
:10BB200071F48091AC149091AD140E943321109265
:10BB3000AD141092AC141092AF141092AE14809108
:10BB4000B2149091B3148C179D0771F48091B014C6
:10BB50009091B1140E9433211092B1141092B0143C
:10BB60001092B3141092B214E5ECF8E28381948140
:10BB70008C179D0719F4148213821082BC96CF0192
:10BB80008597885F984290F3E0E0FEE28589968988
:10BB90008C179D0711F4118A108A79968EE2E23390
:10BBA000F807A0F3DF91CF910895AC011092AB1488
:10BBB000ECEAF4E120E014C08081918184179507BC
:10BBC00069F4828193818617970741F42093AB141F
:10BBD00011821082CA010E943321089534962F5F8A
:10BBE000223050F32093AB140895CF93DF93EA01F2
:10BBF0000E94502CFC01009711F0D68BC58BCF0111
:10BC0000DF91CF9108950F931F93DF93CF93CDB71B
:10BC1000DEB760970FB6F894DEBF0FBECDBF8C01C4
:10BC2000AB018FEF92E09A8389831C821B821E8274
:10BC30001D8218861F821A8619861C861B861E8600
:10BC40001D8680E091E0988B8F87CE010196B80128
:10BC50000E94F55DFC01009711F0118B008BCF0164
:10BC600060960FB6F894DEBF0FBECDBFCF91DF91C7
:10BC70001F910F910895AC011092AA14ECEAF4E11F
:10BC800020E012C0322F3F5F80819181892B51F4D7
:10BC90002093AA145183408373836283CA010E9454
:10BCA000502108953496232F223060F32093AA1454
:10BCB00008950F931F93CF93DF938A010E948921E8
:10BCC000EC01009721F019A708A70E946F5DCE0133
:10BCD000DF91CF911F910F910895CF92DF92EF9254
:10BCE000FF920F931F93DF93CF93CDB7DEB7669785
:10BCF0000FB6F894DEBF0FBECDBF8C01FC012081D2
:10BD0000233381F48181833369F48281882331F480
:10BD10008091B81489838091B7142DC08F3F11F49E
:10BD2000F80112C08091BD2F8C708260281781F4B9
:10BD3000F80191818091BE2F981751F48281882358
:10BD400039F48381882321F484818983858113C018
:10BD5000F8018281882309F04CC08381882309F08F
:10BD600048C08481882309F044C08581882309F074
:10BD700040C0298381818A83F8018485958586580E
:10BD80009D4DB9F5DE011996ECEFF8E28EE00190D9
:10BD90000D928150E1F792EFE92E9FEFF92EE60E1A
:10BDA000F71EF0928028E0927F288EE0C82ED12CDA
:10BDB000C00ED11E8CEF98E2B601A7010E946F69F8
:10BDC000CE0101960E949D5528E20C3F120769F4AE
:10BDD000C601B801A7010E946F69D801FE0139961A
:10BDE0008EE001900D928150E1F710928028109220
:10BDF0007F2866960FB6F894DEBF0FBECDBFCF91F9
:10BE0000DF911F910F91FF90EF90DF90CF900895F9
:10BE1000EF92FF920F931F93CF93DF939C018B01BF
:10BE20007A018CEF98E2B901A8010E946F69109223
:10BE3000E02F809114298F3F09F4B4C084E199E286
:10BE40000E94AD32882331F084E199E20E94773379
:10BE5000EC0108C00E94E42EFC01009709F4E9C03F
:10BE6000C081D181209729F0898D853009F047C0A4
:10BE70000AC084E199E260E070E040E020E00E94C6
:10BE8000D433EC0101C0198E84E099E260E840E00F
:10BE90000E94C943892B19F084E099E202C080E036
:10BEA00090E060E070E0AE010E94C2398091E02F26
:10BEB00090E029E730E0829FF001839FF00D929F90
:10BEC000F00D1124E55BF14D6585768587859089B8
:10BED00028EE33E040E050E00E94D76BCA01B90180
:10BEE00028EE33E040E050E00E94A56BAB01BC01BE
:10BEF000CE0182960E94594981E08AA75AC08823C0
:10BF000009F497C0823051F483E0898FCE014A96BC
:10BF100048E853E160E070E00E9459498091E02FC9
:10BF200090E029E730E0829FF001839FF00D929F1F
:10BF3000F00D1124E55BF14D658576858785908947
:10BF400028EE33E040E050E00E94D76BCA01B9010F
:10BF500028EE33E040E050E00E94A56BAB01BC014D
:10BF6000CE0182960E9459498AE099E26CEF78E20C
:10BF7000A8010E946F69809122298F3FD1F08889A2
:10BF80008093FC2889898093FD288A898093FE28E4
:10BF90008B898093FF288C89809300298D898093D9
:10BFA000012907C08AE099E26CEF78E2A8010E94BB
:10BFB0006F69809122298F3FE9F483E38093FC2805
:10BFC0008093FD2880912E298093FE2880912F292F
:10BFD0008093FF2880913029809300298091312916
:10BFE00080930129A6EBB4E1F70189E001900D925D
:10BFF0008150E1F78091BD2F8C708260809302297F
:10C000008091BE2F80930329109204291092052954
:10C01000F70182818093062981818093072986E830
:10C02000809308298DED8093092910928028109221
:10C030007F28DF91CF911F910F91FF90EF9008958E
:10C0400008951092C2141092C11408957F928F9295
:10C050009F92AF92BF92CF92DF92EF92FF920F9397
:10C060001F93CF93DF93EC017B01E8E2FAE000E05D
:10C0700010E02FEDC22E29E0D22E9FE3792E89ED1C
:10C08000882E89E0982EB4C05F010894A11CB11CD1
:10C09000853209F0A8C08181882309F4B0C08834B2
:10C0A00009F43FC089343CF4853209F494C08234E9
:10C0B00009F093C078C08C3409F45DC0843509F070
:10C0C0008CC0C701801B910B06970CF489C08DB7FB
:10C0D0009EB708970FB6F8949EBF0FBE8DBFEDB701
:10C0E000FEB73196ADB7BEB71296DC93CE931197DB
:10C0F000938282828091240A9091250A9583848379
:10C100008091260A9091270A978386830E94066A67
:10C1100090E0C80FD91F080F191F8DB79EB708965A
:10C1200024C0C701801B910B06970CF459C000D0A6
:10C1300000D000D0EDB7FEB73196ADB7BEB71296BE
:10C14000DC93CE931197D382C2828091200A909182
:10C15000210A958384830E94066A90E0C80FD91F44
:10C16000080F191F8DB79EB706960FB6F8949EBF9D
:10C170000FBE8DBF35C0C701801B910B069784F1A0
:10C1800000D000D000D0EDB7FEB73196ADB7BEB746
:10C190001296DC93CE931197D382C2828091220AA9
:10C1A0009091230AD6CFC701801B910B0697C4F04C
:10C1B00000D000D000D0EDB7FEB73196ADB7BEB716
:10C1C0001296DC93CE931197D382C2828091BF14D2
:10C1D0009091C014BECF899301C079920F5F1F4F19
:10C1E000F501319605C08993F5010894E11CF11C15
:10C1F0008081882321F00E151F050CF445CF18828D
:10C2000098012F5F3F4FC901DF91CF911F910F918F
:10C21000FF90EF90DF90CF90BF90AF909F908F9066
:10C220007F9008950F931F93DF93CF93CDB7DEB721
:10C23000E2970FB6F894DEBF0FBECDBF8E010F5F41
:10C240001F4FC80162E370E00E9426608091C31412
:10C25000882349F100D000D000D0EDB7FEB7319669
:10C2600080919C2890919D28ADB7BEB712969C9363
:10C270008E93119782EE99E09383828315830483D2
:10C280000E94066ABC018DB79EB706960FB6F89459
:10C290009EBF0FBE8DBF80919C2890919D280E94CB
:10C2A0008E221092C314E2960FB6F894DEBF0FBE32
:10C2B000CDBFCF91DF911F910F91089540919728A5
:10C2C000242F30E046FF06C081E090E09093C21436
:10C2D0008093C11420733070232B11F447FF02C0E8
:10C2E0000E94216080919728282F30E082FD09C0AC
:10C2F000C90183709070892B21F428743070232B2E
:10C3000011F00E9412610895BC01FC01019000200F
:10C31000E9F73197E81BF90BE33310F080E008955B
:10C3200088E29AE00E94886981E008958EE591E6AE
:10C330000E94875D0895A0E1BAE0FC0180E10190D0
:10C340000D928150E1F78EE591E60E94875D80E1D4
:10C350009AE060E070E54EE551E60E94595E08956E
:10C360008091C1149091C214892B41F480E19AE02C
:10C3700060E070E54EE551E60E94595E81E08093F1
:10C38000C3148EE190E060EB71E60E94C40B089547
:10C390000E94B0610895FC01E053F84F1192119290
:10C3A00080ED97E0918380830895FC01DC01A05328
:10C3B000B84F8D919C911197E80FF91F60830196FA
:10C3C0008D939C9381E090E00895682F89E195E139
:10C3D0000E94D5610895FC01E053F84F808191815E
:10C3E000089508950F931F93CF93DF938C0100530B
:10C3F000184FE801A991B9918E01E881F981025D98
:10C400001740EA1BFB0BEA01E417F5070CF4EF01F8
:10C4100098012A0F3B1FC901AE010E946669F8010D
:10C42000E053F84F808191818C0F9D1F9183808311
:10C43000CE01DF91CF911F910F910895DF93CF939C
:10C4400000D000D0CDB7DEB79FEF99838A836B838E
:10C450001C8289E195E1BE016F5F7F4F44E050E0AF
:10C460000E94F2610F900F900F900F90CF91DF918B
:10C470000895EF92FF920F931F93CF93DF938C0158
:10C48000DB017A01E9011616170644F4FC01E60FF8
:10C49000F71F319780818A3009F411971C161D0609
:10C4A00044F4F701EC0FFD1F319780818A3009F4C5
:10C4B000219789E195E1B801AD010E94F26189E11E
:10C4C00095E1B701AE010E94F26189E195E16AE56B
:10C4D0007AE042E050E00E94F261DF91CF911F913B
:10C4E0000F91FF90EF9008950F931F93CF93DF93D9
:10C4F000EC01C053D84FE881F981C05DD7408B0172
:10C50000E617F7070CF48F01E01BF10B9E01200FDB
:10C51000311FCE01B901AF010E946669FE01E053EF
:10C52000F84F80819181801B910B91838083DF91F3
:10C53000CF911F910F910895609116157091171565
:10C5400089E195E10E9474621092171510921615F8
:10C5500008959C01CB01B9010E9466690895CF93AB
:10C56000DF9389E195E10E94EB61EC01E0919E2867
:10C57000F0919F28868D978DC817D90708F0EC0198
:10C5800060919C2870919D2889E195E1AE010E94FF
:10C59000A96280919C2890919D28BE010E948E22C4
:10C5A000D0931715C0931615DF91CF91089580E0B1
:10C5B00097E16DE873E60E943B5E89E195E10E9498
:10C5C000CB610895BC01DC010D900020E9F71197C3
:10C5D000A81BB90B89E195E1AD010E94F2610895B4
:10C5E000BC01DC010D900020E9F71197A81BB90BE5
:10C5F00089E195E1AD010E94F261089580E090E04B
:10C600000E94730680E090E00E947C068DE893E62D
:10C610000E94875D0895833029F40E94FE620E9483
:10C62000D76208950E9489070895BF92CF92DF9242
:10C63000EF92FF920F931F93CF93DF9300917F2888
:10C6400010918028C0919C28D0919D28BB24B39440
:10C6500033E0C32E24E0D22E95E0E92E82E0F82EBE
:10C660004AC0688180911815823061F1833028F4C6
:10C670008823B1F18130E1F507C0843029F184309D
:10C6800008F18530A9F520C06F3F21F48FEF0E949B
:10C690000B6323C06C3F69F06D3F18F46B3FE9F406
:10C6A00005C06D3F49F06E3FC1F409C0F092181506
:10C6B0001FC0C09218151CC0D092181519C0E09266
:10C6C000181516C08EEF07C0613011F0633011F4F9
:10C6D0008BEF01C08CEF0E941E621092181508C0EB
:10C6E0006F3F19F4B092181503C0862F0E940B6398
:10C6F0002196015010400115110529F08091151562
:10C70000813508F4AECFDF91CF911F910F91FF904B
:10C71000EF90DF90CF90BF9008958091972886FF8B
:10C720001FC089E195E10E94CB611092151510920E
:10C73000181585EE91E60E94730680EF92E60E943E
:10C740007C06E0910201F09103018DE59AE00995E4
:10C750008BEF61E00E941E628BEF63E00E941E621D
:10C7600080911815863071F41092181580E180932D
:10C77000972880E090E00E94730680E090E00E949D
:10C780007C06089590919728892F807311F497FF64
:10C7900008C080E090E00E94730680E090E00E9474
:10C7A0007C068091972880FF02C00E949C62809145
:10C7B000972881FF02C00E94156380919728282F37
:10C7C00030E082FD09C0C90183709070892B21F48B
:10C7D00028743070232B11F00E94AF620895A1E1FC
:10C7E000B0E0E5EFF3E60C94F96B3C017F876E87D0
:10C7F0006A01FC0117821682838181FD03C06FEFFD
:10C800007FEF71C39E012F5F3F4F398B288BF30160
:10C810002381EE85FF8523FD859123FF8191FF878D
:10C82000EE87882309F45CC3853251F4EE85FF85D9
:10C8300023FD859123FF8191FF87EE87853229F4BF
:10C8400090E0B3010E94DA69E2CF982F10E08824CB
:10C8500099241032B0F49B3269F09C3228F4903263
:10C8600051F0933271F40BC09D3239F0903349F49A
:10C87000116028C01260146025C0186023C01061C8
:10C8800021C017FD2AC0892F80538A3078F416FF03
:10C8900006C0FAE09F9E902C1124980E13C03AE037
:10C8A000839E802C1124880E10620CC09E3221F4CD
:10C8B00016FD16C3106406C09C3611F4106802C041
:10C8C000983659F4EE85FF8523FD959123FF9191CC
:10C8D000FF87EE87992309F0BCCF892F85548330D9
:10C8E00020F4812F8061905E07C0892F85568330A8
:10C8F00008F0A1C1812F8F7E86FD02C076E0972EC1
:10C900006FE3F62EF822953619F4F0E4FF2A07C0FB
:10C91000963619F420E8F22A02C091109A94F7FE94
:10C920000BC03BE3391520F427E05CE3B52E0EC0C5
:10C93000B92CB39427E00AC047E0491528F427E052
:10C94000BB2447E0942E02C0292DBB24C6010496C7
:10C950009D878C87F6016081718182819381AE0110
:10C960004F5F5F4F0B2D0E9476686C010981202E6E
:10C97000332400FF04C003FD02C01DE209C0F1FE24
:10C9800002C01BE205C0F2FC02C010E001C010E2D0
:10C99000C1018C709070892BB9F1112311F483E0DF
:10C9A00001C084E0881510F088240AC0881AF3FCBE
:10C9B00007C080E290E0B3010E94DA698A94C9F767
:10C9C000112329F0812F90E0B3010E94DA6923FE40
:10C9D00003C00CE810E00EC000E910E00BC0E11449
:10C9E000F10409F0805290E0B3010E94DA690F5F10
:10C9F0001F4F05C0EF2CFF24F0E1EF22FF24F801C8
:10CA00008491882361F714C1F7FE12C0BC0C24FE88
:10CA100004C08A81813309F4BA941B141CF0BB242E
:10CA2000B3942DC0F8E0FB1550F538E0B32E27C0C5
:10CA3000F6FC25C0892D90E08C159D054CF02CEF5F
:10CA4000C2162FEFD20624F030E8F32A01C09A94E0
:10CA5000992049F0E2E0F0E0EC0FFD1FE90DF11D37
:10CA600080818033A1F3F7FE0AC0B92CB394892DDD
:10CA700090E0C816D90614F0992401C09C18F7FC60
:10CA800003C025E030E009C01C141D041CF021E0A7
:10CA900030E003C096012F5F3F4F112311F02F5F4D
:10CAA0003F4F992029F0892D90E00196280F391FDA
:10CAB000882D90E02817390714F0882401C0821AC5
:10CAC0004F2C5524C20189709070892B39F008C011
:10CAD00080E290E0B3010E94DA698A948820C1F76D
:10CAE000112329F0812F90E0B3010E94DA6943FEFF
:10CAF00007C008C080E390E0B3010E94DA698A941D
:10CB00008820C1F7F7FE46C08601D7FE02C000E0CC
:10CB100010E076010894E11CF11CE01AF10A41E0F2
:10CB200050E04C0F5D1FE40EF51E26014B18510816
:10CB3000892D90E0AA24BB24A81AB90A5FEF0F3F01
:10CB4000150729F48EE290E0B3010E94DA69C0165D
:10CB5000D10634F0401651061CF4F701808101C063
:10CB600080E3015010400894E11CF11C0A151B05DC
:10CB70002CF090E0B3010E94DA69E0CF0C151D059E
:10CB800039F49A81963318F4953311F424FE81E335
:10CB900090E04BC08A81813309F00F7E90E0B301B1
:10CBA0000E94DA699920A1F08EE290E0B3010E9420
:10CBB000DA6912E0E1E0F0E0EC0FFD1FE10FF11D9A
:10CBC0001F5F808190E0B3010E94DA699A9491F727
:10CBD00044FC03C085E690E002C085E490E0B30128
:10CBE0000E94DA69D7FC05C0C114D10441F404FFE6
:10CBF00006C0D094C194D108D3948DE201C08BE2D9
:10CC000090E0B3010E94DA6980E305C08F5F26EFF0
:10CC10003FEFC20ED31E3AE0C316D104BCF790E03A
:10CC2000B3010E94DA69C601C096B3010E94DA69B5
:10CC3000CC84DD8452C1933631F0933799F093352B
:10CC400009F059C023C0F601808189835E010894F0
:10CC5000A11CB11C22E030E0C20ED31E21E0E22E66
:10CC6000F12C12C0F601A080B18016FD03C06FEF59
:10CC70007FEF02C0692D70E022E030E0C20ED31ECB
:10CC8000C5010E948F697C011F7713C0F601A08047
:10CC9000B18016FD03C06FEF7FEF02C0692D70E019
:10CCA00022E030E0C20ED31EC5010E944E697C0115
:10CCB000106813FF07C01BC080E290E0B3010E9420
:10CCC000DA698A94882D90E0E816F906A8F30FC077
:10CCD000F50117FD859117FF81915F0190E0B30188
:10CCE0000E94DA6981108A940894E108F108E1143D
:10CCF000F10471F7F2C0943611F0993689F517FFF7
:10CD000008C0F601208131814281538184E090E0A6
:10CD10000AC0F601808191819C01442737FD40952E
:10CD2000542F82E090E0C80ED91E9FE6F92EF12222
:10CD300057FF09C050954095309521953F4F4F4F73
:10CD40005F4F90E8F92ACA01B901AE014F5F5F4F0A
:10CD50002AE030E00E942A6AE82EE889EE1A41C0F3
:10CD6000953721F41F7E2AE030E01CC0197F9F36E2
:10CD700061F0903720F4983509F0B2C00FC09037B9
:10CD800039F0983709F0ACC004C028E030E00AC0A0
:10CD9000106114FD146020E130E004C014FD166041
:10CDA00020E132E017FF08C0F601608171818281C5
:10CDB000938144E050E008C0F60180819181BC017C
:10CDC00080E090E042E050E0C40ED51EAE014F5F1F
:10CDD0005F4F0E942A6AE82E5889E51A8FE7F82EDD
:10CDE000F122F6FE0BC08EEFF822E91438F4F4FEBF
:10CDF00007C0F2FC05C09FEEF92202C01E2D01C043
:10CE0000192DF4FE0DC0FE01EE0DF11D8081803361
:10CE100019F4E9EEFE2208C01F5FF2FE05C003C050
:10CE20008F2D867809F01F5F0F2DF3FC14C0F0FEE4
:10CE30000FC0181510F09E2C0BC09E2C980C911A48
:10CE4000182D06C080E290E0B3010E94DA691F5FEE
:10CE50001815C0F304C0181510F4811A01C08824F5
:10CE600004FF0FC080E390E0B3010E94DA6902FF83
:10CE70001DC001FD03C088E790E00EC088E590E08A
:10CE80000BC0802F867891F001FF02C08BE201C0B9
:10CE900080E2F7FC8DE290E0B3010E94DA6906C0FF
:10CEA00080E390E0B3010E94DA699A94E914C0F338
:10CEB000EA94E1E0F0E0EC0FFD1FEE0DF11D808142
:10CEC00090E0B3010E94DA69EE2091F706C080E29B
:10CED00090E0B3010E94DA698A948820C1F797CC68
:10CEE000F30166817781CB016196E2E10C94156CC8
:10CEF000EF92FF920F93DF93CF93CDB7DEB760979A
:10CF00000FB6F894DEBF0FBECDBFA82F002309F4E3
:10CF100061C07E010894E11CF11C88E0F7011192C8
:10CF20008A95E9F729833A834B835C836D837E83FB
:10CF3000AF83988780E2801BE82FFF27E7FDF095FD
:10CF40004D815E816F817885181684F01D861E865E
:10CF50001F86188A882799278E1B9F0B04C07695F9
:10CF60006795579547958A95D2F728C0202F332784
:10CF700027FD3095DB01CA01022E04C0B695A795A6
:10CF8000979587950A94D2F78D879E87AF87B88B40
:10CF900004C0440F551F661F771FEA95D2F7898199
:10CFA0009A81AB81BC8104C0B695A795979587956A
:10CFB0002A95D2F7482B592B6A2B7B2B49875A8706
:10CFC0006B877C8729853A854B855C856D857E8559
:10CFD000AF8598898A2F60960FB6F894DEBF0FBE92
:10CFE000CDBFCF91DF910F91FF90EF900895A0E01A
:10CFF000B0E0EDEFF7E60C94016CEC01A880B9808D
:10D00000CA80DB80A114B104C104D10441F484E2DC
:10D01000A82E89EDB82E8BE5C82E87E0D82EC60144
:10D02000B5012DE133EF41E050E00E94606C27EA4A
:10D0300031E440E050E00E94A56B7B018C01C60109
:10D04000B5012DE133EF41E050E00E94606CCA0170
:10D05000B9012CEE34EF4FEF5FEF0E94A56B6E0D20
:10D060007F1D801F911F97FF04C06150704080405A
:10D070009048688379838A839B839B013F77C901AA
:10D08000CDB7DEB7EAE00C941D6C0E94F7670895F7
:10D0900088EA9AE00E94F7670895A0E0B0E08093E4
:10D0A000A80A9093A90AA093AA0AB093AB0A08957C
:10D0B000FC0188279927E89421912032E9F329304F
:10D0C00010F02E30C8F32B3241F02D3239F4689431
:10D0D00004C00E94D269820F911D219120532A30F1
:10D0E000C0F31EF4909581959F4F0895283008F065
:10D0F00027E03327DA01990F311D87FD91600096F3
:10D100006105710539F432602E5F3D9330E32A9555
:10D11000E1F708959F3F30F080387105610509F00F
:10D120003C5F3C5F3D93913008F08068911DDF9338
:10D13000CF931F930F93FF92EF92192F987F96959D
:10D14000E92F96959695E90FFF27E251FF4F992712
:10D150003327EE24FF24A701E701059008940794E4
:10D1600028F4360FE71EF81E491F511D660F771F62
:10D17000881F991F0694A1F70590079428F4E70EDD
:10D18000F81E491F561FC11D770F881F991F661F64
:10D190000694A1F70590079428F4F80E491F561F2E
:10D1A000C71FD11D880F991F661F771F0694A1F70F
:10D1B0000590079420F4490F561FC71FD81F990FD9
:10D1C000661F771F881F0694A9F784911095177022
:10D1D00041F0D695C79557954795F794E7941A95DA
:10D1E000C1F7E4E9F0E068941590159135916591E7
:10D1F000959105907FE27395E118F10A430B560B68
:10D20000C90BD009C0F7E10CF11E431F561FC91FFF
:10D21000D01D7EF4703311F48A95E6CFE894015066
:10D2200030F0080F0AF40027021708F4202F239586
:10D23000022F7A3328F079E37D932A95E9F710C01D
:10D240007D932A9589F60694979567953795179556
:10D250001794E118F10A430B560BC90BD00998F04B
:10D2600023957E9173957A3308F070E37C932013B5
:10D27000B8F77E9170617D9330F0839571E37D9373
:10D2800070E32A95E1F71124EF90FF900F911F9121
:10D29000CF91DF91992787FD90950895FC01059026
:10D2A000615070400110D8F7809590958E0F9F1FA8
:10D2B0000895FB01DC0104C08D910190801921F4D7
:10D2C00041505040C8F7881B990B0895FB01DC01C1
:10D2D00002C001900D9241505040D8F70895681750
:10D2E000790768F4FB01DC01E40FF51FA40FB51FFB
:10D2F00002C002900E9241505040D8F708950C940D
:10D300006669DC0101C06D9341505040E0F708951B
:10D31000FB01DC0101900D920020E1F70895FC0172
:10D320006150704001900110D8F7809590958E0F54
:10D330009F1F0895A0E0B0E0E0EAF9E60C94036CCA
:10D340007C01EB018A01690109C0CE012196F60139
:10D350000995F70181937F010150104001151105D6
:10D36000A1F7CDB7DEB7E8E00C941F6CA0E0B0E009
:10D37000ECEBF9E60C94036CEC017B018A0169018A
:10D3800009C0CE012196F70161917F01F60109954F
:10D390000150104001151105A1F7CDB7DEB7E8E047
:10D3A0000C941F6C7AE0979F902D879F802D910D94
:10D3B000112408950F931F93CF93DF938C01EB01FA
:10D3C0008B8181FF1BC082FF0DC02E813F818C812C
:10D3D0009D812817390764F4E881F9810193F98365
:10D3E000E88306C0E885F985802F0995892B31F4FB
:10D3F0008E819F8101969F838E8302C00FEF1FEF66
:10D40000C801DF91CF911F910F910895AEE0B0E078
:10D41000ECE0FAE60C94076C0D891E8986E08C839B
:10D420001A8309838FEF9FE79E838D839E01275E7A
:10D430003F4FCE0101966F89788DA9010E94EF635D
:10D440002F813885020F131FF80110822E96E4E019
:10D450000C94236CFA01AA27283051F1203181F174
:10D46000E8946F936E7F6E5F7F4F8F4F9F4FAF4FEC
:10D47000B1E03ED0B4E03CD0670F781F891F9A1FFF
:10D48000A11D680F791F8A1F911DA11D6A0F711DB3
:10D49000811D911DA11D20D009F468943F912AE0BF
:10D4A000269F11243019305D3193DEF6CF010895A7
:10D4B000462F4770405D4193B3E00FD0C9F7F6CFD8
:10D4C000462F4F70405D4A3318F0495D31FD4052A0
:10D4D000419302D0A9F7EACFB4E0A6959795879536
:10D4E00077956795BA95C9F7009761057105089515
:10D4F0009B01AC010A2E06945795479537952795C1
:10D50000BA95C9F7620F731F841F951FA01D089558
:10D5100070D088F09F5790F0B92F9927B751A0F09D
:10D52000D1F0660F771F881F991F1AF0BA95C9F7B7
:10D5300012C0B13081F077D0B1E0089574C0672F88
:10D54000782F8827B85F39F0B93FCCF38695779567
:10D550006795B395D9F73EF4909580957095619550
:10D560007F4F8F4F9F4F0895E89409C097FB3EF47B
:10D5700090958095709561957F4F8F4F9F4F992320
:10D58000A9F0F92F96E9BB279395F695879577959E
:10D590006795B795F111F8CFFAF4BB0F11F460FF5E
:10D5A0001BC06F5F7F4F8F4F9F4F16C0882311F0B6
:10D5B00096E911C0772321F09EE8872F762F05C0CA
:10D5C000662371F096E8862F70E060E02AF09A9565
:10D5D000660F771F881FDAF7880F9695879597F95A
:10D5E000089557FD9058440F551F59F05F3F71F053
:10D5F0004795880F97FB991F61F09F3F79F08795BA
:10D600000895121613061406551FF2CF4695F1DF42
:10D6100008C0161617061806991FF1CF86957105D2
:10D62000610508940895E894BB2766277727CB0106
:10D6300097F908950BD078C069D028F06ED018F013
:10D64000952309F05AC05FC01124EECFCADFA0F3C2
:10D65000959FD1F3950F50E0551F629FF001729F87
:10D66000BB27F00DB11D639FAA27F00DB11DAA1FA6
:10D67000649F6627B00DA11D661F829F2227B00DF3
:10D68000A11D621F739FB00DA11D621F839FA00D7E
:10D69000611D221F749F3327A00D611D231F849FCE
:10D6A000600D211D822F762F6A2F11249F57504025
:10D6B0008AF0E1F088234AF0EE0FFF1FBB1F661FC0
:10D6C000771F881F91505040A9F79E3F510570F079
:10D6D00014C0AACF5F3FECF3983EDCF386957795B4
:10D6E0006795B795F795E7959F5FC1F7FE2B880F74
:10D6F000911D9695879597F9089597F99F6780E80A
:10D7000070E060E008959FEF80EC089500240A9493
:10D710001616170618060906089500240A9412160C
:10D720001306140605060895092E0394000C11F43F
:10D73000882352F0BB0F40F4BF2B11F460FF04C0EC
:10D740006F5F7F4F8F4F9F4F0895629FD001739FF0
:10D75000F001829FE00DF11D649FE00DF11D929F8D
:10D76000F00D839FF00D749FF00D659FF00D9927CC
:10D77000729FB00DE11DF91F639FB00DE11DF91FF0
:10D78000BD01CF011124089597FB092E07260AD069
:10D7900077FD04D065D006D000201AF4709561950D
:10D7A0007F4F0895F6F7909581959F4F0895A1E2D8
:10D7B0001A2EAA1BBB1BFD010DC0AA1FBB1FEE1F0B
:10D7C000FF1FA217B307E407F50720F0A21BB30B56
:10D7D000E40BF50B661F771F881F991F1A9469F7D2
:10D7E00060957095809590959B01AC01BD01CF012E
:10D7F00008952F923F924F925F926F927F928F92F5
:10D800009F92AF92BF92CF92DF92EF92FF920F93CF
:10D810001F93CF93DF93CDB7DEB7CA1BDB0B0FB6D9
:10D82000F894DEBF0FBECDBF09942A883988488896
:10D830005F846E847D848C849B84AA84B984C8842C
:10D84000DF80EE80FD800C811B81AA81B981CE0F23
:10D85000D11D0FB6F894DEBF0FBECDBFED01089508
:10D86000AA1BBB1B51E107C0AA1FBB1FA617B70706
:10D8700010F0A61BB70B881F991F5A95A9F7809522
:10D880009095BC01CD010895911106C080538A5036
:10D8900010F0865C06C0089599278827089585FDB5
:10D8A000FBCF80629111F8CF81568A51E0F708953D
:10D8B0009111089581548A5108F4805E855A089523
:10D8C00097FB092E05260ED057FD04D070DF0AD035
:10D8D000001C38F450954095309521953F4F4F4F9F
:10D8E0005F4F0895F6F790958095709561957F4FFD
:06D8F0008F4F9F4F0895C9
:10D8F600EC060A070000000000000000000000001F
:10D906003380E8030D0A643D64756D7020743D74C0
:10D9160061626C6520693D696E666F20703D706955
:10D926006E6720733D73747265616D20503D706142
:10D93600757365000D0A523D485454504320536593
:10D9460072766572204D3D48545450204D65737370
:10D9560061676500203A000D0A0D0A5245472044CA
:10D96600554D500D0A00252D313573202D202530BB
:10D97600325820000D0A000D0A50696E67696E67FD
:10D9860020636F6F72640D0A000D0A73686F7274FC
:10D99600203D20253034580D0A706172656E742062
:10D9A6003D20253034580D0A726F7574653D25305B
:10D9B60034580D0A006368616E203D2025640D0A07
:10D9C6000050414E204944203D2030780025780003
:10D9D600526164696F205374617465203D20005064
:10D9E6005F4F4E00425553595F52580042555359A6
:10D9F6005F54580052585F4F4E005452585F4F467E
:10DA06004600504C4C5F4F4E00425553595F52589A
:10DA16005F4141434B00425553595F54585F415251
:10DA260045540052585F4141434B5F4F4E00545896
:10DA36005F415245545F4F4E0052585F4F4E5F4E06
:10DA46004F434C4B0052585F4141434B5F4F4E5F33
:10DA56004E4F434C4B00425553595F52585F41411C
:10DA6600434B5F4E4F434C4B00556E6B6E6F776E5C
:10DA76003F006C6F6E67203D2030782530386C583B
:10DA86002530386C580D0A0066616C736500747237
:10DA96007565006173736F63203D2025730D0A4819
:10DAA6006F7073203D20253034580D0A0072616E68
:10DAB60064203D20253032580D0A00506172743DB5
:10DAC60052460025752C205265763D25640D0A00C8
:10DAD600536C656570203D2025730D0A00596573EA
:10DAE6000046726571203D2025644D487A0D0A0076
:10DAF600364C6F5750414E203D2025730D0A004489
:10DB0600656D6F206D6F6465203D2025730D0A00DD
:10DB16004E6F000D0A495076362045746865726E60
:10DB26006574204946203D20006E6F742079657427
:10DB36002076616C6964000D0A4950763620364CB1
:10DB46004F5750414E204946203D20000D0A456E54
:10DB56007465722073686F727420616464723A002F
:10DB66000D0A53747265616D206D6F646520746F64
:10DB760020616464723A000D0A5061757365642C05
:10DB86002070726573732027502720746F20756E7E
:10DB96007061757365000D0A495076362052656DC1
:10DBA6006F746520536572766572205B005D203A5E
:10DBB60020000D0A4368616E676564000D0A4E6FAA
:10DBC60074204368616E6765642E000D0A485454DC
:10DBD6005043204D657373616765205B000D0A53E2
:10DBE60063616E20676F6F642C2073656C65637468
:10DBF600206368616E20002564000D0A5363616E20
:10DC06002062616400726F7574000D0A4173736F50
:10DC160063696174696E6720746F2000206F6E20DF
:10DC2600636820002C20686F7073203D20000D0A69
:10DC360050696E6720726571756573742066726FC0
:10DC46006D206E6F646520000D0A4173736F636902
:10DC56006174656420746F200020617320000D0AD2
:10DC66004661696C656420746F206173736F6369C4
:10DC7600617465000D0A5374617274207363616E7A
:10DC8600000D0A537461727475702C204920616D01
:10DC960020726F757465722F656E642E000D0A4EC4
:10DCA6006F726D616C206D6F6465000D0A46616967
:10DCB6006C3D000D0A44726F70706564206368697C
:10DCC6006C6420626373207061636B657420736596
:10DCD6006E64206661696C65642E000D0A50696E7B
:10DCE6006720726573706F6E73652066726F6D2044
:10DCF60000204C51493D0020525353493D00545297
:10DD0600585F5354415455530000000000005452CC
:10DD1600585F53544154450000000000000054521F
:10DD2600585F4354524C5F300000000000005452CC
:10DD3600585F4354524C5F310000000000005048C9
:10DD4600595F54585F505752000000000000504879
:10DD5600595F52535349000000000000000050482C
:10DD6600595F45445F4C4556454C000000005048FD
:10DD7600595F43435F4343410000000000004343B3
:10DD8600415F5448524553000000000000005452C1
:10DD9600585F4354524C5F32000000000000495265
:10DDA600515F4D41534B00000000000000004952F6
:10DDB600515F535441545553000000000000565221
:10DDC60045475F4354524C000000000000004241AA
:10DDD600544D4F4E00000000000000000000584F58
:10DDE60053435F4354524C00000000000000525859
:10DDF6005F53594E0000000000000000000052462C
:10DE06005F4354524C5F3000000000000000584150
:10DE1600485F4354524C5F310000000000004654F6
:10DE26004E5F4354524C0000000000000000524672
:10DE36005F4354524C5F3100000000000000504C1C
:10DE46004C5F434600000000000000000000504CFC
:10DE56004C5F4443550000000000000000005041A4
:10DE660052545F4E554D000000000000000056451C
:10DE76005253494F4E5F4E554D00000000004D4134
:10DE86004E5F49445F3000000000000000004D4135
:10DE96004E5F49445F310000000000000000534817
:10DEA6004F52545F414444525F30000000005348D3
:10DEB6004F52545F414444525F31000000005041CC
:10DEC6004E5F49445F3000000000000000005041F2
:10DED6004E5F49445F3100000000000000004945E4
:10DEE60045455F414444525F30000000000049450B
:10DEF60045455F414444525F3100000000004945FA
:10DF060045455F414444525F3200000000004945E8
:10DF160045455F414444525F3300000000004945D7
:10DF260045455F414444525F3400000000004945C6
:10DF360045455F414444525F3500000000004945B5
:10DF460045455F414444525F3600000000004945A4
:10DF560045455F414444525F370000000000584188
:10DF6600485F4354524C5F300000000000004353AA
:10DF76004D415F534545445F300000000000435368
:10DF86004D415F534545445F310000000000435357
:10DF96004D415F4245000000000000000000010204
:10DFA600030405060708090C0E0F101112151617A3
:10DFB60018161A1B1C1D1E1F202122232425262766
:10DFC60028292A2B2C2D2E2F4368696C6420546136
:10DFD600626C6520666F72206E6F64652000253066
:10DFE60034580D0A000D0A000D0A52656D6F7669E8
:10DFF6006E67206368696C64206E6F646520002517
:10E0060078000D0A52652D616464696E6720636845
:10E01600696C642000416464696E67206368696C9A
:10E0260064206E6F646520000D0A526F757465205A
:10E036006461746120746F206368696C6400526F58
:10E04600757465206461746120646F776E20746FE7
:10E0560020002578000D0A526F757465206461747E
:10E0660061207570000D0A526563656976656420E6
:10E076006173736F6320726571000D0A53657420B6
:10E08600726F7574653D0014000F004E756D626504
:10E096007209095374617465090949502041646421
:10E0A600726573730D0A002020202564200909205B
:10E0B600202025640909000D0A0020010470F13CA6
:10E0C60001000000000000000000736963736C6FBC
:10E0D6007770616E20756E636F6D70726573735FB6
:10E0E6006864723A206572726F7220636F6E74652F
:10E0F6007874206E6F7420666F756E640D0A0073F7
:10E106006963736C6F7770616E20756E636F6D7087
:10E11600726573735F6864723A206572726F7220FB
:10E12600756E6B6E6F776E20636F6D70726573734D
:10E136006564206D636173742061646472657373D2
:10E146000D0A00736963736C6F7770616E20756E6C
:10E15600636F6D70726573735F6864723A2065727F
:10E16600726F7220756E737570706F72746564204D
:10E1760055445020636F6D7072657373696F6E0DD1
:10E186000A00525320446F6E65206F6E200045745E
:10E196006865726E657400364C6F7750414E004F5D
:10E1A60074686572002C2041737369676E6564201C
:10E1B6006164647265737365733A0D0A00257800AD
:10E1C60020002530327800060225642E25640025BD
:10E1D6006400474554202F6367692D62696E2F706E
:10E1E60075743F257320485454502F312E310D0A33
:10E1F600486F73743A203A3A310D0A0D0A0D0A0037
:10E20600200105C01000000B0000000000004BAB11
:10E216003C00230017000600543D25540000000072
:10E2260000000000000000000000000000000000E8
:10E2360000000000000000000000000000000000D8
:10E24600000000000000000000000D0A0057656C89
:10E25600636F6D6520746F20746865206D616769F2
:10E2660063616C20776F726C64206F662041746DF9
:10E27600656C277320364C6F5750414E204E6F64A5
:10E28600652E205072657373206920666F7220694F
:0CE296006E666F2E200D0A0001000000D3
:020000021000EC
:10FC00002F923F924F925F926F927F928F929F922C
:10FC1000AF92BF92CF92DF92EF92FF920F931F931A
:10FC2000DF93CF9300D000D0CDB7DEB7F8948091AA
:10FC3000712790917227A0917327B09174278983BF
:10FC40009A83AB83BC83612C712C91E0892E912C1B
:10FC500071E065E052C0F999FECF93E0F101409266
:10FC60005B0090935700E89507B600FCFDCFA1E13B
:10FC7000A0935700E89507B606FCFDCF6401530139
:10FC8000EE24FF248701CBBEF501279137914791E0
:10FC90005691D801C701820D931DA41DB51D090100
:10FCA000FC01A0935B0070935700E895112482E05B
:10FCB00090E0A0E0B0E0A80EB91ECA1EDB1EE80E60
:10FCC000F91E0A1F1B1F90E0E91691E0F90690E06B
:10FCD000090790E01907B9F680E091E0A0E0B0E0F4
:10FCE000680E791E8A1E9B1EF10140925B00609394
:10FCF0005700E89507B600FCFDCF212C312C8FEF83
:10FD0000482E8FEF582E260C371C481C591C898111
:10FD10009A81AB81BC81681679068A069B0608F435
:10FD20009ACF81E180935700E8952BE088E190E03D
:10FD30000FB6F894A895809360000FBE20936000E2
:10FD4000FFCFAF92BF92CF92DF92EF92FF920F93CD
:10FD50001F93CF93DF937B018C016A01AFB6F894B8
:10FD6000F999FECF83E0F70100935B008093570081
:10FD7000E89507B600FCFDCF40E050E060E070E0A1
:10FD8000BB24B394F6018081D181C0E09E01280F8D
:10FD9000311D82E090E0C80ED91EDB01CA018E0D34
:10FDA0009F1DA01FB11F0901FC01A0935B00B09231
:10FDB0005700E89511244E5F5F4F6F4F7F4F4030E3
:10FDC00091E0590790E0690790E07907D9F685E05E
:10FDD000F70100935B0080935700E89507B600FC9D
:10FDE000FDCF81E180935700E895AFBEDF91CF91C1
:10FDF0001F910F91FF90EF90DF90CF90BF90AF9049
:02FE0000089563
:00000001FF
